:100000000C94B91E0C94EA1E0C94EA1E0C94EA1E81
:100010000C94EA1E0C9412530C94EA1E0C94EA1EE3
:100020000C9493520C94EA1E0C94EA1E0C9459B54D
:100030000C94EA1E0D9435910C94EA1E0C94EA1E61
:100040000C94EA1E0D9446090C94EA1E0C94EA1EC8
:100050000C94EA1E0C94EA1E0D94771F0D94668989
:100060000C94EA1E0C94B42E0C94EA1E0C94EA1E16
:100070000C94EA1E0C94EA1E0C94EA1E0C94EA1EE0
:100080000C94EA1E0C94EA1E0C94EA1E0C94EA1ED0
:100090000C94EA1E0C94EA1E0C94EA1E0C94EA1EC0
:1000A0000C94EA1E0C94EA1E0C94EA1E0C94EA1EB0
:1000B0000C94EA1E0C94EA1E0C94EA1E0C94EA1EA0
:1000C0000C94EA1E0C94EA1E0C94EA1E0C94F42E76
:1000D0000C94EA1E0C94EA1E0C94EA1E0C94EA1E80
:1000E0000C94EA1E71015F01390175014D014B014C
:1000F000AF012F011F019301C5019D01A101C7019E
:100100007F0149012301A501410197016501AB016F
:10011000A3012101B30195015701BB013701CB01B7
:100120005D019F01A70135013301C1018901B701BB
:10013000CB01B10191016B018D018101A9016F0119
:100140001501190155015B0147012901B501B901EB
:10015000BF01310119013D014F015301084AD73B4D
:100160003BCE016E84BCBFFDC12F3D6C74319ABD86
:1001700056833DDA3D00C77F11BED9E4BB4C3E91AA
:100180006BAAAABE000000803F05A84CCDB2D44E99
:10019000B93836A9020C50B9918688083CA6AAAA9B
:1001A0002ABE000000803F07634236B79BD8A71ADB
:1001B00039685618AEBAAB558C1D3CB7CC5763BDE9
:1001C0006DEDFD753EF6177231BF000000803F08EF
:1001D000000000BE922449123EABAAAA2ABECDCC92
:1001E000CC4C3E00000080BEABAAAAAA3E00000094
:1001F00000BF000000803F0000000000084178D3ED
:10020000BB4387D1133D190E3CC3BD4282AD2B3E8B
:1002100068EC8276BED98FE1A93E4C80EFFFBE012B
:10022000C4FF7F3F0000000000000D945C8B0D9424
:10023000186A0D949A8B0D945D440D945F350D945E
:100240007C200D94DF530D9468530D946E2F0D9404
:10025000F47E0D94758B0D94BF6F0D9441560D94E3
:100260007A200D94878B0D94F38A0D94E98A0D946E
:10027000C58A0D9426200D94EB520D948D8B0D9410
:1002800052320D9490530D940C300D94B8500D943F
:10029000718B0D9458530D945C200D944E200D9449
:1002A000918B0D94874E0D94958B0D94678B0D94C7
:1002B000B18A0D94612C0D946B8B0D94CF8A0D94A3
:1002C0000A200D94B62D0D94E4510D94BA530D945B
:1002D000F72F0D94593E0D94348B0D94E1300D940D
:1002E000568B0D94FC1F0D943D780D9434200D9485
:1002F000280C0D940E500D94DF470D9423610D943E
:10030000D8200D94638B0D94E6440D948C620D946B
:10031000F34F0D940C8B0D9405500D94608B0D9440
:10032000FC4F0D942A8B0D9480200D94AC8A0D9473
:10033000B5530D94A3490D9424590D9490200D9418
:10034000D78A0D94AA200D94CF530D947B530D940E
:10035000DF8A0D94528B0D94BF530D94318C0D9404
:1003600076200D94208B0D94A78A0D94798B0D9493
:10037000168B0D947F8B0D94BB8A0D94AF5E0D94FC
:10038000838B0D94FD8A0D9474410D9482200D94FD
:10039000B8200D9406300D943E8B48617264636FF3
:1003A0006465642044656661756C7420536574747B
:1003B000696E6773204C6F616465640053746F727B
:1003C00065642073657474696E67732072657472F6
:1003D000696576656400202020452F44203D20007B
:1003E0002020204D393030204B004C696E65617201
:1003F00020616476616E63652073657474696E67ED
:10040000733A0046696C616D656E7420736574742F
:10041000696E67733A2044697361626C6564002099
:1004200020204D32303020440046696C616D656E8D
:10043000742073657474696E67733A002020204DD0
:100440003230392053004175746F2D5265747261DA
:1004500063743A20533D3020746F20646973616285
:100460006C652C203120746F20696E746572707217
:10047000657420657874727564652D6F6E6C792073
:100480006D6F766573206173207265747261637439
:1004900073206F72207265636F7665726965730091
:1004A0002046002020204D32303820530052656312
:1004B0006F7665723A20533D4578747261206C65A1
:1004C0006E67746820286D6D2920463A5370656503
:1004D0006420286D6D2F6D2900205A0020460020D1
:1004E00020204D323037205300526574726163749E
:1004F0003A20533D4C656E67746820286D6D292045
:10050000463A537065656420286D6D2F6D29205A19
:100510003A205A4C69667420286D6D2900204400E9
:100520002049002020204D333034205000504944D1
:1005300020686561746265642073657474696E67B0
:10054000733A002044002049002020204D333031F0
:100550002050005049442073657474696E67733A83
:1005600000205A0020590020204D323036205800FB
:10057000486F6D65206F666673657420286D6D2900
:100580003A00204500205A002059002058002042FF
:100590000020540020204D32303520530041647635
:1005A000616E636564207661726961626C65733A3D
:1005B00020533D4D696E20666565647261746520E7
:1005C000286D6D2F73292C20543D4D696E20747257
:1005D0006176656C20666565647261746520286D5E
:1005E0006D2F73292C20423D6D696E696D756D20EC
:1005F0007365676D656E742074696D6520286D7311
:10060000292C20583D6D6178696D756D20585920F1
:100610006A65726B20286D6D2F73292C20205A3D3E
:100620006D6178696D756D205A206A65726B20283E
:100630006D6D2F73292C2020453D6D6178696D7596
:100640006D2045206A65726B20286D6D2F7329001F
:1006500020540020204D3230342053004163636524
:100660006C65726174696F6E3A20533D61636365B6
:100670006C65726174696F6E2C20543D7265747282
:1006800061637420616363656C65726174696F6E28
:1006900000204500205A0020590020204D323031E2
:1006A0002058004D6178696D756D20416363656CFC
:1006B00065726174696F6E20286D6D2F7332293AEF
:1006C00000204500205A0020590020204D323033B0
:1006D0002058004D6178696D756D2066656564729E
:1006E0006174657320286D6D2F73293A00204500D1
:1006F000205A0020590020204D39322058005374D0
:100700006570732070657220756E69743A00536568
:100710007474696E67732053746F72656400454525
:1007200050524F4D204572726F72000020006D656F
:10073000736820626564206C6576656C696E673AE3
:10074000200029002C20002C200070687973696338
:10075000616C20636F6F7264696E617465733A20B7
:10076000280029002C20002C2000776F726C642058
:10077000636F6F7264696E617465733A202800203C
:1007800046002045004731205A004D3234004D329A
:10079000362053256C75004D3130362053004731DB
:1007A000204625640047312045312046343830004A
:1007B0004731205A0020463230303000205900475F
:1007C000312058004D383300506F736974696F6E73
:1007D00020726561642066726F6D20656570726F4E
:1007E0006D3A004D3233202573002E67636F00464B
:1007F000656564726174653A007265636F766572EF
:100800005F6D616368696E655F73746174655F6174
:10081000667465725F706F7765725F70616E696331
:100820002C20696E697469616C20007265636F7653
:1008300065725F6D616368696E655F73746174652D
:100840005F61667465725F706F7765725F70616E0D
:1008500069632C20696E697469616C20007265633C
:100860006F7665725F6D616368696E655F737461F1
:1008700074655F61667465725F706F7765725F70D3
:10088000616E69632C20696E697469616C20006314
:10089000757272656E745F706F736974696F6E5B89
:1008A0005A5F415849535D3A0043757272656E74E0
:1008B00020706F736974696F6E20595F4158495396
:1008C0003A0043757272656E7420706F7369746953
:1008D0006F6E20585F415849533A00416674657203
:1008E0002077616974696E6720666F722074656D28
:1008F000703A00473120452D3120463438300047CA
:10090000312045352046313230004D3833004D31ED
:10091000393020532564004D31303920532564008F
:1009200047323820582059004731205A3235204666
:10093000383030004D31343020532564004D313093
:10094000342053256400494E54340055564C4F20F2
:100950002D20656E6400737470730055564C4F0003
:1009600020423A0020453A00543A005A206C6976F9
:10097000652061646A757374206F7574206F6620DA
:1009800072616E67652E2053657474696E6720749A
:100990006F20302E20436C69636B20746F20636F6F
:1009A0006E74696E75652E005A206C6976652061DB
:1009B000646A757374206F7574206F662072616E3F
:1009C00067652E2053657474696E6720746F2030DC
:1009D0000020573A0020453A00543A004B494C4C0D
:1009E0003A20004175746F0020452F443D0041645A
:1009F00076616E6365204B3D002228322900443128
:100A00003030300047323820590047323820580003
:100A10005400496E76616C6964205420636F64658C
:100A20002E00496E76616C6964204D20636F6465A9
:100A30002E004D3232302053256900203A2000002C
:100A40004C414E472053454C20464F5243454400AD
:100A5000222831290020453A00205A3A0020593AEC
:100A60000020453A00205A3A0020593A00583A00EE
:100A700020002E0020423A0020453A00543A00203F
:100A8000413A0020503A002042403A0020403A00CB
:100A9000202F003A00205400202F0020423A00204E
:100AA0002F006F6B20543A002569206D696E2C2051
:100AB00025692073656300496E76616C6964204D19
:100AC00020636F6465004D65736820626564206C07
:100AD0006576656C696E67206E6F742061637469FA
:100AE00076652E000A002020000A4D65617375723C
:100AF000656420706F696E74733A000A5A207365DA
:100B000061726368206865696768743A20002C0028
:100B10004E756D20582C593A2000476F20686F6D34
:100B2000652066696E6973686564004D6573682049
:100B3000626564206C6576656C696E6720616374BC
:100B400069766174656400557073616D706C6520C1
:100B500066696E697368656400426564206C6576D9
:100B6000656C696E6720636F7272656374696F6E1E
:100B70002066696E697368656400206D6963726FD1
:100B80006E7300457863657373697665206265648A
:100B9000206C6576656C696E6720636F7272656341
:100BA00074696F6E3A2000626162797374657020B7
:100BB0006170706C69656400636C65616E2075704E
:100BC0002066696E69736865642000473238205773
:100BD00030003A200054656D7065726174757265FD
:100BE0002063616C6962726174696F6E20646F6EFC
:100BF000652E20436F6E74696E7565207769746821
:100C0000207072657373696E6720746865206B6EFF
:100C10006F622E0000205A20736869667420286D68
:100C20006D293A0050494E44412074656D706572DB
:100C300061747572653A2000002F36005374657038
:100C40003A200000205A20736869667420286D6D70
:100C5000293A0050494E44412074656D70657261B7
:100C6000747572653A20002F362028736B69707096
:100C700065642900537465703A2000005A45524F4C
:100C80003A20000073746172742074656D7065722F
:100C900061747572653A200050494E44412070726B
:100CA0006F62652063616C6962726174696F6E2046
:100CB000737461727400473238205730000A002084
:100CC0005A3A200020593A200020583A2000473252
:100CD000382C2066696E616C20004732382C206603
:100CE000696E616C20004732382C2066696E616C39
:100CF00020004732382C20696E697469616C2000CD
:100D00004732382C20696E697469616C200044395F
:100D10003939004D3239002055706C6F616420699B
:100D20006E2070726F677265737300696E697469A3
:100D3000616C207A737465707320616674657220CB
:100D400072657365743A2000696E697469616C201C
:100D50007A7374657073206F6E20706F7765722080
:100D600075703A2000466163746F72792052455362
:100D700045540020202020334420205072696E7496
:100D800065727320202020002020204F726967693F
:100D90006E616C205072757361202020004E6F765A
:100DA000202037203230313700436F6D70696C6519
:100DB000643A2000286E6F6E652C2064656661754C
:100DC0006C7420636F6E66696729004E6F76202011
:100DD0003720323031372032323A31323A35300032
:100DE00073746172740020202020334420205072DC
:100DF000696E7465727320202020002020204F72BD
:100E00006967696E616C20507275736120202000E3
:100E1000250020202020202000202020202020002D
:100E200045524153494E4720616C6C2064617461A6
:100E300000466163746F727920524553455400FF38
:100E4000FFFF0000A0400000A040000000400000A4
:100E50007F4300005E439AD9514300000000000028
:100E600040C19A99193E00007F43000052430000A0
:100E7000524300000000000040C19A99193E65638A
:100E8000686F3A004572726F723A0000002110429A
:100E90002063308440A550C660E770088129914ADC
:100EA000A16BB18CC1ADD1CEE1EFF1311210027363
:100EB000325222B5529442F772D662399318837B2C
:100EC000B35AA3BDD39CC3FFF3DEE36224433420B3
:100ED000040114E664C774A44485546AA54BB5287C
:100EE000850995EEE5CFF5ACC58DD5533672261143
:100EF000163006D776F6669556B4465BB77AA719CC
:100F0000973887DFF7FEE79DD7BCC7C448E558860A
:100F100068A7784008611802282338CCC9EDD98E1B
:100F2000E9AFF9488969990AA92BB9F55AD44AB7A2
:100F30007A966A711A500A333A122AFDDBDCCBBF6B
:100F4000FB9EEB799B588B3BBB1AABA66C877CE472
:100F50004CC55C222C033C600C411CAEED8FFDECBB
:100F6000CDCDDD2AAD0BBD688D499D977EB66ED582
:100F70005EF44E133E322E511E700E9FFFBEEFDD0B
:100F8000DFFCCF1BBF3AAF599F788F8891A981CAE8
:100F9000B1EBA10CD12DC14EF16FE18010A100C2C7
:100FA00030E3200450254046706760B9839893FB76
:100FB000A3DAB33DC31CD37FE35EF3B1029012F317
:100FC00022D2323542145277625672EAB5CBA5A8C6
:100FD0009589856EF54FE52CD50DC5E234C324A067
:100FE0001481046674476424540544DBA7FAB79956
:100FF00087B8975FE77EF71DC73CD7D326F23691B7
:1010000006B01657667676154634564CD96DC90E1D
:10101000F92FE9C899E9898AB9ABA9445865480606
:10102000782768C018E1088238A3287DCB5CDB3FB5
:10103000EB1EFBF98BD89BBBAB9ABB754A545A3756
:101040006A167AF10AD01AB32A923A2EFD0FED6C85
:10105000DD4DCDAABD8BADE89DC98D267C076C64A6
:101060005C454CA23C832CE01CC10C1FEF3EFF5D95
:10107000CF7CDF9BAFBABFD98FF89F176E367E55F6
:101080004E745E932EB23ED10EF01E7C3C3E5E2B23
:101090003D3F2F5B5D3B2C2A225C004D38342058AD
:1010A0002059205A2045004D3234004D323320253E
:1010B00073006175746F25692E67000A002F000A9E
:1010C000002E0044656C6574696F6E206661696C02
:1010D00065642C2046696C653A200046696C652081
:1010E00064656C657465643A002E002E002E002E37
:1010F000004E6F772066726573682066696C653A8A
:1011000020004E6F7720646F696E672066696C659A
:101110003A20002220706F73002220706172656E89
:10112000743A2200535542524F5554494E4520437C
:10113000414C4C207461726765743A220074727974
:10114000696E6720746F2063616C6C207375622D0B
:1011500067636F64652066696C657320776974687E
:1011600020746F6F206D616E79206C6576656C738D
:101170002E204D4158206C6576656C2069733A00CD
:10118000256920686F757273202569206D696E75F9
:101190007465730054494D454F55543A004D3131F3
:1011A000300046756C6C2052582042756666657238
:1011B0000022206661696C65643A20427566666546
:1011C000722066756C6C2100456E717565696E677D
:1011D00020746F207468652066726F6E743A2022E6
:1011E000002200456E717565696E6720746F20740A
:1011F00068652066726F6E743A2022002220666154
:10120000696C65643A204275666665722066756C25
:101210006C210022004D3630300050727573612011
:101220006933204D4B332072656164792E007A5FFB
:101230006D696E3A20007A5F6D61783A20005A201D
:101240004F666673657400795F6D696E3A20007948
:101250005F6D61783A200059657300785F6D696E43
:101260003A2000785F6D61783A20002057617463FE
:1012700068646F6720526573657400496E666F20FD
:1012800073637265656E0057616974696E67206685
:101290006F72206E6F7A7A6C6520616E6420626571
:1012A0006420636F6F6C696E6700576169742066B4
:1012B0006F7220757365722E2E2E00557365642033
:1012C000647572696E67207072696E7400556E6C19
:1012D0006F61642066696C616D656E7400556E6C3B
:1012E0006F6164696E672066696C616D656E74001C
:1012F000556E6B6E6F776E20636F6D6D616E643AC5
:1013000020220054756E650053442063617264208E
:101310005B466C73684169725D005344206361727F
:1013200064205B6E6F726D616C5D0054656D702E34
:101330002063616C2E205B4F4E5D0054656D702EF6
:101340002063616C2E205B4F46465D0054656D70D6
:10135000657261747572652063616C696272617433
:10136000696F6E2069732066696E69736865642EA3
:1013700020436C69636B20746F20636F6E74696EB9
:1013800075652E0054656D702E2063616C2E2020D3
:1013900020202020202020200054656D706572617F
:1013A0007475726500537570706F72740053746F4A
:1013B00070207072696E740053544F505045442E23
:1013C0002000537465707261746520746F6F2068BB
:1013D0006967683A2000546F74616C207072696E9E
:1013E000742074696D65203A00546F74616C2066D6
:1013F000696C616D656E74203A005072696E74207C
:1014000074696D653A20200046696C616D656E7483
:1014100020757365643A2020005374617469737495
:101420006963732020004572726F72202D207374DF
:1014300061746963206D656D6F72792068617320D6
:101440006265656E206F7665727772697474656E19
:101450000053706565640020536F66747761726530
:10146000205265736574004D6F6465202020202034
:101470005B73696C656E745D004D6F6465205B68BD
:1014800069676820706F7765725D0053686F7720B9
:10149000656E642073746F70730053657420746597
:1014A0006D70657261747572653A00536574746924
:1014B0006E677300576972696E67206572726F722A
:1014C0000053656C66207465737420737461727464
:1014D000202000506C6561736520636865636B2034
:1014E0003A0053656C662074657374204F4B004E50
:1014F0006F7420636F6E6E6563746564004D6F7406
:101500006F72004865617465722F546865726D6909
:1015100073746F720046616E207465737400536556
:101520006C6674657374206661696C656420200064
:101530004C65667420686F74656E642066616E3FEA
:101540000053656C6674657374206572726F7220E7
:101550002100456E6473746F70206E6F742068692B
:101560007400456E6473746F707300456E647374B9
:101570006F700046726F6E74207072696E742066B0
:10158000616E3F00436865636B696E67205A206136
:10159000786973202000436865636B696E67205922
:1015A0002061786973202000436865636B696E670A
:1015B00020582061786973202000436865636B6957
:1015C0006E6720686F74656E6420200043686563F1
:1015D0006B696E6720656E6473746F707300436827
:1015E00065636B696E67206265642020202020009F
:1015F000416C6C20636F7272656374202020202020
:101600002000426564202F204865617465720041A6
:10161000786973206C656E6774680041786973003F
:1016200053656C6674657374202020202020202070
:10163000200057726974696E6720746F2066696C48
:10164000653A2000766F6C756D652E696E69742041
:101650006661696C6564002053697A653A200043CD
:101660006172642072656D6F76656400534420700A
:1016700072696E74696E67206279746520006F709C
:10168000656E206661696C65642C2046696C653AFC
:1016900020006F70656E526F6F74206661696C65B3
:1016A00064004361726420696E73657274656400DE
:1016B000534420696E6974206661696C0046696CE8
:1016C000652073656C65637465640046696C6520AC
:1016D0006F70656E65643A20006572726F72207774
:1016E000726974696E6720746F2066696C65005357
:1016F000442063617264206F6B0043616E6E6F748F
:1017000020656E746572207375626469723A200098
:10171000526573756D696E67207072696E740052E0
:101720006573756D696E67207072696E74005265BD
:1017300073756D65207072696E7400526573656EA5
:10174000643A2000426C61636B6F7574206F636351
:1017500075727265642E205265636F7665722070B3
:1017600072696E743F005265636F766572696E6769
:10177000207072696E742020202000686F77746F6B
:101780002E707275736133642E636F6D00666F72B5
:10179000756D2E707275736133642E636F6D00709A
:1017A0007275736133642E636F6D005072696E746D
:1017B00020706175736564005072696E7420616297
:1017C0006F72746564005072696E7465722064692A
:1017D00073636F6E6E656374656400616E64207020
:1017E0007265737320746865206B6E6F620050724F
:1017F000656865617420746865206E6F7A7A6C65BF
:1018000021005072656865617400506F776572558C
:101810007000506C656173652077616974002020E9
:10182000506C616E6E65724275666665724279745F
:1018300065733A200050494E4441204865617469FF
:101840006E67005049442063616C2E2020202020C8
:10185000202020202020005049442063616C2E204D
:1018600066696E6973686564005049442063616C01
:101870006962726174696F6E005061757365207082
:1018800072696E7400506C616365206120736865D5
:101890006574206F6620706170657220756E646576
:1018A0007220746865206E6F7A7A6C652064757238
:1018B000696E67207468652063616C696272617427
:1018C000696F6E206F6620666972737420342070B1
:1018D0006F696E74732E20496620746865206E6F80
:1018E0007A7A6C65206361746368657320746865D7
:1018F0002070617065722C20706F776572206F6642
:101900006620746865207072696E74657220696DF6
:101910006D6564696174656C792E006F6B004F664C
:1019200066004E6F206D6F76652E004E6F2053441B
:101930002063617264004E6F7A7A6C650046696C50
:10194000616D656E74206E6F74206C6F6164656488
:1019500000436F6C6F72206E6F7420636C656172F0
:10196000004E6F00506C6561736520757067726121
:1019700064652E004E6577206669726D77617265C9
:101980002076657273696F6E20617661696C616241
:101990006C653A004D6F7665205A004D6F76652074
:1019A00059004D6F766520580045787472756465EE
:1019B00072004D6F76652061786973004D657368BC
:1019C00020426564204C6576656C696E67004361F2
:1019D0006C6962726174696F6E00206F66203900F5
:1019E0004D6561737572696E6720726566657265B3
:1019F0006E636520686569676874206F662063613F
:101A00006C6962726174696F6E20706F696E7400C8
:101A10004D61696E004D32323120496E76616C69DC
:101A20006420657874727564657220004D323138B7
:101A300020496E76616C696420657874727564659E
:101A40007220004D32303020496E76616C6964201E
:101A5000657874727564657220005265706F727477
:101A6000696E6720656E6473746F7020737461743F
:101A70007573004649524D574152455F4E414D45A1
:101A80003A4D61726C696E2056312E302E323B20F9
:101A9000537072696E7465722F6772626C206D612B
:101AA0007368757020666F722067656E36204649D0
:101AB000524D574152455F55524C3A687474707399
:101AC0003A2F2F6769746875622E636F6D2F70727D
:101AD00075736133642F50727573612D69332D50A6
:101AE0006C75732F2050524F544F434F4C5F5645E7
:101AF0005253494F4E3A312E30204D414348494EC2
:101B0000455F545950453A507275736120693320CE
:101B10004D4B332045585452554445525F434F5521
:101B20004E543A3120555549443A303030303030F7
:101B300030302D303030302D303030302D303030AE
:101B4000302D3030303030303030303030300A00EE
:101B50004D31303920496E76616C69642065787446
:101B6000727564657220004D31303520496E7661A2
:101B70006C696420657874727564657220004D31FB
:101B8000303420496E76616C6964206578747275B2
:101B900064657220004C6F6F73652070756C6C65A6
:101BA00079004C6F61642066696C616D656E7400CC
:101BB0004C6F6164696E672066696C616D656E74F7
:101BC000004C6F6164696E6720636F6C6F720053C5
:101BD000656C656374206C616E6775616765004B49
:101BE000494C4C45442E2000496E76616C69642056
:101BF000657874727564657200496E7365727420DD
:101C000066696C616D656E74005072696E74204611
:101C1000414E3A20004E6F7A7A6C652046414E3A2A
:101C200000457874727564657220696E666F002075
:101C30006F66203900496D70726F76696E67206239
:101C400065642063616C6962726174696F6E207093
:101C50006F696E740043616C6962726174696E676A
:101C6000205A0043616C6962726174696F6E20640E
:101C70006F6E650043616C696272617465205A0021
:101C800048656174696E6720646F6E652E004865F3
:101C90006174696E670046696C2E2073656E736FA0
:101CA0007220205B6F6E5D0046696C2E2073656E3E
:101CB000736F72205B6F66665D00204672656520FB
:101CC0004D656D6F72793A2000466C6F77004669FA
:101CD0006E697368696E67206D6F76656D656E7489
:101CE0007300206F66203400536561726368696E0B
:101CF00067206265642063616C6962726174696FF8
:101D00006E20706F696E7400497465726174696FDA
:101D10006E2000446F6E6520736176696E67206681
:101D2000696C652E00446F6E65207072696E74690F
:101D30006E672066696C6500497320636F6C6F7213
:101D400020636C6561723F004368616E6765206661
:101D5000696C616D656E740046616E2073706565B7
:101D60006400656E717565696E6720220045787440
:101D70007275646572002045787465726E616C20BE
:101D80005265736574005072696E74657220737465
:101D90006F707065642064756520746F2065727261
:101DA0006F72732E204669782074686520657272A0
:101DB0006F7220616E6420757365204D393939204A
:101DC000746F20726573746172742E202854656D6F
:101DD00070657261747572652069732072657365D0
:101DE000742E2053657420697420616674657220B6
:101DF00072657374617274696E6729004E6F204C4E
:101E0000696E65204E756D62657220776974682011
:101E1000636865636B73756D2C204C617374204C23
:101E2000696E653A20004E6F20436865636B737579
:101E30006D2077697468206C696E65206E756D62BF
:101E400065722C204C617374204C696E653A2000D9
:101E500020746F6F206C6F6E672065787472757375
:101E6000696F6E2070726576656E746564004C698A
:101E70006E65204E756D626572206973206E6F7499
:101E8000204C617374204C696E65204E756D6265DF
:101E9000722B312C204C617374204C696E653A2092
:101EA000005072696E7465722068616C7465642E8E
:101EB000206B696C6C28292063616C6C656421005F
:101EC00020636F6C6420657874727573696F6E201F
:101ED00070726576656E74656400636865636B73C4
:101EE000756D206D69736D617463682C204C61732E
:101EF00074204C696E653A20004552524F523A00A8
:101F0000456E642066696C65206C697374006F703F
:101F1000656E0054524947474552454400656E641A
:101F200073746F7073206869743A2000536C656530
:101F3000702E2E2E0044697361626C652073746587
:101F400070706572730043757272656E74004372CF
:101F5000617368206465742E2020205B6F6E5D00C5
:101F60004372617368206465742E20205B6F66661F
:101F70005D0020436F756E7420583A2000436861FD
:101F80006E67656420636F72726563746C793F007D
:101F9000436F6F6C646F776E00204C6173742055D3
:101FA0007064617465643A200043686F6F736520E4
:101FB00065787472756465723A004368616E67652E
:101FC000207375636365737321005072696E7420AA
:101FD00066726F6D2053440054656D702E206361EE
:101FE0006C6962726174696F6E0043616C696272E0
:101FF0006174650052657365742058595A20636195
:102000006C6962722E0043616C6962726174652052
:1020100058595A002042726F776E206F75742052A3
:102020006573657400426567696E2066696C65203A
:102030006C6973740058595A2063616C69627261EB
:1020400074696F6E20636F6D70726F6D6973656414
:102050002E204C6566742066726F6E742063616C0E
:102060006962726174696F6E20706F696E74206E40
:102070006F7420726561636861626C652E005859E7
:102080005A2063616C6962726174696F6E20636F5C
:102090006D70726F6D697365642E2046726F6E7419
:1020A0002063616C6962726174696F6E20706F6920
:1020B0006E7473206E6F7420726561636861626C08
:1020C000652E0058595A2063616C696272617469A7
:1020D0006F6E20616C6C2072696768742E20582FB7
:1020E0005920617865732061726520736C69676837
:1020F000746C7920736B657765642E20476F6F640D
:10210000206A6F62210058595A2063616C696272BB
:102110006174696F6E20616C6C2072696768742EDF
:1021200020536B65772077696C6C20626520636F44
:1021300072726563746564206175746F6D61746932
:1021400063616C6C792E0058595A2063616C696226
:10215000726174696F6E206661696C65642E2042DD
:1021600065642063616C6962726174696F6E20706E
:102170006F696E7420776173206E6F7420666F755F
:102180006E642E0058595A2063616C6962726174E2
:10219000696F6E206F6B2E20582F59206178657300
:1021A000206172652070657270656E646963756C1C
:1021B00061722E20436F6E67726174756C61746911
:1021C0006F6E73210058595A2063616C69627261A5
:1021D00074696F6E206661696C65642E20506C6551
:1021E00061736520636F6E73756C7420746865200D
:1021F0006D616E75616C2E0058595A2063616C696F
:1022000062726174696F6E206661696C65642E200C
:102210004C6566742066726F6E742063616C6962CF
:10222000726174696F6E20706F696E74206E6F7466
:1022300020726561636861626C652E0058595A208E
:1022400063616C6962726174696F6E206661696C4A
:1022500065642E2046726F6E742063616C696272D1
:102260006174696F6E20706F696E7473206E6F7425
:1022700020726561636861626C652E00426564204E
:102280006C6576656C696E67206661696C65642E45
:102290002053656E736F7220646973636F6E6E6531
:1022A00063746564206F72206361626C6520627282
:1022B0006F6B656E2E2057616974696E6720666F5B
:1022C000722072657365742E00426564206C6576B9
:1022D000656C696E67206661696C65642E20536564
:1022E0006E736F72206469646E74207472696767BC
:1022F00065722E20446562726973206F6E206E6F66
:102300007A7A6C653F2057616974696E6720666FE1
:10231000722072657365742E00426564206C657668
:10232000656C696E67206661696C65642E20536513
:102330006E736F722074726967676572656420746A
:102340006F6F20686967682E2057616974696E67CE
:1023500020666F722072657365742E00426564207A
:1023600048656174696E670042656420646F6E65DC
:1023700000526967687420736964655B756D5D0000
:1023800052657365740052656172207369646520DB
:102390005B756D5D00426564206C6576656C2063DD
:1023A0006F7272656374004C65667420736964654E
:1023B000205B756D5D0046726F6E74207369646595
:1023C0005B756D5D004265640044697374616E63A2
:1023D00065206265747765656E20746970206F662C
:1023E00020746865206E6F7A7A6C6520616E642057
:1023F0007468652062656420737572666163652028
:10240000686173206E6F74206265656E20736574F9
:10241000207965742E20506C6561736520666F6C41
:102420006C6F7720746865206D616E75616C2C200F
:102430006368617074657220466972737420737486
:102440006570732C2073656374696F6E20466972C2
:102450007374206C617965722063616C696272616A
:1024600074696F6E2E004C6976652061646A7573BD
:1024700074205A0041646A757374696E67205A004B
:102480004175746F20686F6D6500207C2041757404
:10249000686F723A2000416C6C0041637469766524
:1024A0002045787472756465723A20001A122E12F3
:1024B00036123E1247124F1257125B1263126B1202
:1024C0007B128712AA12BB12CD12DD12F012031377
:1024D00008131A132B133B134C1384139913A513CE
:1024E000AD13B813C213D613E913FA130814191451
:1024F000261451145714671479148B149A14AB14BE
:10250000B414C114D314E214EF14FD1403151515FB
:102510001E1530154115521562156B15731584156E
:102520009615A815BA15CC15DE15F01502160F165E
:102530001B1620163216441657165F166C167E169A
:102540009216A216B016BD16CB16D916EF16FA16AD
:1025500010171F172E173B17441766177B178D1779
:102560009F17AB17B817C617DB17EE1702180A1814
:1025700012181E1835184318571869187918851835
:102580001B191E1922192B1936193D1951196119D8
:102590006419741994199B19A219A919B219BC19B3
:1025A000CE19DA19E019101A151A2C1A431A5A1AE8
:1025B000731A501B671B7E1B951BA21BB01BC11BF4
:1025C000CF1BDF1BE81BF91B091C151C211C2F1C32
:1025D000351C551C631C741C801C8E1C961CA81C6E
:1025E000BA1CC91CCE1CE21CE81C081D131D251DAD
:1025F000381D481D581D621D6D1D761D861DFC1D54
:10260000261E501E6E1EA11EC01EDA1EF91E001FC1
:102610000E1F131F1D1F2C1F351F461F4E1F601F2F
:10262000721F7D1F901F991FA91FBA1FCA1FD81F95
:10263000EA1FF41F06201420252035207E20C32009
:10264000062147218421C521F8213C227C22C92270
:1026500019235C2368237123802386239523A723D2
:10266000B623C523C9236624742480248A2496248F
:102670009A24457872656D65207370616E206F666F
:1026800020746865205A2076616C7565732100435B
:10269000616C63756C6174696F6E206F662074681D
:1026A00065206D616368696E6520736B6577206175
:1026B0006E64206F6666736574206661696C65641C
:1026C0002E00203C20005741524E494E473A2046AA
:1026D000726F6E7420706F696E74206E6F742072EA
:1026E0006561636861626C652E205920636F6F724B
:1026F00064696E6174653A00004974657261746959
:102700006F6E3A2000496E76616C69642062656480
:1027100020636F7272656374696F6E206D6174728D
:1027200069782E20526573657474696E6720746FC2
:10273000206964656E746974792E00496E76616CE7
:1027400069642062656420636F7272656374696F87
:102750006E206D61747269782E20582F592061782F
:10276000657320617265206661722066726F6D20EC
:102770006265696E672070657270656E6469637505
:102780006C61722E00496E76616C696420626564CA
:1027900020636F7272656374696F6E206D6174720D
:1027A00069782E205368696674206F7574206F668F
:1027B0002072616E67652E005A65726F20706F69B6
:1027C0006E7420636F7272656374696F6E3A00494C
:1027D0006E76616C69642062656420636F727265F5
:1027E0006374696F6E206D61747269782E204C6518
:1027F0006E677468206F662074686520592076655E
:1028000063746F72206F7574206F662072616E67DB
:10281000652E005920766563746F72206C656E6753
:1028200074683A00496E76616C6964206265642060
:10283000636F7272656374696F6E206D6174726923
:10284000782E204C656E677468206F66207468650A
:10285000205820766563746F72206F7574206F66E0
:102860002072616E67652E005820766563746F7202
:10287000206C656E6774683A00556E646566696EB3
:1028800065642062656420636F7272656374696F4A
:102890006E206D61747269782E0000004041000066
:1028A000000000005C430000000000005C430000EA
:1028B0004043000040410000404300004041000010
:1028C00000000000E4420000000000005743000048
:1028D0000000000057430000C0420000E442000036
:1028E000C042000040410000C042000040410000E2
:1028F00040430000E4420000404300005743000012
:1029000040435A00205A3A00590020593A005800D2
:1029100020583A0024F4D43050C38E20C2A240176D
:10292000828B7011127A910D816CD90AA861E1082D
:10293000C7586607615143061E4B5D05C145A70494
:102940001A411104093D9803713931034036DB0205
:1029500065339102D4305402802E1D02632CEE01A7
:10296000752AC501B028A001102781018F256401B7
:102970002B244B01E0223401AC211F018D200D01DD
:10298000801FFC00841EED00971DDF00B81CD200E4
:10299000E61BC600201BBC00641AB200B219A800D6
:1029A0000A19A0006A189900D117910040178B00EE
:1029B000B516840031167E00B31579003A15730000
:1029C000C7146F0058146A00EE1366008813630082
:1029D00025135E00C7125B006C12570015125400DD
:1029E000C111510070114F0021114B00D610490048
:1029F0008D1047004610440002104200C00F4000F6
:102A0000800F3E00420F3C00060F3B00CB0E38000B
:102A1000930E37005C0E3500270E3400F30D3200A4
:102A2000C10D3100900D3000600D2E00320D2D00D3
:102A3000050D2C00D90C2B00AE0C2900850C2900AB
:102A40005C0C2700350C27000E0C2600E80B240038
:102A5000C40B2400A00B23007D0B23005A0B210084
:102A6000390B2100180B2000F80A1F00D90A1E009C
:102A7000BB0A1E009D0A1D00800A1D00630A1C007F
:102A8000470A1B002C0A1B00110A1A00F7091A003A
:102A9000DD091900C4091900AB09190092091700D2
:102AA0007B091800630917004C0916003609160047
:102AB000200916000A091500F5081500E0081400A1
:102AC000CC081400B8081400A408140090081300DF
:102AD0007D0812006B081300580812004608120007
:102AE0003408110023081100120811000108110018
:102AF000F0071000E0071000D0071000C00710001A
:102B0000B0070F00A107100091070E0083070F0008
:102B100074070F0065070E0057070E0049070E00E7
:102B20003B070D002E070E0020070D0013070D00B8
:102B300006070D00F9060C00ED060D00E0060C007E
:102B4000D4060C00C8060C00BC060C00B0060C0035
:102B5000A4060B0099060C008D060B0082060B00E4
:102B600077060B006C060B0061060A0057060B0087
:102B70004C060A0042060A0038060A002E060A0021
:102B800024060A001A060A001006090007060A00B1
:102B9000FD050900F4050900EB050900E20509003F
:102BA000D9050900D0050900C7050900BE050900BF
:102BB000B5050800AD050800A50509009C0508003D
:102BC000940508008C050800840508007C050800B1
:102BD000740508006C050700650508005D05070021
:102BE000560508004E050700470507004005080088
:102BF00038050700310507002A05070023050700EF
:102C00001C050600160507000F050700080506004D
:102C100002050700FB040600F5040700EE040600A9
:102C2000E8040600E2040700DB040600D504060001
:102C3000CF040600C9040600C3040600BD04060054
:102C4000B7040600B1040500AC040600A6040600A3
:102C5000A00405009B0406009504050090040600EE
:102C60008A04050085040500800406007A04050036
:102C700075040500700405006B040500660405007A
:102C8000610405005C0405005704050052040500BA
:102C90004D04050048040500430405003E040400FB
:102CA0003A04050035040500300404002C04050036
:102CB00027040400230405001E0404001A04040071
:102CC00016040500110404000D04040009040500A5
:102CD0000404040000040400FC030400F8030400DE
:102CE000F4030400F0030400EC030400E803040010
:102CF000E4030400E0030400DC030400D803040040
:102D0000D4030400D0030400CC030400C803030070
:102D1000C503030024F404D9201BC40C5C0E9804E2
:102D2000C4095F0265077101F405F900FB04B300F3
:102D300048048700C1036900580355000303450098
:102D4000BE023A008402310053022A002902250003
:102D500004022000E4011C00C8011900AF011700A3
:102D6000980114008401130071011000610110002A
:102D700051010E0043010D0036010B002B010B0029
:102D800020010B00150109000C01090003010800D6
:102D9000FB000800F3000800EB000700E400060059
:102DA000DE000600D8000600D2000600CC000500B8
:102DB000C7000500C2000500BD000400B900040002
:102DC000B5000400B1000400AD000400A900040037
:102DD000A5000300A20003009F0004009B00030065
:102DE0009800030095000200930003009000030088
:102DF0008D0002008B0003008800020086000200A4
:102E000084000300810002007F0002007D000200B8
:102E10007B000200790002007700010076000200CA
:102E20007400020072000100710002006F000200D5
:102E30006D0001006C0002006A00010069000200E0
:102E400067000100660001006500010064000200E7
:102E50006200010061000100600001005F000200EB
:102E60005D0001005C0001005B0001005A000100F0
:102E700059000100580001005700010056000100F0
:102E800055000100540001005300000053000100F0
:102E90005200010051000100500001004F000100EC
:102EA0004E0000004E0001004D0001004C000100EA
:102EB0004B0000004B0001004A00010049000100E6
:102EC00048000000480001004700010046000000E3
:102ED00046000100450000004500010044000100DB
:102EE00043000000430001004200000042000100D6
:102EF0004100000041000100400001003F000000CF
:102F00003F0001003E0000003E0001003D000000C7
:102F10003D0001003C0000003C0000003C000100BE
:102F20003B0000003B0001003A0000003A000100B5
:102F300039000000390001003800000038000000AE
:102F400038000100370000003700010036000000A3
:102F5000360000003600010035000000350000009A
:102F6000350001003400000034000000340001008E
:102F70003300000033000000330001003200000085
:102F8000320000003200010031000000310000007A
:102F9000310001003000000030000000300001006E
:102FA0002F0000002F0000002F0000002F00010064
:102FB0002E0000002E0000002E0001002D00000059
:102FC0002D0000002D0000002D0001002C0000004D
:102FD0002C0000002C0000002C0001002B00000041
:102FE0002B0000002B0000002B0001002A00000035
:102FF0002A0000002A0000002A0001002900000029
:10300000290000002900000029000000290001001B
:103010002800000028000000280000002800000010
:103020002800010027000000270000002700000002
:1030300027000000270001002600000026000000F5
:1030400026000000260000002600010025000000E8
:1030500025000000250000002500000025000000DC
:1030600025000100240000002400000024000000CE
:1030700024000000240001002300000023000000C1
:1030800023000000230000002300000023000000B4
:1030900023000100220000002200000022000000A6
:1030A0002200000022000000220001002100000098
:1030B000210000002100000021000000210000008C
:1030C000210000002100010020000000200000007D
:1030D0002000000020000000200000002000000070
:1030E00020000000200001001F0000001F00000061
:1030F0001F0000001F0000001F0000001F00000054
:103100001F0001001E0000001E0000001E00000045
:103110001E0000004572723A204D494E54454D50F4
:10312000204245440054656D706572617475726526
:1031300020686561746564206265642073776974D2
:1031400063686564206F66662E204D494E54454D78
:10315000502074726967676572656420210045724A
:10316000723A204D415854454D5020424544005438
:10317000656D7065726174757265206865617465EE
:103180006420626564207377697463686564206F86
:1031900066662E204D415854454D50207472696723
:1031A00067657265642021004572723A204D494E70
:1031B00054454D50003A204578747275646572200C
:1031C0007377697463686564206F66662E204D4965
:1031D0004E54454D5020747269676765726564206E
:1031E00021004572723A204D415854454D50003AE5
:1031F00020457874727564657220737769746368AA
:103200006564206F66662E204D415854454D502010
:1032100074726967676572656420210020484F54A5
:10322000454E4420544845524D414C2052554E4144
:10323000574159002048454154424544205448458F
:10324000524D414C2052554E41574159005448452A
:10325000524D414C2052554E415741590042454430
:1032600020544845524D414C2052554E41574159EA
:103270000020544845524D414C2052554E41574133
:10328000592028205052454845415420484F544524
:103290004E44290020544845524D414C2052554E31
:1032A0004157415920282050524548454154204813
:1032B0004541544245442900505245484541542017
:1032C0004552524F520042454420505245484541D4
:1032D00054204552524F52004572723A2050524982
:1032E0004E542046414E204552524F5200455252B4
:1032F0004F523A205072696E742066616E2073706E
:10330000656564206973206C6F77657220746865E9
:103310006E206578706563746564004572723A204A
:10332000455854522E2046414E204552524F52008D
:103330004552524F523A2045787472756465722036
:1033400066616E207370656564206973206C6F77A9
:103350006572207468656E20657870656374656455
:1033600000202D20496E76616C6964206578747246
:1033700075646572206E756D62657220210050491A
:1033800044204175746F74756E652066696E69734B
:10339000686564212050757420746865206C6173C1
:1033A00074204B702C204B6920616E64204B64208C
:1033B000636F6E7374616E74732066726F6D2061DB
:1033C000626F766520696E746F20436F6E66696701
:1033D00075726174696F6E2E6800504944204175A2
:1033E000746F74756E65206661696C656421207404
:1033F000696D656F75740020403A006F6B20543A18
:10340000006F6B20423A00504944204175746F743C
:10341000756E65206661696C6564212054656D7008
:103420006572617475726520746F6F206869676872
:1034300000204B643A2000204B693A2000204B705A
:103440003A200020436C6173736963205049442023
:10345000002054753A2000204B753A2000206D6101
:10346000783A2000206D696E3A200020643A2000EE
:1034700020626961733A200010137D0020157800E6
:1034800060177300C0196E00401C6900E01E6400E4
:1034900080215F0040245A00F026550090295000FA
:1034A000202C4B00802E4600C0304100D0323C0022
:1034B000B034370050363200C0372D0000392800B4
:1034C000103A2300F03A1E00B03B1900503C1400A3
:1034D000D03C0F00303D0A00803D0500C03D00009B
:1034E000F03DFBFF103EF6FF303EF1FF403EECFFAB
:1034F000503EE7FF603EE2FF703EDDFF703ED8FFCA
:103500001000C90210012C014001220170011801B4
:10351000B0010E01F00104015002FA00B002F00007
:103520003003E600D003DC009004D2007005C80030
:10353000A006BE000008B400B009AA00D00BA0008D
:10354000600E960060118C00001582002019780032
:10355000C01D6E00A0226400B0275A00902C5000BD
:1035600000314600E0343C0010383200903A280028
:10357000603C1E00A03D1400803E0A00203F000079
:1035800070012C0190012701B0012201C0011D0131
:10359000F00118011002130130020E01600209014E
:1035A00090020401C002FF000003FA004003F5008E
:1035B0008003F000D003EB002004E6007004E1007B
:1035C000E004DC004005D700C005D2004006CD0075
:1035D000D006C8008007C3003008BE00F008B9005C
:1035E000C009B400B00AAF00B00BAA00D00CA5000F
:1035F000000EA000500F9B00C010960050129100CA
:1036000000148C00C0158700B0178200B0197D002F
:10361000D01B7800001E730040206E0090226900CD
:10362000F024640040275F0090295A00E02B5500E9
:10363000102E500020304B0010324600E033410085
:1036400090353C001037370070383200A0392D001B
:10365000B03A2800A03B2300603C1E00103D19003A
:10366000903D1400103E0F00703E0A00C03E050061
:10367000003F0000544D4320445249564552204FCC
:1036800056455254454D502000436F6E74696E7517
:1036900065207769746820616E6F74686572206256
:1036A0006F7764656E3F00473736004D3435205ADA
:1036B000004D3435004738300020003E003E0020E9
:1036C000003E003E000053657665726520736B65B1
:1036D000773A0000536C6967687420736B65773ABA
:1036E000002D2D2D2D2D2D2D2D2D2D2D2D2D2D2D37
:1036F0002D2D2D2D2D004E2F41004D6561737572BE
:10370000656420736B65773A20004E2F41006D6D24
:10371000000052696768743A004C6566743A005953
:103720002064697374616E63652066726F6D206DCD
:10373000696E3A004D373031004D373032004D352B
:103740003030004731205A31352046313530300095
:103750004739310047312058353020593139302030
:10376000453020463730303000473930004D373053
:1037700032004D3730322043004D37303220550073
:103780004D373032004731205A31352046313530FF
:103790003000473931004731205835302059313910
:1037A00030204530204637303030004D3833004728
:1037B0003930004D3834004D31303420533000471B
:1037C0003930004731204531004D3832004D383313
:1037D000004D31303620532564004D3232302053B5
:1037E0002564003A200020202020202020202020B6
:1037F00020202020202020202000203A20002020EF
:1038000020202020202020202020202020202020B8
:1038100020200020202020202020202020202020C8
:10382000002573002020002D2D3A2D2D0020002092
:103830000020004C002020002046002D2D2D003EB1
:10384000555342005344002D2D00252020202020D8
:10385000002020002020000120002020202D2D2DE0
:10386000200020205A002020000120004D3630305A
:1038700000464C4558202D20203233302F35300063
:1038800050502020202D20203235342F3130300070
:1038900048495053202D20203232302F3130300013
:1038A00050455420202D20203234302F3930005004
:1038B0004C4120202D20203231352F35350041421A
:1038C0005320202D20203235352F313030006661D5
:1038D000726D20202D20203235302F3430004D32B3
:1038E00034004D323320257300052E2E0058005928
:1038F000005A004578747275646572004739390062
:1039000044697361626C65206661726D206D6F64DD
:10391000653F0044697361626C65206661726D2069
:103920006D6F6465004661726D206E756D626572C3
:10393000004D3834005072696E742066616E3A0032
:1039400045787472756465722066616E3A004178DC
:103950006973206C656E6774682064696666657259
:10396000656E63653A004D656173757265642061CB
:10397000786973206C656E6774683A004D3834005E
:103980004732382057005A30005A31005930005918
:103990003100583000583100456E642073746F70E8
:1039A000732064696167004D343400473238205712
:1039B000004175746F207265636F76657220637263
:1039C00061736800436865636B2066616E73205B9A
:1039D0004449535D00436865636B2066616E7320E4
:1039E0005B454E5D0054656D7065726174757265FE
:1039F000730058595A2063616C2E206465746169A4
:103A00006C73002D2D2D2D2D2D2D2D2D2D2D2D00BB
:103A1000466C617368416972204950204164647248
:103A20003A002D2D2D2D2D2D2D2D2D2D2D2D004EF2
:103A30006F76202037203230313700446174653A88
:103A400020002D2D2D2D2D2D2D2D2D2D2D2D0045F5
:103A50003344763666756C6C0045494E595F303498
:103A60006100315F37356D6D5F4D4B33002D2D2D6E
:103A70002D2D2D2D2D2D2D2D2D0020332E302E31A1
:103A8000322D5243322062313037004669726D77F1
:103A90006172653A0025642E25642E25642E256406
:103AA000004661696C207374617473004661726DC5
:103AB000206E756D626572000072630062657461EC
:103AC00000616C7068610064657600505255534126
:103AD0003344465700332E302E31322D52433200BC
:103AE00000000A0B02090C0D0E0807030401000078
:103AF00000000000000000000000000000000000C6
:103B00000000000000000000000000001211100082
:103B100000000000000000000000000000000000A5
:103B20000000000000000000000000000000000095
:103B300000000000000001021020200808102040B2
:103B40001020408002010201080402010102040861
:103B500010204080804020100804020180040201EF
:103B60008040201008040201080402010102040838
:103B70001020408001020408102040801008040832
:103B80008010204004408010204004800505050579
:103B9000070508080808020202020A0A08080404C5
:103BA00004040101010101010101030303030303F3
:103BB0000303040707070C0C0C0C0C0C0C0C020282
:103BC000020206060606060606060B0B0B0B0B0B7F
:103BD0000B0B07070A0A0A0A0A0A0505050404046A
:103BE0000808000020002300260029002C002F00D8
:103BF000320000010000030106010901000022005B
:103C0000250028002B002E003100340002010000A6
:103C1000050108010B0100002100240027002A00F3
:103C20002D003000330001010000040107010A01EA
:103C3000024E414E494E495459494E46CDCCCC3D99
:103C40000AD7233C17B7D13877CC2B329595E62489
:103C50001FB14F0A000020410000C84200401C462E
:103C600020BCBE4CCA1B0E5AAEC59D7400407A10D3
:103C7000F35A00A0724E18090010A5D4E80000E81D
:103C80007648170000E40B54020000CA9A3B00007B
:103C900000E1F505000080969800000040420F000A
:103CA0000000A08601000000102700000000E803CB
:103CB000000000006400000000000A000000000096
:103CC0000100000000002C76D888DC674F0823DF55
:103CD000C1DFAE59E1B1B796E5E3E453C63AE65128
:103CE000997696E8E6C28426EB898C9B62ED407C4F
:103CF0006FFCEFBC9C9F40F2BAA56FA5F490055AEB
:103D00002AF75C936B6CF9676DC11BFCE0E40D470F
:103D1000FEF520E6B500D0ED902E03009435770532
:103D20000080841E080000204E0A000000C80C33EA
:103D30003333330F986E12831141EF8D2114893B79
:103D4000E65516CFFEE6DB18D1844B381BF77C1DF9
:103D5000901DA4BBE424203284725E228100C9F14C
:103D600024ECA1E53D27218EAFB45BE6770151013C
:103D7000528E11241FBECFEFD1E2DEBFCDBF00E0D7
:103D80000CBF19E0A0E0B2E0ECE7F2E403E00BBF07
:103D900002C007900D92AA3DB107D9F72CE1AAED18
:103DA000B9E001C01D92A631B207E1F71DE3C0E7FB
:103DB000DDE300E006C022970109FE010BBF0F946E
:103DC000AE97C636D10780E00807A9F70F94959102
:103DD0000D942CA10C940000CF92DF92EF92FF92F1
:103DE0000F931F93CF93DF938C01D42EC62FD72F21
:103DF000D60EDC1671F1F801E080F180C990C701A0
:103E00000F94F09DC816F1F06C2DC7010F94209E01
:103E1000C7010F94F09D8C15A9F0EEE1F7E08491B5
:103E2000882341F09091C00095FFFCCF8093C6009D
:103E30003196F5CF8091C00085FFFCCF8AE080935A
:103E4000C60007C0F801808191810196918380832B
:103E5000D0CFDF91CF911F910F91FF90EF90DF9026
:103E6000CF900895EF92FF920F931F93CF93DF931C
:103E70001F92CDB7DEB78C017B01460FF801808120
:103E8000918149830F94F09DF70181937F01F8019F
:103E90008081918101969183808349814E11EECF7B
:103EA0000F90DF91CF911F910F91FF90EF900895A8
:103EB000FF920F931F93CF93DF93CDB7DEB72C976D
:103EC0000FB6F894DEBF0FBECDBF8C01F62E80E397
:103ED00090E3A0E3B0E08D839E83AF83B8871C8717
:103EE0000B8744E0BE016B5F7F4FCE010B9674DF02
:103EF00040E160E779E1CE010B966EDF40E160E8DA
:103F000079E1CE010B9668DF40E160E679E1CE0110
:103F10000B9662DF44E068E579E1CE010B965CDF49
:103F200044E064E579E1CE010B9656DF44E06CE5B0
:103F300079E1CE010B9650DF44E060E479E1CE01F7
:103F40000B964ADF44E060E979E1CE010B9644DF4D
:103F500044E064E479E1CE010B963EDF44E068E49E
:103F600079E1CE010B9638DF44E06CE479E1CE01D3
:103F70000B9632DF44E060E579E1CE010B962CDF51
:103F80004CE064E17BE0CE010B9626DF44E06DE07F
:103F90007BE0CE010B9620DF44E06EE972E0CE01BB
:103FA0000B961ADF44E06AE972E0CE010B9614DF4B
:103FB00044E066E972E0CE010B960EDF44E06EE865
:103FC00072E0CE010B9608DF44E06AE872E0CE01B1
:103FD0000B9602DF44E066E872E0CE010B96FCDE51
:103FE00080E290E09A87898742E0BE01675F7F4F59
:103FF000CE010B96F1DE41E069E07BE0CE010B964D
:10400000EBDE44E06DE172E0CE010B96E5DE44E0CC
:1040100065E172E0CE010B96DFDE44E064E07BE018
:10402000CE010B96D9DE44E060E07BE0CE010B963A
:10403000D3DE44E061E172E0CE010B96CDDE41E0DB
:1040400060E37BE0CE010B96C7DE44E06DE372E0F7
:10405000CE010B96C1DE89E08F1560F444E06FE875
:1040600073E1CE010B96B8DE44E06BE873E1CE015C
:104070000B96B2DE46E551E360E070E049835A8377
:104080006B837C831C870B8744E0BE016F5F7F4F8F
:10409000CE010B96A1DEEEE7FEE08491882341F08D
:1040A0009091C00095FFFCCF8093C6003196F5CF6C
:1040B000EEE0F7E08491882341F09091C00095FFF5
:1040C000FCCF8093C6003196F5CF8091C00085FF6C
:1040D000FCCF8AE08093C6002C960FB6F894DEBF22
:1040E0000FBECDBFDF91CF911F910F91FF9008952B
:1040F0001F93CF93DF93182FCEE7DEE0FE0184916C
:10410000882341F09091C00095FFFCCF8093C600BA
:104110003196F5CFEEEFF6E08491882341F090914F
:10412000C00095FFFCCF8093C6003196F5CF8091FB
:10413000C00085FFFCCF8AE08093C600FE01849119
:10414000EEE7FEE0882349F09091C00095FFFCCF98
:104150008093C60031968491F5CF409170195091AB
:104160007119609172197091731986EF96E00E942F
:10417000A03640917419509175196091761970911B
:10418000771983EF96E00E94A036409178195091FC
:10419000791960917A1970917B1980EF96E00E94ED
:1041A000A03640917C1950917D1960917E197091D3
:1041B0007F198DEE96E00E94A0368091C00085FFA9
:1041C000FCCF8AE08093C600FE018491EEE7FEE01A
:1041D000882349F09091C00095FFFCCF8093C600E2
:1041E00031968491F5CFE3EDF6E08491882341F098
:1041F0009091C00095FFFCCF8093C6003196F5CF1B
:104200008091C00085FFFCCF8AE08093C600FE014C
:104210008491EEE7FEE0882349F09091C00095FF7D
:10422000FCCF8093C60031968491F5CF40918019E0
:104230005091811960918219709183198AEC96E0EE
:104240000E94A03640918419509185196091861979
:104250007091871987EC96E00E94A03640918819EA
:104260005091891960918A1970918B1984EC96E0AC
:104270000E94A03640918C1950918D1960918E1931
:1042800070918F1981EC96E00E94A0368091C00059
:1042900085FFFCCF8AE08093C600FE018491EEE7A3
:1042A000FEE0882349F09091C00095FFFCCF8093F9
:1042B000C60031968491F5CFE3EAF6E08491882335
:1042C00041F09091C00095FFFCCF8093C6003196DD
:1042D000F5CF8091C00085FFFCCF8AE08093C600B7
:1042E000FE018491EEE7FEE0882349F09091C00042
:1042F00095FFFCCF8093C60031968491F5CF409115
:1043000060195091611960916219709163198AE97D
:1043100096E00E94B1364091641950916519609100
:1043200066197091671987E996E00E94B13640914D
:1043300068195091691960916A1970916B1984E933
:1043400096E00E94B13640916C1950916D196091C0
:104350006E1970916F1981E996E00E94B1368091D3
:10436000C00085FFFCCF8AE08093C600FE018491E7
:10437000EEE7FEE0882349F09091C00095FFFCCF66
:104380008093C60031968491F5CFECE5F6E08491F8
:10439000882341F09091C00095FFFCCF8093C60028
:1043A0003196F5CF8091C00085FFFCCF8AE08093E5
:1043B000C600FE018491EEE7FEE0882349F090916B
:1043C000C00095FFFCCF8093C60031968491F5CF55
:1043D000409158195091591960915A1970915B196F
:1043E00083E596E00E94A0364091541950915519EA
:1043F000609156197091571980E596E00E94A03699
:104400008091C00085FFFCCF8AE08093C600FE014A
:104410008491EEE7FEE0882349F09091C00095FF7B
:10442000FCCF8093C60031968491F5CFEDE9F5E09D
:104430008491882341F09091C00095FFFCCF809338
:10444000C6003196F5CF8091C00085FFFCCF8AE091
:104450008093C600FE018491EEE7FEE0882349F0D8
:104460009091C00095FFFCCF8093C6003196849157
:10447000F5CF40915C1950915D1960915E19709172
:104480005F1984E995E00E94A0364091401950914F
:104490004119609142197091431981E995E00E9498
:1044A000A036409190195091911960919219709194
:1044B00093198EE895E00E94B136409144195091CD
:1044C000451960914619709147198BE895E00E9453
:1044D000A036409148195091491960914A1970913C
:1044E0004B1988E895E00E94A03640914C195091F4
:1044F0004D1960914E1970914F1985E895E00E9411
:10450000A0364091501950915119609152197091F3
:10451000531982E895E00E94A0368091C00085FF83
:10452000FCCF8AE08093C600FE018491EEE7FEE0B6
:10453000882349F09091C00095FFFCCF8093C6007E
:1045400031968491F5CFE0E7F5E08491882341F03E
:104550009091C00095FFFCCF8093C6003196F5CFB7
:104560008091C00085FFFCCF8AE08093C600FE01E9
:104570008491EEE7FEE0882349F09091C00095FF1A
:10458000FCCF8093C60031968491F5CF4091140BF7
:104590005091150B6091160B7091170B87E695E003
:1045A0000E94A0364091180B5091190B60911A0B84
:1045B00070911B0B84E695E00E94A03640911C0B85
:1045C00050911D0B60911E0B70911F0B81E695E0C1
:1045D0000E94A0368091C00085FFFCCF8AE08093C6
:1045E000C600FE018491EEE7FEE0882349F0909139
:1045F000C00095FFFCCF8093C60031968491F5CF23
:10460000E3E5F5E08491882341F09091C00095FFA7
:10461000FCCF8093C6003196F5CF8091C00085FF16
:10462000FCCF8AE08093C600FE018491EEE7FEE0B5
:10463000882349F09091C00095FFFCCF8093C6007D
:1046400031968491F5CF40919E0250919F026091E6
:10465000A0027091A10289E495E00E94A0366091C9
:104660009A0270919B0280919C0290919D020F94FE
:10467000B021AB01BC0186E495E00E94A0366091B8
:1046800096027091970280919802909199020F94EE
:10469000BC21AB01BC0183E495E00E94A03680916F
:1046A000C00085FFFCCF8AE08093C600FE018491A4
:1046B000EEE7FEE0882349F09091C00095FFFCCF23
:1046C0008093C60031968491F5CFEDE2F5E08491B8
:1046D000882341F09091C00095FFFCCF8093C600E5
:1046E0003196F5CF8091C00085FFFCCF8AE08093A2
:1046F000C600FE018491EEE7FEE0882349F0909128
:10470000C00095FFFCCF8093C60031968491F5CF11
:1047100040918E0250918F026091900270919102AF
:1047200083E295E00E94A03660918A0270918B022C
:1047300080918C0290918D020F94B021AB01BC014D
:1047400080E295E00E94A036609186027091870217
:1047500080918802909189020F94BC21AB01BC0129
:104760008DE195E00E94A0368091C00085FFFCCFCE
:104770008AE08093C600FE018491EEE7FEE0882384
:1047800049F09091C00095FFFCCF8093C600319610
:104790008491F5CFE9EEF4E08491882341F0909183
:1047A000C00095FFFCCF8093C6003196F5CF809175
:1047B000C00085FFFCCF8AE08093C600FE01849193
:1047C000EEE7FEE0882349F09091C00095FFFCCF12
:1047D0008093C60031968491F5CF40911D0250918F
:1047E0001E0260911F02709120028FED94E00E94E2
:1047F000A03620E030E040E752E46091150270916D
:10480000160280911702909118020F945295AB01F5
:10481000BC018CED94E00E94A0364091040B5091B5
:10482000050B6091060B7091070B89ED94E00E94D7
:10483000A0368091C00085FFFCCF8AE08093C6003F
:10484000FE018491EEE7FEE0882349F09091C000DC
:1048500095FFFCCF8093C60031968491F5CFEDEAA9
:10486000F4E08491882341F09091C00095FFFCCF43
:104870008093C6003196F5CF8091C00085FFFCCFB4
:104880008AE08093C600FE018491EEE7FEE0882373
:1048900049F09091C00095FFFCCF8093C6003196FF
:1048A0008491F5CF4091000B5091010B6091020B68
:1048B0007091030B83EA94E00E94A03620E030E080
:1048C00040E752E46091110270911202809113024C
:1048D000909114020F945295AB01BC0180EA94E0D0
:1048E0000E94A0368091C00085FFFCCF8AE08093B3
:1048F000C600FE018491EEE7FEE0882349F0909126
:10490000C00095FFFCCF8093C60031968491F5CF0F
:10491000E6E4F4E08491882341F09091C00095FF93
:10492000FCCF8093C6003196F5CF8091C00085FF03
:10493000FCCF8AE08093C600FE018491EEE7FEE0A2
:10494000882349F09091C00095FFFCCF8093C6006A
:1049500031968491F5CF4091090B50E060E070E012
:104960008CE394E00E94B1368091C00085FFFCCFBB
:104970008AE08093C600FE018491EEE7FEE0882382
:1049800049F09091C00095FFFCCF8093C60031960E
:104990008491F5CF8091300B8823A1F1E9E2F4E016
:1049A0008491882341F09091C00095FFFCCF8093C3
:1049B000C6003196F5CF8091C00085FFFCCF8AE01C
:1049C0008093C600FE018491EEE7FEE0882349F063
:1049D0009091C00095FFFCCF8093C60031968491E2
:1049E000F5CF40913D0250913E0260913F0270919F
:1049F00040028FE194E00E94A0368091C00085FFC4
:104A0000FCCF11C0E3E0F4E08491882341F0909161
:104A1000C00095FFFCCF8093C6003196F5CF809102
:104A2000C00085FFFCCF8AE08093C6001A3008F4EE
:104A30003EC0FE01C491EEE7FEE0CC2349F0809138
:104A4000C00085FFFCCFC093C6003196C491F5CF5E
:104A5000EAEEF3E08491882341F09091C00095FF45
:104A6000FCCF8093C6003196F5CF8091C00085FFC2
:104A7000FCCF8AE08093C60040918F135091901331
:104A8000609191137091921380EE93E00E94A03692
:104A900040918B1350918C1360918D1370918E13F4
:104AA00086ED93E0DF91CF911F910C94A036DF91BA
:104AB000CF911F910895AF92BF92CF92DF92EF9264
:104AC000FF920F931F93CF93DF93CDB7DEB7E0979D
:104AD0000FB6F894DEBF0FBECDBF80E1E3EDF2E08C
:104AE000DE01919601900D928A95E1F780E1E3EE67
:104AF000F2E0DE01519601900D928A95E1F780E196
:104B0000E3EFF2E0DE01119601900D928A95E1F754
:104B10006E0181E2C80ED11C80E7E82E89E1F82EF3
:104B20008E010F5E1F4F60E879E1AE014F5F5F4F6E
:104B300090E6A92E99E1B92E20E030E0F6018191AE
:104B40009191A191B1916F01F70181939193A193FB
:104B5000B1937F01F80181919191A191B1918F0160
:104B6000FB0181939193A193B193BF01FA018191CC
:104B70009191A191B191AF01F50181939193A1938D
:104B8000B1935F012F5F3F4F24303105B9F60E948A
:104B900051FE80E090E4ACE9B4E48093581990931E
:104BA0005919A0935A19B0935B1980935419909393
:104BB0005519A0935619B093571910925C19109279
:104BC0005D1910925E1910925F1980E29EE4A0E0D8
:104BD000B0E08093901990939119A0939219B0939B
:104BE0009319109240191092411910924219109283
:104BF000431980E090E0A0E7B1E4809344199093DA
:104C00004519A0934619B09347198093481990937A
:104C10004919A0934A19B0934B198DEC9CECACEC5C
:104C2000BEE380934C1990934D19A0934E19B09305
:104C30004F1980E090E0A0E2B0E480935019909387
:104C40005119A0935219B093531910921C0B109242
:104C50001D0B10921E0B10921F0B1092180B10922E
:104C6000190B10921A0B10921B0B1092140B10922E
:104C7000150B1092160B1092170B8DE39AE0A1E81A
:104C8000B1E480939E0290939F02A093A002B09300
:104C9000A1026DEC7CEC84E99FE30F94AA21609360
:104CA0009A0270939B0280939C0290939D0265E808
:104CB0007BEE80E692E40F94B621609396027093A7
:104CC000970280939802909399020F94F01080E0DD
:104CD00090E0A0E8BFE38093920290939302A093A8
:104CE0009402B09395021092090B80E090E0A0E44A
:104CF000B0E480931D0290931E02A0931F02B09314
:104D0000200240E050E064E372E4409315025093C7
:104D1000160260931702709318021092040B1092FF
:104D2000050B1092060B1092070B1092000B1092BD
:104D3000010B1092020B1092030B40E050E060E078
:104D400071E4409311025093120260931302709326
:104D500014021092300B80933D0290933E02A09378
:104D60003F02B09340020E940049EEE7FEE08491CA
:104D7000882341F09091C00095FFFCCF8093C6003E
:104D80003196F5CFEAE9F3E08491882341F09091E0
:104D9000C00095FFFCCF8093C6003196F5CF80917F
:104DA000C00085FFFCCF8AE08093C600E0960FB676
:104DB000F894DEBF0FBECDBFDF91CF911F910F9151
:104DC000FF90EF90DF90CF90BF90AF9008951F932A
:104DD000CF93DF93CDB7DEB72C970FB6F894DEBF35
:104DE0000FBECDBF162F9C878B8786E591E3A0E091
:104DF000B0E089839A83AB83BC8344E0BE016B5FE0
:104E00007F4FCE010B962ED843E050E0BE016B5F82
:104E10007F4FCE0101960F945F9B892B09F0FFC055
:104E200040E160E779E1CE010B961CD840E160E8F3
:104E300079E1CE010B9616D840E160E679E1CE012A
:104E40000B9610D80E9451FE44E068E579E1CE014E
:104E50000B9608D844E064E579E1CE010B9602D8C0
:104E600044E06CE579E1CE010B960E94321F44E0EC
:104E700060E479E1CE010B960E94321F44E060E9C4
:104E800079E1CE010B960E94321F44E064E479E19F
:104E9000CE010B960E94321F44E068E479E1CE0116
:104EA0000B960E94321F44E06CE479E1CE010B9630
:104EB0000E94321F44E060E579E1CE010B960E942A
:104EC000321F4CE064E17BE0CE010B960E94321F62
:104ED00044E06DE07BE0CE010B960E94321F44E07F
:104EE0006EE972E0CE010B960E94321F44E06AE93F
:104EF00072E0CE010B960E94321F44E066E972E038
:104F0000CE010B960E94321F44E06EE872E0CE01A3
:104F10000B960E94321F44E06AE872E0CE010B96C5
:104F20000E94321F44E066E872E0CE010B960E94B8
:104F3000321F42E0BE01675F7F4FCE010B960E9499
:104F4000321F41E069E07BE0CE010B960E94321FE8
:104F500044E06DE172E0CE010B960E94321F44E006
:104F600065E172E0CE010B960E94321F44E064E0DE
:104F70007BE0CE010B960E94321F44E060E07BE0B4
:104F8000CE010B960E94321F44E061E172E0CE0137
:104F90000B960E94321F41E060E37BE0CE010B964E
:104FA0000E94321F44E06DE372E0CE010B960E9436
:104FB000321F1A3070F044E06FE873E1CE010B96B7
:104FC0000E94321F44E06BE873E1CE010B960E9411
:104FD000321F0E9400490F94F010EEE7FEE084912A
:104FE000882341F09091C00095FFFCCF8093C600CC
:104FF0003196F5CFECEBF3E08491882341F090916A
:10500000C00095FFFCCF8093C6003196F5CF80910C
:10501000C00085FFFCCF8AE08093C60001C04BDD55
:105020002C960FB6F894DEBF0FBECDBFDF91CF91A7
:105030001F910895682F772767FD709580917410F0
:105040009091751087589F4E0F94449B90936B10CE
:1050500080936A1021E0892B09F420E0822F0895C3
:1050600080916A1090916B1060E070E001960D9451
:10507000ED978A3010F0895A01C0805D9091C00090
:1050800095FFFCCF8093C6000895CF93C82F8295DB
:105090008F70EFDF8C2F8F70CF91EBCFCF93C82F16
:1050A000892FF3DF8C2FCF91F0CFCF93DF93FB01CC
:1050B00020E030E0DC01ED018D918823A1F1411564
:1050C000510519F02417350774F58032A1F38A30A1
:1050D00051F190ED980F9A3020F4682F6295607F1F
:1050E00008C09FE9980F9630A8F4682F6295607FFA
:1050F0006057CE0102967981A0EDA70FAA3018F46F
:10510000762F7A2B0CC0AFE9A70FA63018F477558D
:10511000762B05C088279927821B930B05C07193B6
:105120002F5F3F4FC7CFC901DF91CF910895E09125
:105130006A10F0916B1081818823C1F06BE573E0F8
:105140008AED99E0F6D782E475DF882369F0F89458
:1051500028E088E190E00FB6F894A895809360006D
:105160000FBE20936000FFCF0C9400000895CF93F2
:10517000DF9366E673E08AED99E0DBD7F894C0E050
:10518000D0E060E0CE010F94209E2196C11580E111
:10519000D807B9F77894DF91CF910895AF92BF9275
:1051A000CF92DF92EF92FF920F931F93CF93DF93F3
:1051B000CDB7DEB760970FB6F894DEBF0FBECDBF98
:1051C00068E773E08AED99E0B4D781E433DF8823A0
:1051D000A9F080916A1090916B10FC012181283711
:1051E00041F440E150E060E070E002960F94559980
:1051F00003C036DF0F94EC927B0102C0E12CF12C4E
:1052000083E418DF882331F02BDF0F94EC92262FF4
:10521000872F02C020E080E2FFE1FF22022F182F3B
:10522000013020E2120710F000E010E2C8018E0DFC
:105230009F1D8130904220F000E010E20E191F09FE
:1052400088E5F8DE882371F180916A1090916B10E7
:1052500040E150E0BE016F5F7F4F019626DF8C0179
:10526000009701F1FE013196CF01800F911FD70108
:10527000E817F90719F021912D93FACF4AE050E091
:10528000B8018AED99E0BAD76CE873E08AED99E04D
:1052900050D7C70103DF8091C00085FFFCCF8AE0B3
:1052A0008093C60080E2B82E9AE0A92E0115110560
:1052B00029F1C701F3DE8091C00085FFFCCFB092D9
:1052C000C6006701F0E1CF0ED11CF7012FEFE21A03
:1052D000F20A80819091C00095FFFCCFB092C60089
:1052E000D4DE0150110919F0EC14FD0471F780911E
:1052F000C00085FFFCCFA092C600D8CF60960FB645
:10530000F894DEBF0FBECDBFDF91CF911F910F91FB
:10531000FF90EF90DF90CF90BF90AF900895AF9245
:10532000BF92CF92DF92EF92FF920F931F93CF9392
:10533000DF93CDB7DEB760970FB6F894DEBF0FBE30
:10534000CDBF6DEA73E08AED99E0F3D681E472DEB9
:105350008823A9F080916A1090916B10FC01218143
:10536000283741F440E150E060E070E002960F948D
:10537000559903C075DE0F94EC927B0102C0E12CBD
:10538000F12C83E457DE882331F06ADE0F94EC922F
:10539000262F872F02C020E080E2FFE1FF22022FAC
:1053A000182F013020E2120710F000E010E2C801CF
:1053B0008E0D9F1D8130904220F000E010E20E190A
:1053C0001F0988E537DE8823B1F180916A1090913A
:1053D0006B1040E150E0BE016F5F7F4F019665DECC
:1053E0008C01009741F1CE0101965C01C12CD12CBA
:1053F000C016D10661F0F50161915F01C6018E0D05
:105400009F1D0F94209EFFEFCF1ADF0AF1CF4AE0D5
:1054100050E0B8018AED99E0F1D664EC73E08AEDD2
:1054200099E087D6C7013ADE8091C00085FFFCCFA6
:105430008AE08093C60020E2B22E3AE0A32E011546
:10544000110531F1C7012ADE8091C00085FFFCCF34
:10545000B092C600670120E1C20ED11CC701EFEF78
:10546000EE1AFE0A0F94F09D9091C00095FFFCCFBC
:10547000B092C6000ADE0150110919F0EC14FD04C7
:1054800069F78091C00085FFFCCFA092C600D7CFFE
:1054900060960FB6F894DEBF0FBECDBFDF91CF91FF
:1054A0001F910F91FF90EF90DF90CF90BF90AF9042
:1054B0000895CF92DF92EF92FF92CF93DF9368EE41
:1054C00073E08AED99E035D680E5B4DD882309F4F0
:1054D0006BC0C6DD0F94EC926B017C018FEFC81698
:1054E000D10411F008F060C086E4A4DD882379F0CF
:1054F000B7DD0F94EC926115710511F460E004C002
:105500006130710521F461E08C2D0F949B8B86E551
:1055100091DD8823B1F0A4DD0F94EC926115710543
:1055200011F460E005C06130710509F03DC061E033
:105530008C2DDF91CF91FF90EF90DF90CF900D9465
:10554000D48B8C2D0F94098CC1E0D0E0892B11F401
:10555000C0E0D0E0E8EFF3E08191882339F090914A
:10556000C00095FFFCCF8093C600F6CF4AE050E024
:10557000B6018AED99E0EAD5EAE5F4E08191882365
:1055800039F09091C00095FFFCCF8093C600F6CF14
:105590004AE050E0BE018AED99E0DF91CF91FF90A3
:1055A000EF90DF90CF90D9C5DF91CF91FF90EF9032
:1055B000DF90CF9008956CEF73E08AED99E0B9C564
:1055C000CF9362E174E08AED99E0B3D5E0916A107F
:1055D000F0916B1085818F3311F0811170C0E2E280
:1055E000F4E08191882339F09091C00095FFFCCFC1
:1055F0008093C600F6CF4AE050E0609173138AEDC5
:1056000099E0E9D5E9E2F4E08191882339F09091BD
:10561000C00095FFFCCF8093C600F6CF4AE050E073
:10562000609172138AED99E0D6D5E1E3F4E08191BF
:10563000882339F09091C00095FFFCCF8093C6007D
:10564000F6CF60917013709171134AE050E08AEDCB
:1056500099E07CD5E5E3F4E08191882339F09091DD
:10566000C00095FFFCCF8093C600F6CF60916E130B
:1056700070916F134AE050E08AED99E067D5E9E355
:10568000F4E08191882339F09091C00095FFFCCF20
:105690008093C600F6CF4AE050E060916D138AED2A
:1056A00099E099D5EDE3F4E08191882309F455C0A0
:1056B0009091C00095FFFCCF8093C600F5CF81325A
:1056C00009F053C00E94F1E9E2E3F4E081918823FC
:1056D00039F09091C00095FFFCCF8093C600F6CFC3
:1056E00060917013709171134AE050E08AED99E077
:1056F0002DD5E5E3F4E08191882339F09091C00045
:1057000095FFFCCF8093C600F6CF60916E13709129
:105710006F134AE050E08AED99E018D5E9E3F4E030
:105720008191882339F09091C00095FFFCCF809340
:10573000C600F6CF4AE050E060916D138AED99E023
:105740004AD5EDE3F4E08191882339F09091C000CF
:1057500095FFFCCF8093C600F6CF4AE050E0609101
:105760006C138AED99E0CF913CC582E563DC882318
:1057700061F176DC0F94EC92C62FE1E4F4E08191C4
:10578000882339F09091C00095FFFCCF8093C6002C
:10579000F6CF4AE050E06C2F8AED99E01CD5E9E5A0
:1057A000F4E08191882339F09091C00095FFFCCFFF
:1057B0008093C600F6CF6C2F8C2F0E947DEA4AE0C2
:1057C00050E0BC018AED99E0C8D488E533DC882339
:1057D000E1F046DC0F94EC927093711360937013B8
:1057E000ECE5F4E08191882339F09091C00095FFB9
:1057F000FCCF8093C600F6CF609170137091711347
:105800004AE050E08AED99E0A1D489E513DC8823D1
:10581000E9F026DC0F94EC9270936F1360936E1393
:10582000E7E6F4E08191882339F09091C00095FF7C
:10583000FCCF8093C600F6CF60916E1370916F130A
:105840004AE050E08AED99E0CF9180C4CF9108956D
:10585000CF93DF93EC0160E08E810F94D48B81E0D5
:1058600090E00F94168A61E08E810F94D48B81E0D2
:1058700090E00F94168A60E08E810F94D48B84E6BA
:1058800090E0DF91CF910D94168ACF92DF92EF9244
:10589000FF920F931F93CF93DF937C01C0E0D0E082
:1058A000C62ED12C87010C0F1D1F61E0F8018781E6
:1058B0000F949B8BB6010C2E02C0759567950A94C8
:1058C000E2F76170F80187810F94D48B2196C43080
:1058D000D10541F7C701DF91CF911F910F91FF9043
:1058E000EF90DF90CF90B4CFCF92DF92EF92FF9204
:1058F0000F931F93CF93DF937C01C0E0D0E0C62EBF
:10590000D12C87010C0F1D1F61E0F80187810F94D6
:105910009B8BB6010C2E02C0759567950A94E2F731
:105920006170F80187810F94D48B2196C830D1051E
:1059300041F7C701DF91CF911F910F91FF90EF9039
:10594000DF90CF9085CF1F93CF93DF93EC01162F7D
:10595000642F8C810F94D48B8D818F3F19F060E080
:105960000F94D48B8F85612F84FF05C0CE01DF910A
:10597000CF911F91B9CF70E084E0759567958A95B6
:10598000E1F7CE0182DF612FCE01DF91CF911F9130
:105990007CCF40E0D8CF61E0FCDF80E496E00D945E
:1059A000168A62E0F6DF80E496E00D94168ACF93C3
:1059B000DF93CDB7DEB728970FB6F894DEBF0FBEE2
:1059C000CDBF28E0E3E0F3E0DE01119601900D92F7
:1059D0002A95E1F7FC012389421710F04FEF420F9F
:1059E000FE013196E40FF11DE40FF11D2081260F19
:1059F0002068622F28960FB6F894DEBF0FBECDBF89
:105A0000DF91CF91C6CFFC016089262F2460208BC7
:105A10006C60BFCFCF93DF93EC01423018F08F85DD
:105A200088608F874B8B1C8A222329F0413019F420
:105A30008F8584608F8780E593EC0F94168A60E0F1
:105A40008C810F94D48B60E08E810F94D48B8D81E8
:105A50008F3F19F060E00F94D48B6F8564FD19C0FF
:105A600063E0CE0112DF84E991E10F94168A63E0CE
:105A7000CE010BDF84E991E10F94168A63E0CE0139
:105A800004DF86E990E00F94168A62E0CE01FDDE25
:105A900013C06062CE017DDF84E991E10F94168A24
:105AA0006F856062CE0175DF86E990E00F94168AFB
:105AB0006F856062CE016DDF6F856062CE0169DF48
:105AC0008CE390E00F94168A84E0888BCE019BDFF4
:105AD0008CE390E00F94168ACE015DDF88EB9BE0AB
:105AE0000F94168A82E0898B66E0CE0152DF8CE348
:105AF00090E0DF91CF910D94168A6F927F928F92F2
:105B0000AF92CF92EF920F931F93CF93DF93CDB7C6
:105B1000DEB73C01162F842F5E854F853889998921
:105B2000F301848325830683E782C086A18682866B
:105B3000538744873587968761E00F949B8BF301E9
:105B400085818F3F19F061E00F949B8B61E0F30139
:105B500086810F949B8B112319F0F301178603C0E4
:105B600080E1F301878720E041E060E1C301DF913C
:105B7000CF911F910F91EF90CF90AF908F907F902A
:105B80006F9048CF8F92AF92CF92EF920F93DC013C
:105B900013961C921E921297E6E7F4E0ED93FC93A5
:105BA0001F921F921F921F928C2CAE2CC02EE22EA1
:105BB000042F2FEF462F61E0A0DF0F900F900F9082
:105BC0000F900F91EF90CF90AF908F900895CF935B
:105BD000DF93EC01423018F08F8588608F874B8B04
:105BE0001C8A222329F0413019F48F8584608F8725
:105BF00080E593EC0F94168A60E08C810F94D48B2F
:105C000060E08E810F94D48B8D818F3F19F060E01E
:105C10000F94D48B6F8564FD19C063E0CE0135DE2F
:105C200084E991E10F94168A63E0CE012EDE84E9C7
:105C300091E10F94168A63E0CE0127DE86E990E0B9
:105C40000F94168A62E0CE0120DE13C06062CE019E
:105C5000A0DE84E991E10F94168A6F856062CE011F
:105C600098DE86E990E00F94168A6F856062CE0117
:105C700090DE6F856062CE018CDE8CE390E00F9445
:105C8000168A84E0888BCE01BEDE8CE390E00F9410
:105C9000168ACE0186DE80E496E00F94168A82E0B2
:105CA000898B66E0CE0175DE8CE390E00F94168A56
:105CB00040E068E0CE017BDE62E579E0CE010F9442
:105CC0006F8C41E068E0CE0172DE62E579E0CE01E2
:105CD0000F946F8C42E066E0CE0169DE60E579E00A
:105CE000CE01DF91CF910D946F8CCF92DF92EF9226
:105CF000FF920F931F93CF93DF931F921F92CDB705
:105D0000DEB78C01677088E0689FB0011124606481
:105D1000C80149835A833DDE4981C42E5A81D52E5C
:105D2000E12CF12CD6016D916D01D801ED91FC9122
:105D30000190F081E02DC8011995BFEFEB1AFB0A25
:105D4000E8E0EE16F10471F70F900F90DF91CF911C
:105D50001F910F91FF90EF90DF90CF90089541E059
:105D6000F2DD81E090E008951F920F920FB60F923E
:105D700011240BB60F922F933F934F935F936F9322
:105D80008F939F93EF93FF938091C00084FF03C094
:105D90008091C60019C06091C60020915B0A3091C5
:105DA0005C0AC90101968F77992740915D0A50914D
:105DB0005E0A8417950741F0F901E552F64F6083BA
:105DC00090935C0A80935B0AFF91EF919F918F9172
:105DD0006F915F914F913F912F910F900BBE0F905C
:105DE0000FBE0F901F9018951F920F920FB60F9233
:105DF00011240BB60F922F933F934F935F936F93A2
:105E00008F939F93EF93FF9380915F0A813001F509
:105E10008091D00084FF03C08091D60019C06091AA
:105E2000D60020915B0A30915C0AC90101968F77F8
:105E3000992740915D0A50915E0A8417950741F0B9
:105E4000F901E552F64F608390935C0A80935B0AF8
:105E5000FF91EF919F918F916F915F914F913F9142
:105E60002F910F900BBE0F900FBE0F901F901895A3
:105E7000CF92DF92EF92FF926A017B01411581EE92
:105E800058076105710509F463C082E08093C00082
:105E900060E079E08DE390E0A70196010F9476979A
:105EA0002150310941095109CA01B90122E030E00C
:105EB00040E050E00F94769791E03093C500209336
:105EC000C4008091C10080618093C1008091C100B5
:105ED00088608093C1008091C10080688093C10078
:105EE00080915F0A8130D1F5992341F082E080935F
:105EF000D00060E079E08DE390E006C01092D00021
:105F000060E874E88EE190E0A70196010F9476971F
:105F10002150310941095109CA01B90122E030E09B
:105F200040E050E00F9476973093D5002093D40052
:105F30008091D10080618093D1008091D1008860F0
:105F40008093D1008091D10080688093D10006C0F9
:105F50001092C00090E020E130E0AFCFFF90EF90D2
:105F6000DF90CF90089520915D0A30915E0A809174
:105F70005B0A90915C0A8217930771F0F901E55270
:105F8000F64F80812F5F3F4F2F77332730935E0A84
:105F900020935D0A90E008958FEF9FEF0895809120
:105FA0005D0A90915E0A90935C0A80935B0A089563
:105FB0004F925F926F927F928F929F92AF92BF9219
:105FC000CF92DF92EF92FF920F931F93CF93DF93C5
:105FD000CDB7DEB7A0970FB6F894DEBF0FBECDBF2A
:105FE0005C014115510561057105E9F420E030E0DF
:105FF00040E350E060E070E0A0960FB6F894DEBF9A
:106000000FBECDBFDF91CF911F910F91FF90EF9009
:10601000DF90CF90BF90AF909F908F907F906F90C8
:106020005F904F905BC08E010F5F1F4FC12CD12C32
:1060300076014801422E512C612C712C8FEFC81A29
:10604000D80AE80AF80ACB01BA01A30192010F9419
:106050005497CA01F80161938F01A901BC01411550
:1060600051056105710551F7F1E0CF1AD108E1083A
:10607000F108F401EC0DFD1D80818A3010F440E33D
:1060800001C047E3480F552747FD5095652F752FF1
:1060900020E030E0C50122D081E0C81AD108E10833
:1060A000F108EFEFCE16DE06EE06FE0611F7A0961B
:1060B0000FB6F894DEBF0FBECDBFDF91CF911F9119
:1060C0000F91FF90EF90DF90CF90BF90AF909F9097
:1060D0008F907F906F905F904F90089521153105BC
:1060E00039F48091C00085FFFCCF4093C60008952D
:1060F0002A30310509F43FC05BCF9A01462F55275E
:1061000047FD5095652F752FE9CFCF93DF93EC01B5
:1061100020E030E04DE050E060E070E0DFDF20E0C4
:1061200030E04AE050E060E070E0CE01DF91CF91D6
:10613000D5CFFB012191BF01222339F03091C0005E
:1061400035FFFCCF2093C600F4CFDFCF9A01AB011F
:10615000662757FD6095762FC1CFCF93DF93EC0173
:106160009A01AB01662757FD6095762FB7DFCE0108
:10617000DF91CF91CACFCF92DF92EF92FF92CF9370
:10618000DF93EC016A017B0177FF0FC020E030E074
:106190004DE250E060E070E0A1DFF094E094D09434
:1061A000C094C11CD11CE11CF11C2AE0B701A6015E
:1061B000CE01DF91CF91FF90EF90DF90CF90F8CE9E
:1061C0002115310539F48091C00085FFFCCF409343
:1061D000C6000895EDCE9A01462F50E060E070E0D1
:1061E000EFCFCF93DF93EC019A01462F50E060E0B0
:1061F00070E0E6DFCE01DF91CF9187CF9A01AB014E
:1062000060E070E0DDCFCF93DF93EC019A01AB014A
:1062100060E070E0D5DFCE01DF91CF9176CFCF93F4
:10622000DF93EC01CDDFCE01DF91CF916ECF8F9266
:106230009F92AF92BF92CF92DF92EF92FF921F9305
:10624000CF93DF93EC016A017B01122F20E030E055
:10625000A901C701B6010F947D9287FF0CC020E011
:1062600030E04DE250E060E070E0CE0137DFF7FA59
:10627000F094F7F8F094B12C60E070E080E09FE3D8
:10628000B11641F020E030E040E251E40F948492F6
:10629000B394F6CF9B01AC01C701B6010F94A49152
:1062A0006B017C010F94F1924B015C010F941D93E3
:1062B0009B01AC01C701B6010F94A3916B017C0156
:1062C0002AE0B501A401CE0173DE112361F0E0EDF7
:1062D000F6E08191882339F09091C00095FFFCCFC2
:1062E0008093C600F6CF112319F120E030E040E2A0
:1062F00051E4C701B6010F9452956B017C010F94D4
:10630000EC924B01AA2497FCA094BA2CB501A401ED
:10631000CE0131DFC501B4010F941F939B01AC0185
:10632000C701B6010F94A3916B017C011150DBCF23
:10633000DF91CF911F91FF90EF90DF90CF90BF90B2
:10634000AF909F908F90089572CFCF93DF93EC0121
:106350006EDFCE01DF91CF91D8CEFC0165917591B2
:10636000859194910895EF92FF920F931F93CF938D
:10637000DF93EC01CC0FDD1FCC0FDD1FCE01865A61
:10638000914FEBDF9E01205E344F79018E010C5E50
:10639000144FF80120813181428153810F94A491DF
:1063A000F7016083718382839383CE018E58914F6E
:1063B000D4DF9E01235D3D4F7901F80120813181B9
:1063C000428153810F94A491F7016083718382838A
:1063D0009383CE018A59914FC0DFCF5DDD4FF80125
:1063E00020813181428153810F94A4916883798304
:1063F0008A839B83DF91CF911F910F91FF90EF9044
:106400000895CF93C82F40910C0250910D026091D6
:106410000E0270910F024093D70A5093D80A6093EE
:10642000D90A7093DA0A20914702309148023093DA
:10643000920B2093910B24E630E030934802209396
:1064400047020F94B0896093D20A7093D30A809365
:10645000D40A9093D50A8C2FCF910C94FAFF80E048
:106460000E94FAFF8091D70A9091D80AA091D90A88
:10647000B091DA0A80930C0290930D02A0930E0261
:10648000B0930F028091910B9091920B90934802E0
:10649000809347020F94B0896093D20A7093D30A15
:1064A0008093D40A9093D50A0895682F772767FDC3
:1064B0007095809174109091751087589F4E0F942D
:1064C000449B90936B1080936A1021E0892B09F410
:1064D00020E0822F08952091741030917510BC0136
:1064E000C90187589F4E0F947C9B90936B108093AB
:1064F0006A1021E0892B09F420E0822F0895809111
:106500006A1090916B104AE050E060E070E00196F4
:106510000D94559980916A1090916B104AE050E06B
:1065200060E070E001960F945599CB0108950F93A8
:106530001F93CF93DF9300916A1010916B1065E465
:1065400070E0C8010F94449BEC01009751F460E0A7
:1065500070E0C8010196DF91CF911F910F910D94CA
:10656000ED97188280916A1090916B1060E070E056
:1065700001960F94ED9725E42883DF91CF911F9129
:106580000F91089580916A1090916B1060E070E017
:1065900001960D94ED972F923F924F925F926F92DA
:1065A0007F928F929F92AF92BF92CF92DF92EF92A3
:1065B000FF920F931F93CF93DF93CDB7DEB7609712
:1065C0000FB6F894DEBF0FBECDBF1C012A013B0100
:1065D0004801590120E030E04CE052E4C301B2012F
:1065E0000F94A39125E535E547E052E40F9484929A
:1065F0006B017C010F945A930F94EC928B0177FFFF
:1066000012C020E030E040E85FE3C701B6010F941C
:10661000809418160CF05DC0C12CD12CE0E8EE2E51
:10662000EFE3FE2E56C066307105DCF02AEA3AE24E
:106630004CE453E4C301B2010F94A39125E535E581
:1066400047E052E40F9484926B017C0120E030E03B
:10665000A9010F947D9287FF3FC0C12CD12C7601F8
:106660003BC0882777FD8095982F0F941F9325E5D1
:1066700035E547E052E40F94529520E030E04CE0DD
:1066800052E40F94A4919B01AC01C301B2010F9499
:10669000A39125E535E547E052E40F9484926B0120
:1066A0007C0120E030E0A9010F947D9287FD17C0A6
:1066B00020E030E040E85FE3C701B6010F9480942A
:1066C000181684F4C12CD12C70E8E72E7FE3F72E46
:1066D00009C000E010E006C005E010E003C0C12CD6
:1066E000D12C760120E030E040EC50E4C501B4014B
:1066F0000F94A3912BEA3AEA42E052E40F94849279
:106700002B013C010F945A930F94EC92788B6F8776
:1067100077FF12C020E030E040E85FE3C301B20140
:106720000F94809418160CF05FC0412C512C60E837
:10673000662E6FE3762E58C0AF85B8891697E4F0C1
:1067400026E535E549E253E4C501B4010F94A39170
:106750002BEA3AEA42E052E40F9484922B013C0186
:1067600020E030E0A9010F947D9287FD40C0E5E074
:10677000F0E0F88BEF8746C0882777FD8095982F4B
:106780000F941F932BEA3AEA42E052E40F94529599
:1067900020E030E040EC50E40F94A4919B01AC0168
:1067A000C501B4010F94A3912BEA3AEA42E052E406
:1067B0000F9484922B013C0120E030E0A9010F945A
:1067C0007D9287FD1CC020E030E040E85FE3C3011C
:1067D000B2010F9480941816ACF4412C512C50E85F
:1067E000652E5FE3752E0EC0188A1F860BC0412CE4
:1067F000512C320125E030E0388B2F8703C0412C2B
:10680000512C3201A701960160E070E080E89FE31F
:106810000F94A39169837A838B839C83C80101962B
:106820009E838D83AF85B8891196BA87A987A30106
:10683000920160E070E080E89FE30F94A3916B8782
:106840007C878D879E8747E02F853889429FF0019E
:10685000439FF00D1124F887EF83E00FF11FEE0F37
:10686000FF1FEE0FFF1FE20DF31D218132814381D7
:10687000548169817A818B819C810F9452954B015F
:106880005C01EF81F8858D819E81E80FF91FEE0F85
:10689000FF1FEE0FFF1FE20DF31D218132814381A7
:1068A0005481C701B6010F9452959B01AC01C501FB
:1068B000B4010F94A4919B01AC016B857C858D85FF
:1068C0009E850F9452954B015C0127E0E985FA857E
:1068D0002E9FD0012F9FB00D1124B887AF83FD01EB
:1068E000E00FF11FEE0FFF1FEE0FFF1FE20DF31D74
:1068F000218132814381548169817A818B819C819C
:106900000F94529569837A838B839C83AF81B8857A
:106910008D819E81A80FB91FAA0FBB1FAA0FBB1F95
:10692000A20DB31D11962D913D914D915C9114973F
:10693000C701B6010F9452959B01AC0169817A8120
:106940008B819C810F94A4919B01AC01C301B20186
:106950000F9452959B01AC01C501B4010F94A49111
:1069600060960FB6F894DEBF0FBECDBFDF91CF911A
:106970001F910F91FF90EF90DF90CF90BF90AF905D
:106980009F908F907F906F905F904F903F902F904F
:1069900008954F925F926F927F929F92AF92BF92B3
:1069A000CF92DF92EF92FF920F931F93CF93DF93DB
:1069B0007C015B018A01E9019090A612911014C03C
:1069C000FC0180819181A281B381FA01808391834E
:1069D000A283B383FB0180819181A281B3818883EB
:1069E0009983AA83BB837FC091FE55C0FC0120819F
:1069F00031814281538160919612709197128091FA
:106A00009812909199120F9452952B013C01F50127
:106A1000208131814281538160919A1270919B1241
:106A200080919C1290919D120F9452959B01AC0104
:106A3000C301B2010F94A491F80160837183828332
:106A40009383F701208131814281538160919E12AD
:106A500070919F128091A0129091A1120F94529563
:106A60006B017C01F501208131814281538160916C
:106A7000A2127091A3128091A4129091A5120F946A
:106A800052959B01AC01C701B6010F94A491688394
:106A900079838A839B8390FE26C020917E12309159
:106AA0007F124091801250918112F80160817181B2
:106AB000828193810F94A491F80160837183828312
:106AC00093832091821230918312409184125091CD
:106AD0008512688179818A819B810F94A491688352
:106AE00079838A839B83DF91CF911F910F91FF90D0
:106AF000EF90DF90CF90BF90AF909F907F906F907E
:106B00005F904F9008952F923F924F925F926F92B5
:106B10007F928F929F92AF92BF92CF92DF92EF922D
:106B2000FF920F931F93CF93DF93CDB7DEB72897D4
:106B30000FB6F894DEBF0FBECDBF8C011B019E01C6
:106B40002F5F3F4FAE014B5F5F4F23DF20E030E010
:106B5000A9016D817E818F8198850F947D9287FF39
:106B600007C01D821E821F821886FF24F39401C075
:106B7000F12C20E030E040E451EC69817A818B8196
:106B80009C810F947D9287FF0AC080E090E0A0E492
:106B9000B1EC89839A83AB83BC83FF24F39420E018
:106BA00030E04FE753E46D817E818F8198850F94AB
:106BB0008094181654F480E090E0AFE7B3E48D833E
:106BC0009E83AF83B887FF24F39420E030E042E552
:106BD00053E469817A818B819C810F94809418168B
:106BE0004CF480E090E0A2E5B3E489839A83AB8320
:106BF000BC8303C0FF2009F483C0C980DA80EB8026
:106C0000FC808D809E80AF80B8847090A612711039
:106C10000BC0F80180829182A282B382F101C0820E
:106C2000D182E282F3826AC070FE1CC020917E1283
:106C300030917F124091801250918112C501B401B0
:106C40000F94A3914B015C01209182123091831229
:106C50004091841250918512C701B6010F94A391FF
:106C60006B017C0171FE4AC020918612309187121F
:106C70004091881250918912C501B4010F94529528
:106C80002B013C0120918A1230918B1240918C1281
:106C900050918D12C701B6010F9452959B01AC0122
:106CA000C301B2010F94A491F801608371838283C0
:106CB000938320918E1230918F12409190125091B7
:106CC0009112C501B4010F9452954B015C012091C2
:106CD0009212309193124091941250919512C701E3
:106CE000B6010F9452959B01AC01C501B4010F94FC
:106CF000A491F1016083718382839383FF24F394D1
:106D00008F2D28960FB6F894DEBF0FBECDBFDF9152
:106D1000CF911F910F91FF90EF90DF90CF90BF9098
:106D2000AF909F908F907F906F905F904F903F902B
:106D30002F900895682F87EF9FE00D94029E08958D
:106D4000FC012491222341F03091C00035FFFCCF9B
:106D50002093C6000196F4CF22E030E08AED99E05E
:106D6000F3CAFC012491222341F03091C00035FF89
:106D7000FCCF2093C6000196F4CF2AE030E08AEDE4
:106D800099E01ECACF936AE774E08AED99E0D1D901
:106D9000C1E0C093A2026FEF89E69FE00F94029ECC
:106DA000C093CF02CF9108956AE874E08AED99E02C
:106DB000C0D91092A20260E089E69FE00F94029E83
:106DC0001092CF020895EF92FF920F931F93CF93EB
:106DD000DF931F92CDB7DEB789830F94263989815F
:106DE000823009F468C0B4F5882309F442C08130C8
:106DF00009F0F4C09FB7F8948091020184608093F9
:106E000002019FBFEFEFF1EE24E0E150F04020409F
:106E1000E1F700C000009FB7F894809102018B7FDA
:106E2000809302019FBF40E050E0BA018DEE9FE0E9
:106E30000F94149E40E050E0BA0181EF9FE00F9460
:106E4000149E0F90DF91CF911F910F91FF90EF90C3
:106E50000D94AF5E833009F45CC0843009F0BEC08D
:106E60000F90DF91CF911F910F91FF90EF900D94B4
:106E7000BD669FB7F89480910201846080930201FF
:106E80009FBF2FEF81EE94E0215080409040E1F7CA
:106E900000C000009FB7F894809102018B7F80931F
:106EA00002019FBF0F90DF91CF911F910F91FF9033
:106EB000EF900D94CE390F94CE3980EF3BDF1092D6
:106EC000B11B1092B01B6091B21B84EC9FE00F9439
:106ED000029E60EB7BE181EC9FE00F9452399FB7FB
:106EE000F894809102018460809302019FBF8FEF2C
:106EF00091EEE4E081509040E040E1F700C00000F6
:106F00009FB7F894809102018B7F809302019FBF0D
:106F100065C081E39EE00F94B84E40E25EE062E01F
:106F200081E00F94B46A9FB7F89480910201846065
:106F3000809302019FBFFFEF21EE84E0F1502040DB
:106F40008040E1F700C000009FB7F89480910201F3
:106F50008B7F809302019FBF1092BE0A1092BD0AE0
:106F600049E15EE063E083E00F94B46A4091BD0ABA
:106F70005091BE0A63E083E00F943139E12CF12C8B
:106F800009E210E06FEFC7010F94209EC701B8011E
:106F90000F944197892BD9F48091BD0A9091BE0A34
:106FA00001969093BE0A8093BD0A42E15EE063E0E1
:106FB00083E00F94B46A4091BD0A5091BE0A63E029
:106FC00083E00F94313980E19EE00F94B84E9FEF3B
:106FD000E91AF90AE114E0E1FE06A1F60F90DF914B
:106FE000CF911F910F91FF90EF90089580E1E0E223
:106FF000FBE0ABEEBAE001900D928A95E1F70895BF
:107000004F925F926F927F928F929F92AF92BF92B8
:10701000CF92DF92EF92FF92CF93DF9300D01F9237
:10702000CDB7DEB70F946D098BE43FDA882391F07A
:107030007EDA6B017C0120E030E0A9010F9480949E
:1070400087FD08C0C0928F13D0929013E0929113E5
:10705000F092921382E529DA882359F068DA6B01FD
:107060007C0120E030E0A9010F947D9287FF83C06E
:1070700006C0C12CD12C60E8E62E6FEBF62E84E41E
:1070800014DA882321F053DA4B015C0106C0812C0D
:10709000912C50E8A52E5FEBB52E87E506DA882304
:1070A00021F045DA2B013C0106C0412C512C40E86F
:1070B000642E4FEB742E88E4F8D9882331F037DA48
:1070C00069837A838B839C8308C080E090E0A0E88A
:1070D000BFEB89839A83AB83BC8320E030E0A901B6
:1070E000C501B4010F94809487FD45C020E030E0D5
:1070F000A901C301B2010F94809487FD3CC020E038
:1071000030E0A90169817A818B819C810F94809400
:1071100087FD31C020E030E0A901C501B4010F9422
:107120007D92882391F120E030E040E05FE3C501EB
:10713000B4010F9452956B017C0129813A814B81F6
:107140005C81C301B2010F9452954B015C01A70110
:107150009601C701B6010F9452952BED3FE049E42B
:1071600050E40F9452959B01AC01C501B4010F94FA
:1071700084926B017C0120E030E0A901C701B601D7
:107180000F94809487FF04C00BC0C12CD12C7601D2
:10719000C0928B13D0928C13E0928D13F0928E13C9
:1071A000EEE7FEE08491882341F09091C00095FFC6
:1071B000FCCF8093C6003196F5CFEEEEF9E08491D6
:1071C000882341F09091C00095FFFCCF8093C600CA
:1071D0003196F5CF40918F13509190136091911398
:1071E0007091921322E030E08AED99E0ADD8809161
:1071F000C00085FFFCCF8AE08093C600E8EEF9E08E
:107200008491882341F09091C00095FFFCCF80933A
:10721000C6003196F5CFC0908B13D0908C13E090C0
:107220008D13F0908E1320E030E0A901C701B60164
:107230000F947D92882361F022E030E0B701A6012F
:107240008AED99E081D88091C00085FFFCCF11C004
:10725000E3EEF9E08491882341F09091C00095FF1E
:10726000FCCF8093C6003196F5CF8091C00085FF9A
:10727000FCCF8AE08093C6000F900F900F900F9084
:10728000DF91CF91FF90EF90DF90CF90BF90AF90C4
:107290009F908F907F906F905F904F9008952F9266
:1072A0003F924F925F926F927F928F929F92AF9296
:1072B000BF92CF92DF92EF92FF920F931F93CF93E3
:1072C000DF931F92CDB7DEB781E00E94FAFF89837A
:1072D000E1E4FEE0E4918E2F992781950CF49095DE
:1072E0001C0184E00F94EA24A8E2BBE01D921D92E9
:1072F0001D921C921397E4E2FBE0208131814281D0
:107300005381A0E2BBE06D917D918D919C91ECE267
:10731000CE2EEBE0DE2EE12CF12C87010E948CFCBE
:1073200065DE86E59EE019D82DEC3CEC4CE85FE389
:107330000F9452954B015C01B101882777FD809530
:10734000982F0F941F939B01AC01C501B4010F94BA
:107350005295E3EFFAE020813181428153810F940D
:10736000A4912B013C01A3EFBAE06D937D938D9323
:107370009C931397E1E5F2E06081718182819381B2
:1073800060930C0270930D0280930E0290930F0293
:1073900020E030E040E752E40F9484924B015C011E
:1073A000AFEEBAE02D913D914D915C91EBEEFAE09C
:1073B0006081718182819381ACE0BBE0BF93AF9328
:1073C000F7EFCF2EFAE0DF2E830172010E94DEEF8D
:1073D00082E00F945F220F946D090F946A2580E07C
:1073E0000E94FAFFA8E2BBE01D921D921D921C9222
:1073F0001397E4E2FBE02081318142815381A0E2D6
:10740000BBE06D917D918D919C91ACE2CA2EABE079
:10741000DA2EE12CF12C87010E948CFCE7DD2AE0BA
:10742000229DC001239D900D1124BC01882777FD6A
:107430008095982F0F941F93E3EFFAE0208131811C
:10744000428153810F94A4912B013C01A3EFBAE038
:107450006D937D938D939C93139720E030E040E0F3
:107460005FE3E1E5F2E060817181828193810F94B5
:10747000529560930C0270930D0280930E029093CC
:107480000F0220E030E040E752E40F9484924B0179
:107490005C01AFEEBAE02D913D914D915C91EBEE28
:1074A000FAE06081718182819381ACE0BBE0BF939F
:1074B000AF93B7EFCB2EBAE0DB2E830172010E94AF
:1074C000DEEF0F946D0989810E94FAFF80E090E061
:1074D000AFE4B3E4E8E2FBE080839183A283B3836B
:1074E000A4E2BBE02D913D914D915C91E0E2FBE087
:1074F00060817181828193811CE2C12E1BE0D12EBB
:10750000E12CF12C0FE413E40E948CFC81E00F903D
:107510000F900F900F900F90DF91CF911F910F91CF
:10752000FF90EF90DF90CF90BF90AF909F908F90A3
:107530007F906F905F904F903F902F9008952F9283
:107540003F924F925F926F927F928F929F92AF92F3
:10755000BF92CF92DF92EF92FF920F931F93CF9340
:10756000DF93CDB7DEB729970FB6F894DEBF0FBE15
:10757000CDBF3C0181E00E94FAFF8F8382E0681654
:10758000710408F081C2F301E15CF14FE491D30191
:10759000AA0FBB1FAA0FBB1FBA83A983A75BBD4F4E
:1075A000BE83AD838D919D910D90BC91A02D809354
:1075B0000C0290930D02A0930E02B0930F0281E093
:1075C000062C01C0880F0A94EAF70F94EA24E98197
:1075D000FA81E05EF44FF987E88710821182128207
:1075E0001382E090280BF090290B00912A0B109148
:1075F0002B0B2091240B3091250B4091260B5091A1
:10760000270B6091200B7091210B8091220B9091A0
:10761000230BECE2CE2EEBE0DE2E0E948CFCE98107
:10762000FA81E551F54F2F0180E090E0A0E4B0E44D
:1076300080839183A283B38320E030E040E752E46B
:1076400060910C0270910D0280910E0290910F02D8
:107650000F9484924B015C01E090F30AF090F40ADD
:107660000091F50A1091F60A2091EF0A3091F00A84
:107670004091F10A5091F20A6091EB0A7091EC0A84
:107680008091ED0A9091EE0AFCE02F2EFBE03F2E58
:107690003F922F92A7EFCA2EAAE0DA2E0E94DEEFC9
:1076A0000F946D090E94E2FF80E00E94FAFFA88516
:1076B000B9851D921D921D921C921397E090280B84
:1076C000F090290B00912A0B10912B0B2091240B89
:1076D0003091250B4091260B5091270B6091200B88
:1076E0007091210B8091220B9091230BBCE2CB2E49
:1076F000BBE0DB2E0E948CFC80E090E0A0E8BFEBBA
:10770000F20180839183A283B38320E030E040E7DD
:1077100052E460910C0270910D0280910E029091E2
:107720000F020F9484924B015C01E090F30AF090F9
:10773000F40A0091F50A1091F60A2091EF0A3091AF
:10774000F00A4091F10A5091F20A6091EB0A7091AF
:10775000EC0A8091ED0A9091EE0A3F922F92E7EFAA
:10776000CE2EEAE0DE2E0E94DEEF0F946D0981E05E
:107770000E94FAFF89819A81825B914F0E94AD310C
:107780002DEC3CEC4CE85FEB0F945295D2016D93DD
:107790007D938D939C93139720E030E040E752E473
:1077A00060910C0270910D0280910E0290910F0277
:1077B0000F9484924B015C01E090F30AF090F40A7C
:1077C0000091F50A1091F60A2091EF0A3091F00A23
:1077D0004091F10A5091F20A6091EB0A7091EC0A23
:1077E0008091ED0A9091EE0A3F922F920E94DEEF77
:1077F0000F946D090E94E2FF80E00E94FAFFE88585
:10780000F9851082118212821382E090280BF09089
:10781000290B00912A0B10912B0B2091240B3091F6
:10782000250B4091260B5091270B6091200B7091F6
:10783000210B8091220B9091230BFCE2CF2EFBE0D9
:10784000DF2E0E948CFC80E090E0A0E2B1E4F20127
:1078500080839183A283B38320E030E040E752E449
:1078600060910C0270910D0280910E0290910F02B6
:107870000F9484924B015C01E090F30AF090F40ABB
:107880000091F50A1091F60A2091EF0A3091F00A62
:107890004091F10A5091F20A6091EB0A7091EC0A62
:1078A0008091ED0A9091EE0A3F922F92A7EFCA2E97
:1078B000AAE0DA2E0E94DEEF0F946D090E94E2FF2B
:1078C00081E00E94FAFF80E090E0A0E7B1ECF201D5
:1078D00080839183A283B38320E030E040E05FE3C4
:1078E000AD81BE816D917D918D919C910F9452954A
:1078F00060930C0270930D0280930E0290930F021E
:1079000020E030E040E752E40F9484924B015C01A8
:10791000E090F30AF090F40A0091F50A1091F60A4B
:107920002091EF0A3091F00A4091F10A5091F20A49
:107930006091EB0A7091EC0A8091ED0A9091EE0A49
:107940003F922F920E94DEEF0F946D09C3010E94B7
:10795000B331F301EF5EF44F81E080830F946A2529
:107960000E94E2FF80E00E94FAFF2AE037ED43E246
:107970005FE3E885F98560817181828193810F944D
:10798000A391A885B9856D937D938D939C9313974F
:10799000E090280BF090290B00912A0B10912B0BF3
:1079A0002091240B3091250B4091260B5091270BF1
:1079B0006091200B7091210B8091220B9091230BF1
:1079C000BCE2CB2EBBE0DB2E0E948CFC2AE037ED24
:1079D00043E25FE3E885F98560817181828193816B
:1079E0000F94A491A885B9856D937D938D939C93F5
:1079F0001397F20160837183828393832AE939E9C3
:107A000049E95EE360910C0270910D0280910E02D3
:107A100090910F020F94529520E030E040E752E43D
:107A20000F9484924B015C01E090F30AF090F40A09
:107A30000091F50A1091F60A2091EF0A3091F00AB0
:107A40004091F10A5091F20A6091EB0A7091EC0AB0
:107A50008091ED0A9091EE0A3F922F92E7EFCE2EA1
:107A6000EAE0DE2E0E94DEEF0F946D0910920C0208
:107A700010920D0210920E0210920F020FB6F8949F
:107A8000DEBF0FBECDBF62C192E06916710409F07E
:107A90005DC1E1E4FEE074901092280B1092290B76
:107AA00010922A0B10922B0B2091240B3091250B56
:107AB0004091260B5091270B6091200B7091210B68
:107AC0008091220B9091230BFCE2CF2EFBE0DF2E66
:107AD000E12CF12C87010E948CFC86E59EE00E943F
:107AE000AD314B015C01672D772767FD7095872FBE
:107AF000972F0F941F932B013C0120E030E040ECC6
:107B00005FE3C501B4010F945295A30192010F9454
:107B1000529569837A838B839C836093F30A709375
:107B2000F40A8093F50A9093F60A609151027091DD
:107B30005202809153029091540260930C02709310
:107B40000D0280930E0290930F0220E030E040E798
:107B500052E40F9484924B015C012091EF0A309122
:107B6000F00A4091F10A5091F20A6091EB0A70918B
:107B7000EC0A8091ED0A9091EE0AACE02A2EABE07F
:107B80003A2E3F922F92B7EFCB2EBAE0DB2EE98050
:107B9000FA800B811C810E94DEEF0F946D09109218
:107BA000280B1092290B10922A0B10922B0B20916C
:107BB000240B3091250B4091260B5091270B60919F
:107BC000200B7091210B8091220B9091230B1CE2D2
:107BD000C12E1BE0D12EE12CF12C87010E948CFCE0
:107BE0008AE49EE00E94AD319058A30192010F9467
:107BF000529569837A838B839C836093F30A709395
:107C0000F40A8093F50A9093F60A20E030E040E70A
:107C100052E460910C0270910D0280910E029091DD
:107C20000F020F9484924B015C012091EF0A309176
:107C3000F00A4091F10A5091F20A6091EB0A7091BA
:107C4000EC0A8091ED0A9091EE0A3F922F9207EF95
:107C5000C02E0AE0D02EE980FA800B811C810E94A0
:107C6000DEEF0F946D098AE49EE00E94AD319B0126
:107C7000AC010F94A491A30192010F9452952B0192
:107C80003C016093F30A7093F40A8093F50A909391
:107C9000F60A20E030E040E05FE36091510270912D
:107CA000520280915302909154020F945295609326
:107CB0000C0270930D0280930E0290930F0220E04D
:107CC00030E040E752E40F9484924B015C01209134
:107CD000EF0A3091F00A4091F10A5091F20A609156
:107CE000EB0A7091EC0A8091ED0A9091EE0A3F92B6
:107CF0002F92830172010E94DEEF0F946D0982E0E2
:107D000090E00E94B3318091280B9091290BA091B3
:107D10002A0BB0912B0B8093F30A9093F40AA09353
:107D2000F50AB093F60A10920C0210920D0210920E
:107D30000E0210920F020E94E2FF81E08093130B6B
:107D40000F900F900F900F900F900F908F812996AA
:107D50000FB6F894DEBF0FBECDBFDF91CF911F915C
:107D60000F91FF90EF90DF90CF90BF90AF909F90DA
:107D70008F907F906F905F904F903F902F900C94DA
:107D8000FAFFCF92DF92EF92FF920F931F932ED9BB
:107D900080E090E0D4DB81E090E0D1DBE090280B44
:107DA000F090290B00912A0B10912B0B2091240BA2
:107DB0003091250B4091260B5091270B6091200BA1
:107DC0007091210B8091220B9091230BFCE2CF2E1E
:107DD000FBE0DF2E0E948CFC1F910F91FF90EF9033
:107DE000DF90CF900C94E2FF0F94B0896093D20A99
:107DF0007093D30A8093D40A9093D50A089520E013
:107E000030E0A90168EB71E084E50F94FE8D69E133
:107E100070E080E090E00F94DF8984E50F94229178
:107E200064E170E080E090E00D94DF897F928F92B2
:107E30009F92AF92BF92CF92DF92EF92FF920F93F9
:107E40001F93CF93DF9300D01F92CDB7DEB7109270
:107E5000A81A1092A71A1092A61A1092A51A0F9497
:107E6000263987E19DE00F94B84E8E010F5F1F4FBA
:107E70007E0125E0E20EF11C8AED99E00E94B32F0D
:107E80008F3FEFEF9E07C1F3F80181938F01EE154D
:107E9000FF0591F789809A80AB80BC808091C000FB
:107EA00085FFFCCF8BE28093C600C12CD12C7601DC
:107EB000ABE27A2E8091540B882309F450C00CE772
:107EC0001AE0C814D904EA04FB04A1F08AED99E091
:107ED0000E94B32F8F3FFFEF9F07C1F32FEFC21A0E
:107EE000D20AE20AF20AF80181938F01FAE00C3B10
:107EF0001F0739F76CE77AE08BE99BE00E94B2A597
:107F00008091C00085FFFCCF7092C6000F94031BC8
:107F1000C814D904EA04FB0469F671DF60E08BE958
:107F20009BE00E94E5A61092540BECEEF5E28591E1
:107F30009491FC012491222341F03091C00035FF3F
:107F4000FCCF2093C6000196F4CF8091C00085FF3E
:107F5000FCCF8AE08093C60080E090E000C00F90E4
:107F60000F900F900F90DF91CF911F910F91FF9085
:107F7000EF90DF90CF90BF90AF909F908F907F90C9
:107F800008950F94B0896093D20A7093D30A8093B6
:107F9000D40A9093D50AE0917410F0917510EA58C4
:107FA000FF4E80818130B9F4E0E8F5E2859194914B
:107FB000FC012491222341F03091C00035FFFCCF19
:107FC0002093C6000196F4CF8091C00085FFFCCFBE
:107FD0008AE08093C60008958AED99E00E94CF2F31
:107FE000E6E5F5E285919491FC012491222341F08C
:107FF0003091C00035FFFCCF2093C6000196F4CF2E
:1080000040915A1050915B1060915C1070915D101E
:108010004F5F5F4F6F4F7F4F2AE030E08AED99E06E
:108020000E946E308091C00085FFFCCF8AE0809373
:10803000C600A7CF8F929F92AF92BF92CF92DF924E
:10804000EF92FF920F931F93CF93DF93BCE7EB2E3A
:10805000B6E0FB2E00E21BE0CBEEDAE083E9C82EAF
:108060008BE0D82EF70181917F010E945532882341
:1080700019F10E94C2324B015C01F601808181112D
:1080800003C06091D60A01C061E070E080E090E03A
:108090000F941F93F80120813181428153810F9405
:1080A00052959B01AC01C501B4010F94A491688362
:1080B00079838A839B8309C0F80180819181A281A1
:1080C000B38188839983AA83BB830C5F1F4F249657
:1080D000FFEFCF1ADF0A80E8E81686E0F80611F60F
:1080E00086E40E9455328823D9F00E94C2326B0187
:1080F0007C016093DB0A7093DC0A8093DD0A909325
:10810000DE0A20E030E0A9010F948094181644F4B0
:10811000C0920C02D0920D02E0920E02F0920F0279
:10812000DF91CF911F910F91FF90EF90DF90CF9053
:10813000BF90AF909F908F9008957CDF89E40E945C
:108140005532882359F00E94C2326093DF0A70933F
:10815000E00A8093E10A9093E20A08C01092DF0AD5
:108160001092E00A1092E10A1092E20A8AE40E9458
:108170005532882359F00E94C2326093E30A70930B
:10818000E40A8093E50A9093E60A08951092E30AC0
:108190001092E40A1092E50A1092E60A0895CF922E
:1081A000DF92EF92FF92CF93DF93EC01BC016C5F03
:1081B0007F4F0E94833520E030E0A90160913502B5
:1081C0007091360280913702909138020F94A491F9
:1081D0006B017C019B01AC01688579858A859B8553
:1081E0000F947D9287FF04C0C886D986EA86FB86F5
:1081F000C0902902D0902A02E0902B02F0902C022D
:10820000A7019601688579858A859B850F9480945E
:10821000181624F4C886D986EA86FB86DF91CF91AA
:10822000FF90EF90DF90CF9008952F923F924F9262
:108230005F926F927F928F929F92AF92BF92CF92F6
:10824000DF92EF92FF920F931F93CF93DF93CDB7FF
:10825000DEB7AB970FB6F894DEBF0FBECDBF9F87DA
:108260008E87798B688B5B8B4A8B3D8B2C8B1F8B1E
:108270000E8BED82DC018D909D90AD90BC90409076
:10828000200B5090210B6090220B7090230BDB0190
:108290008D919D910D90BC91A02D88879987AA877B
:1082A000BB87C090240BD090250BE090260BF0905C
:1082B000270B2091280B3091290B40912A0B5091CC
:1082C0002B0BEA89FB8960817181828193810F94F4
:1082D000A391688F798F8A8F9B8F8091A7128111CC
:1082E00073C0AE89BF898D909D90AD90BC90EA8996
:1082F000FB89E080F18002811381A889B9892D91E1
:108300003D914D915C91EE85FF8560817181828107
:108310009381FE013596FF93EF93CC88DD880E9410
:10832000DEEFEE85FF8580819181A281B38180930C
:10833000200B9093210BA093220BB093230BE88981
:10834000F98980819181A281B3818093240B9093DC
:10835000250BA093260BB093270BEA89FB8980811C
:108360009181A281B3818093280B9093290BA093D4
:108370002A0BB0932B0BEC89FD8980819181A2811E
:10838000B38180932C0B90932D0BA0932E0BB09365
:108390002F0B0F900F90AB960FB6F894DEBF0FBE69
:1083A000CDBFDF91CF911F910F91FF90EF90DF90A4
:1083B000CF90BF90AF909F908F907F906F905F9085
:1083C0004F903F902F900895A3019201C501B401F1
:1083D0000F94A3912B013C0120E030E0A9010F9400
:1083E000809453014201181624F0B7FAB094B7F8FC
:1083F000B094A7019601688579858A859B850F943D
:10840000A391688779878A879B8720E030E0A9015C
:108410000F948094288539854A855B8518160CF061
:108420005058C501B4010F94A4916B017C0120E068
:1084300030E0A9010F94809418160CF052CF20E080
:1084400030E040EF51E4C701B6010F9484920F94DD
:108450006A920F94EC927D876C87623071050CF400
:1084600040CF20912C0B30912D0B40912E0B509131
:108470002F0BAC89BD896D917D918D919C910F944D
:10848000A3916C8F7D8F8E8F9F8F22242394312C0C
:108490008C859D85AA2797FDA095BA2F88A799A7B7
:1084A000AAA7BBA7DE011596BF83AE83B1018827BB
:1084B00077FD8095982F0F941F936B017C0168A521
:1084C00079A58AA59BA50F941F939B01AC01C701B9
:1084D000B6010F9484926B017C01EE89FF89808044
:1084E0009180A280B3802C8D3D8D4E8D5F8D0F9439
:1084F00052959B01AC0160912C0B70912D0B8091DA
:108500002E0B90912F0B0F94A49169837A838B8308
:108510009C83288D398D4A8D5B8DC701B6010F94E0
:1085200052952091280B3091290B40912A0B5091A4
:108530002B0B0F94A49168A379A38AA39BA32885EE
:1085400039854A855B85C701B6010F945295209104
:10855000240B3091250B4091260B5091270B0F9443
:10856000A4916CA37DA38EA39FA3A3019201C70135
:10857000B6010F9452952091200B3091210B409120
:10858000220B5091230B0F94A491FF81FF932E8116
:108590002F93DE0111966D01E8A0F9A00AA11BA19D
:1085A0002CA13DA14EA15FA10E94DEEFBFEF2B1ACF
:1085B0003B0A0F900F90EC85FD852E163F0609F0C3
:1085C00075CF8FCE4F925F926F927F928F929F92D4
:1085D000AF92BF92CF92DF92EF92FF920F931F93D1
:1085E000CF93DF93CDB7DEB728970FB6F894DEBFF1
:1085F0000FBECDBF8BEE9AE0D2DD0F94B0896093B1
:10860000D20A7093D30A8093D40A9093D50A8091AA
:10861000EB0A9091EC0AA091ED0AB091EE0A8D83DD
:108620009E83AF83B8879C01AD016091200B709150
:10863000210B8091220B9091230B0F947D9281113D
:1086400097C04090EF0A5090F00A6090F10A709045
:10865000F20AA30192016091240B7091250B809185
:10866000260B9091270B0F947D92811181C020E001
:1086700030E040E752E460910C0270910D0280916D
:108680000E0290910F020F9484924B015C01E090D6
:10869000F30AF090F40A0091F50A1091F60A8CE0C2
:1086A0009BE09F938F9327EFC22E2AE0D22EA30147
:1086B00092016D817E818F8198850E94DEEF0F90FF
:1086C0000F908091EB0A9091EC0AA091ED0AB09185
:1086D000EE0A8093200B9093210BA093220BB09372
:1086E000230B8091EF0A9091F00AA091F10AB091CA
:1086F000F20A8093240B9093250BA093260BB09342
:10870000270B8091F30A9091F40AA091F50AB09199
:10871000F60A8093280B9093290BA0932A0BB09311
:108720002B0B8091F70A9091F80AA091F90AB09169
:10873000FA0A80932C0B90932D0BA0932E0BB093E1
:108740002F0B28960FB6F894DEBF0FBECDBFDF917A
:10875000CF911F910F91FF90EF90DF90CF90BF903E
:10876000AF909F908F907F906F905F904F90089503
:10877000E0900C0B6091470270914802882777FDCA
:108780008095982F0F941F9320910C0230910D0229
:1087900040910E0250910F020F9452952EE333EC4C
:1087A0004EE259E30F94529569837A838B839C83BD
:1087B0008E010F5F1F4F27EF3AE043EF5AE06FEE55
:1087C0007AE08BEE9AE031DD7CCF4F925F926F9230
:1087D0007F928F929F92AF92BF92CF92DF92EF9251
:1087E000FF920F931F93CF93C62FE0910C0BF0E0F5
:1087F000882309F4D9C0DF01A85FB44F8C9181119F
:10880000AFC18091200B9091210BA091220BB091D0
:10881000230B8093EB0A9093EC0AA093ED0AB0939C
:10882000EE0A8091240B9091250BA091260BB0911C
:10883000270B8093EF0A9093F00AA093F10AB0936C
:10884000F20A8091280B9091290BA0912A0BB091EC
:108850002B0B8093F30A9093F40AA093F50AB0933C
:10886000F60AC0902C0BD0902D0BE0902E0BF090C0
:108870002F0BC092F70AD092F80AE092F90AF09210
:10888000FA0AEE0FFF1FEE0FFF1FE75CFD4F20817E
:10889000318142815381662349F0609119027091C0
:1088A0001A0280911B0290911C0208C060911D0267
:1088B00070911E0280911F02909120020F94849269
:1088C0009B01AC01C701B6010F94A49160932C0BDE
:1088D00070932D0B80932E0B90932F0B8CE29BE0CB
:1088E0000E942BFE80900C0290900D02A0900E0230
:1088F000B0900F0220E030E040E752E460911502B2
:108900007091160280911702909118020F9452955F
:1089100060930C0270930D0280930E0290930F02ED
:10892000E0910C0BF0E0E85FF44F81E080834ADED9
:108930002091040B3091050B4091060B5091070BD1
:108940006091280B7091290B80912A0B90912B0B31
:108950000F94A3917B018C016093280B7093290BDA
:1089600080932A0B90932B0B2091240B3091250B95
:108970004091260B5091270B6091200B7091210B99
:108980008091220B9091230BECE2CE2EEBE0DE2EB9
:108990000E948CFC17DE80920C0290920D02A09235
:1089A0000E02B0920F02DCC0E85FF44F8081882392
:1089B00009F4D6C08090200B9090210BA090220B40
:1089C000B090230B8092EB0A9092EC0AA092ED0AF1
:1089D000B092EE0A4090240B5090250B6090260B2D
:1089E0007090270B4092EF0A5092F00A6092F10AC1
:1089F0007092F20A6091280B7091290B80912A0BDA
:108A000090912B0B6093F30A7093F40A8093F50A0C
:108A10009093F60A00912C0B10912D0B20912E0BA8
:108A200030912F0B0093F70A1093F80A2093F90A5C
:108A30003093FA0A2091040B3091050B4091060BFC
:108A40005091070B0F94A4917B018C016093280B2C
:108A50007093290B80932A0B90932B0B3CE2C32E2F
:108A60003BE0D32EA3019201C501B4010E948CFC0E
:108A700010910C0BCC2389F02091FC0A3091FD0A57
:108A80004091FE0A5091FF0A6091190270911A02FA
:108A900080911B0290911C0210C02091000B30911C
:108AA000010B4091020B5091030B60911D027091DC
:108AB0001E0280911F02909120020F94A49124E045
:108AC000129FF0011124E75CFD4F2081318142812A
:108AD00053810F9484929B01AC0160912C0B709197
:108AE0002D0B80912E0B90912F0B0F94A3916093DF
:108AF0002C0B70932D0B80932E0B90932F0B8CE2ED
:108B00009BE00E942BFEC0900C02D0900D02E090E2
:108B10000E02F0900F0220E030E040E752E4609156
:108B200011027091120280911302909114020F941D
:108B3000529560930C0270930D0280930E029093F5
:108B40000F02E0910C0BF0E0E85FF44F10823ADD89
:108B5000C0920C02D0920D02E0920E02F0920F022F
:108B6000CF911F910F91FF90EF90DF90CF90BF902A
:108B7000AF909F908F907F906F905F904F900895EF
:108B8000AF92BF92CF92DF92EF92FF920F931F931B
:108B9000CF93DF93D82F2091E30A3091E40A4091DC
:108BA000E50A5091E60A6091DF0A7091E00A80912F
:108BB000E10A9091E20A0F948D94C62F172F082F87
:108BC000F92E6091470270914802882777FD8095C1
:108BD000982F0F941F9320910C0230910D02409119
:108BE0000E0250910F020F94529520E030E040E7C2
:108BF00052E40F94849220E030E048EC52E40F9469
:108C0000849220910C0B2F93DF93FF920F931F936D
:108C1000CF935B016C01B2E0EB2E01E020E04FED61
:108C20005AE06BEE7AE080E29BE00E945EE6809183
:108C3000EB0A9091EC0AA091ED0AB091EE0A8093B4
:108C4000200B9093210BA093220BB093230B8091C8
:108C5000EF0A9091F00AA091F10AB091F20A809384
:108C6000240B9093250BA093260BB093270B809198
:108C7000F30A9091F40AA091F50AB091F60A809354
:108C8000280B9093290BA0932A0BB0932B0B809168
:108C9000F70A9091F80AA091F90AB091FA0A809324
:108CA0002C0B90932D0BA0932E0BB0932F0B0F94A6
:108CB000B0896093D20A7093D30A8093D40A9093B8
:108CC000D50A0F900F900F900F900F900F90DF919B
:108CD000CF911F910F91FF90EF90DF90CF90BF90B9
:108CE000AF900895CF93DF931F92CDB7DEB78C017D
:108CF000ECEDF9E08491882341F09091C00095FF5C
:108D0000FCCF8093C6003196F5CF70E04AE050E08A
:108D10008AED99E00E94AD30F8940F949D13179A54
:108D20001092110B169A1092120B149AE4E8FEE0BE
:108D30008491882341F09091C00095FFFCCF8093EF
:108D4000C6003196F5CFE6E0F6E285919491FC01FC
:108D50002491222341F03091C00035FFFCCF2093B5
:108D6000C6000196F4CF8091C00085FFFCCF8AE059
:108D70008093C60001151105E1F0F8018491F80116
:108D8000882349F09091C00095FFFCCF8093C600E6
:108D900031968491F5CF8091C00085FFFCCF8AE0A9
:108DA0008093C600BE016F5F7F4FC8010F94653D81
:108DB00006C0E2ECF5E2859194910F94633A7894C1
:108DC00006E010E00150110951F068EC70E080E01D
:108DD00090E00F94DF8980E00F94BC3BF3CFF894D0
:108DE000FFCFCF92DF92EF92FF920F931F93CF931B
:108DF000C82F8091701090917110039714F40E9405
:108E000036AF0F94B0890091CE0A1091CF0A20910D
:108E1000D00A3091D10AC090D20AD090D30AE09003
:108E2000D40AF090D50A6C197D098E099F0906179E
:108E300017072807390740F4012B022B032B21F0D9
:108E400064E084E998E04EDF409108025091090205
:108E500060910A0270910B02452B462B472B19F1AA
:108E60000F94B0890091D20A1091D30A2091D40AAC
:108E70003091D50A601B710B820B930B0091080295
:108E80001091090220910A0230910B020617170770
:108E90002807390740F49091941380919313981305
:108EA00002C0CC2349F0CF911F910F91FF90EF901A
:108EB000DF90CF900C940CEE179A1092110B169A2B
:108EC0001092120B149AEFCF0F949D138091C00A49
:108ED00081113DC081E08093C00A80915A10909129
:108EE0005B10A0915C10B0915D1080935610909330
:108EF0005710A0935810B0935910E4E8FEE0849105
:108F0000882341F09091C00095FFFCCF8093C6006C
:108F10003196F5CFECEFF5E285919491FC01249127
:108F2000222341F03091C00035FFFCCF2093C600D2
:108F30000196F4CF8091C00085FFFCCF8AE080933A
:108F4000C600E2EEF4E2859194910D943D3A0895C5
:108F50008091C00A0895CF93DF93EC0180910C0BB0
:108F60008093C10A84E50E945532811102C080E0DD
:108F700084C00E94C2320F94F1926093C10A6623AA
:108F8000B1F3EEE7FEE08491882341F09091C000B8
:108F900095FFFCCF8093C6003196F5CFCD36D10535
:108FA00009F435C064F4C836D105B1F0C936D1052D
:108FB00009F052C0E4EBF5E2A591B49124C0CA3D9A
:108FC000D10509F432C0CD3DD10509F045C0E8EA2C
:108FD000F5E2A591B4913DC0E6EBF5E2859194915F
:108FE000FC012491222309F437C03091C00035FFE1
:108FF000FCCF2093C6000196F3CF9091C00095FF5F
:10900000FCCF8093C6008D918111F7CF25C0E2EB94
:10901000F5E2A591B4918D918823F1F09091C00073
:1090200095FFFCCF8093C600F6CFEAEAF5E2A59162
:10903000B4918D91882381F09091C00095FFFCCF71
:109040008093C600F6CF9091C00095FFFCCF80932F
:10905000C6008D918111F7CF6091C10A70E04AE09E
:1090600050E08AED99E00E94A6308091C00085FF13
:10907000FCCF8AE08093C60081E0DF91CF91089514
:109080004F925F926F927F928F929F92AF92BF9218
:10909000CF92DF92EF92FF92CF93DF9300D01F9297
:1090A000CDB7DEB72B013C0129833A834B835C8328
:1090B0008DEE9FE00F94F09D8F3F01F58EEE9FE0C7
:1090C0000F94F09D8F3FD1F48FEE9FE00F94F09DB1
:1090D0008F3FA1F480EF9FE00F94F09D8F3F71F4DC
:1090E00040E050E0BA018DEE9FE00F94149E40E006
:1090F00050E0BA0181EF9FE00F94149E81EF9FE052
:109100000F94F89D4B015C018DEE9FE00F94F89D4C
:109110006B017C0169817A818B819C812CE330E039
:1091200040E050E00F945497C20ED31EE41EF51E8B
:10913000B701A6018DEE9FE00F94149EC301B2010A
:1091400028EE33E040E050E00F945497BA01A901B3
:10915000480D591D6A1D7B1D81EF9FE00F94149EE1
:1091600010924E0B10924F0B1092500B1092510B0D
:109170000F900F900F900F90DF91CF91FF90EF9095
:10918000DF90CF90BF90AF909F908F907F906F9027
:109190005F904F900895CF92DF92EF92FF922091CF
:1091A000300B2223F1F020E030E040E05FE30F9449
:1091B00052956B017C0120E030E0A9010F947D9273
:1091C000882379F0A7019601C701B6010F94529543
:1091D0002BED3FE049E450E40F9452959B01AC0124
:1091E00004C020E030E040E85FE360E070E080E849
:1091F0009FE30F948492FF90EF90DF90CF900895BB
:1092000060913D0270913E0280913F029091400238
:10921000C2DF6093390270933A0280933B029093CD
:109220003C020895CF93DF93EC010F94031B81E080
:10923000D8DD80E00F94BC3B209799F0C233D10574
:1092400040F062E370E080E090E00F94DF89E29705
:10925000ECCFBE0180E090E00F94DF89C0E0D0E069
:10926000E4CFDF91CF9108952F923F924F925F927A
:109270006F927F928F929F92AF92BF92CF92DF9226
:10928000EF92FF921F93CF93DF934B015C01CC24AD
:10929000CA94DC2C760151ED252E59E0352E68EE6E
:1092A000462E63E0562E612C712C1AE08091FB0A49
:1092B000811126C12FEFC216D206E206F20651F046
:1092C000F7FC1EC10F94B0896C197D09683B7B4087
:1092D00008F016C10F94B089681979098A099B09A9
:1092E000693E73408105910508F47FC08091B21BEF
:1092F000811177C0E9EDF9E08491882341F09091E4
:10930000C00095FFFCCF8093C6003196F5CFE09169
:10931000C10A24E0E29FF0011124E156F54E40819C
:1093200051816281738121E030E08AED99E00E94F1
:10933000A431E5EDF9E08491882341F09091C000DB
:1093400095FFFCCF8093C6003196F5CF6091C10A9E
:1093500070E04AE050E08AED99E00E94A630F10109
:109360008491E1EDF9E0882349F09091C00095FFE8
:10937000FCCF8093C60031968491F5CFF7FE03C0F1
:10938000E0E6F9E025C00F94B0894B015C01C7010C
:10939000B6016854744F8F4F9F4F681979098A0935
:1093A0009B09A30192010F945497BA01A9012AE0E5
:1093B00030E08AED99E00E946E308091C00085FF18
:1093C000FCCF0DC09091C00095FFFCCF8093C600EC
:1093D00081918111F7CF8091C00085FFFCCF109360
:1093E000C6000F94B0894B015C010F94031B80E011
:1093F000F8DC80E00F94BC3BFFEFCF16DF06EF06F2
:10940000FF0609F046C08091BF0AE091C10AF0E072
:10941000EF01CC0FDD1FCC0FDD1FC156D54EEE0F77
:10942000FF1FE955F54E8823D1F080819181BC0161
:10943000882777FD8095982F0F941F9320E030E0C8
:1094400040E85FE30F94A3919B01AC0168817981AF
:109450008A819B810F94809487FF4DC027CF8081A4
:109460009181BC01882777FD8095982F0F941F93D9
:1094700020E030E040E85FE30F94A4919B01AC0151
:10948000688179818A819B810F947D9218169CF561
:109490000DCFF7FC0BCFE091C10AF0E0EF01CC0F4C
:1094A000DD1FCC0FDD1FC156D54EEE0FFF1FE95556
:1094B000F54E80819181BC01882777FD8095982F9A
:1094C0000F941F939B01AC01688179818A819B81F4
:1094D0000F94A3910F94EC9297FF07C090958095FD
:1094E000709561957F4F8F4F9F4F66307105810555
:1094F00091050CF4DBCE0F94B0896B017C01D6CEC4
:10950000DF91CF911F91FF90EF90DF90CF90BF90B0
:10951000AF909F908F907F906F905F904F903F9013
:109520002F900895CF93DF931F921F92CDB7DEB790
:10953000BE016F5F7F4F88EF9FE00F946339898191
:109540009A818156904F803A9F4020F11A82198269
:10955000E8EAF9E08491882341F09091C00095FFFA
:10956000FCCF8093C6003196F5CF8091C00085FF77
:10957000FCCF8AE08093C600BE016F5F7F4F88EF0B
:109580009FE00F9452398BE699E00F943D3F81E0C4
:109590000F94293D0F900F90DF91CF9108952F9256
:1095A0003F924F925F926F927F928F929F92AF9273
:1095B000BF92CF92DF92EF92FF920F931F93CF93C0
:1095C000DF93CDB7DEB7CA58D2400FB6F894DEBFEE
:1095D0000FBECDBFC958DD4F688379838A839B83D3
:1095E000C757D240FE01E75FFD4F88E2DF011D92C1
:1095F0008A95E9F7E850F24080E991E0DF019C01AB
:109600001D9221503040E1F7C75ADD4F1982188270
:10961000C955D240CE01875A9D4F5C014E019FE64D
:10962000891A9EEF990ADE01AF51BE4F3D0190EBC2
:10963000C92E9FE0D92E23E2E22EF12C00E010E0AB
:10964000C359DD4F8882CD56D240CD58DD4F988228
:10965000C357D240B701882777FD8095982F0F9484
:109660001F93D3016D937D938D939D933D01F501E0
:10967000619171915F01882777FD8095982F0F94F4
:109680001F93D4016D937D938D939D934D010F5F37
:109690001F4F0630110559F0B501C6010F9463390B
:1096A000B5E0EB0EF11CE2E0CE0ED11CD3CFCF51D2
:1096B000DE4F288139814A815B81C15ED140C95822
:1096C000DD4F688179818A819B81C757D2400F9491
:1096D0007D9287FD2BC3FE01EF51FE4F7F016E018E
:1096E000FFE2CF1AFEEFDF0A3E012BEB621A2DEFED
:1096F000720AC359DD4F0881CD56D240CD58DD4F97
:109700001881C357D24085E090E0CF58DD4F998350
:109710008883C157D240CF58DD4FA881B981C15746
:10972000D2401197CF58DD4FB983A883C157D2409B
:10973000F70120893189428953896489758986892D
:1097400097890F94A3914B015C01D80150962D91FC
:109750003D914D915C91539754966D917D918D9172
:109760009C9157970F94A391A50194010F94849213
:10977000F60192938293729362936F01D301BE922A
:10978000AE929E928E923D0104501109B4E0EB1A04
:10979000F108CF58DD4FE881F981C157D240EF2B56
:1097A00009F0B9CF6E01FFECCF1AFDEFDF0A3E01E1
:1097B00027E4621A2EEF720A2E013DE3430E511C7C
:1097C000CE0101967C0101E010E0D6018D909D90C4
:1097D000AD90BC90139714962D913D914D915C9155
:1097E0001797C501B4010F94A4919B01AC010F948C
:1097F000A491F70164A775A786A797A70130110563
:1098000041F080A691A6A2A6B3A684829582A682E4
:10981000B7820F5F1F4FD30114962D913D914D914B
:109820005C91179718966D917D918D919C911B97E6
:109830000F94A39120E030E040EC50E40F94529557
:10984000F2016083718382839383F4E0CF0ED11C95
:109850002CE2E20EF11C34E0630E711C88E2480E2B
:10986000511C0530110509F0B0CF8E010B5A1F4F66
:109870006E0191E5C90ED11C22242394312C2C0EAB
:109880003D1EA8ED2A0E311CF801B89720813181C8
:1098900042815381F80160817181828193810F94AB
:1098A00084924B015C01E12CF12C3601F8E26F1A35
:1098B000710826014E0C5F1CF301EE0DFF1D248183
:1098C000358146815781C501B4010F9452959B01A2
:1098D000AC01D20114966D917D918D919C91179759
:1098E0000F94A391F2016483758386839783F4E0D8
:1098F000EF0EF11C24E1E216F104D9F6045D1F4FCE
:1099000038E2C30ED11C0215130509F0BDCF1E01AC
:1099100085EB280E311C6E0191EBC90ED11C3E0166
:10992000A7EE6A1AADEF7A0A14E0E12EF12C2701B6
:1099300000E010E0812C912CA12CB12CF601E00F5D
:10994000F11FD301A00FB11F2D913D914D915C915D
:1099500060817181828193810F9452959B01AC014A
:10996000B401C5010F94A4914B015C01BFEF4B1AE8
:109970005B0A0C5F1F4FE5E04E165104F9F69B01A0
:10998000AC01D1016D917D918D919C910F94A3912A
:10999000F60120813181428153810F948492D30159
:1099A0006D937D938D939C931397B1E0EB1AF1081F
:1099B000E8E22E1A3108FCE2CF1AD10824E0621A3C
:1099C0007108E114F10409F0B2CFCB50DE4F888169
:1099D0009981AA81BB81C55FD140C957DD4F88837A
:1099E0009983AA83BB83C758D2408E01075F1D4F5E
:1099F000DE01AF5CBD4FC558DD4FB983A883CB579F
:109A0000D240C359DD4F2880CD56D240CD58DD4FCE
:109A10003880C357D240FE01EF51FE4FC358DD4F8F
:109A2000F983E883CD57D240C358DD4FA881B9816F
:109A3000CD57D240CD90DD90ED90FD90C358DD4FD5
:109A4000B983A883CD57D240C958DD4F28813981C9
:109A50004A815B81C757D240C701B6010F947D92FE
:109A60001816B4F0C358DD4FE881F981CD57D240C4
:109A70002081318142815381C958DD4F68817981CC
:109A80008A819B81C757D2400F947D921816FCF4AF
:109A9000CF58DD4F28813981C157D240243031055C
:109AA00009F01FC1C957DD4F288139814A815B8187
:109AB000C758D240C958DD4F688179818A819B811E
:109AC000C757D2400F94809418160CF00AC1D801E1
:109AD00014968D919D910D90BC91A02DC158DD4F94
:109AE00088839983AA83BB83CF57D240F8014080F3
:109AF000518062807380C558DD4FA881B981CB57F2
:109B0000D2408D919D910D90BC91A02DC359DD4FF8
:109B100088839983AA83BB83CD56D240D1018D918E
:109B20009D910D90BC91A02DCD57DD4F88839983D9
:109B3000AA83BB83C358D240A7019601C958DD4F01
:109B4000688179818A819B81C757D2400F94A39104
:109B5000CD58DD4F688379838A839B83C357D24076
:109B600020E030E040E450E40F94B5956B017C01B7
:109B7000A3019201C158DD4F688179818A819B815F
:109B8000CF57D2400F94A3914B015C0120E030E00D
:109B900040EC50E4C359DD4F688179818A819B8113
:109BA000CD56D2400F9452959B01AC01C501B40132
:109BB0000F948492A70196010F9452956B017C013A
:109BC00020E030E040E05FE3C301B2010F94529522
:109BD0004B015C01CD58DD4F288139814A815B8181
:109BE000C357D240CA01B9010F9452959B01AC01F1
:109BF000C501B4010F9452959B01AC01C701B60198
:109C00000F94A4916B017C01CD57DD4F28813981E0
:109C10004A815B81C358D240F1016481758186819C
:109C200097810F94A391C359DD4F288139814A81CF
:109C30005B81CD56D2400F9484924B015C01C35995
:109C4000DD4F288139814A815B81CD56D240CA01DE
:109C5000B9010F94A491A30192010F9452952B0185
:109C60003C01C359DD4F288139814A815B81CD5642
:109C7000D240C158DD4F688179818A819B81CF575D
:109C8000D2400F9452959B01AC01C301B2010F94D5
:109C9000A49120E030E040EC50E40F9484929B01CA
:109CA000AC01C501B4010F94A391CD58DD4F2881BB
:109CB00039814A815B81C357D2400F9452959B01F1
:109CC000AC01C701B6010F94A491CD57DD4F288197
:109CD00039814A815B81C358D2400F94A4914B01D2
:109CE0005C01CF58DD4F28813981C157D2402F5FA9
:109CF0003F4FCF58DD4F39832883C157D2400C5F87
:109D00001F4FC558DD4F88819981CB57D2400496AB
:109D1000C558DD4F99838883CB57D24094E0290EF4
:109D2000311C2530310509F07FCE04C0812C912CE7
:109D3000A12CB12CB401C501C657DD4F0FB6F89464
:109D4000DEBF0FBECDBFDF91CF911F910F91FF906E
:109D5000EF90DF90CF90BF90AF909F908F907F90CB
:109D60006F905F904F903F902F9008958091860B59
:109D70008823C9F086EA9FE00F94F09D882399F02C
:109D80006091991A70919A1A80919B1A90919C1ADD
:109D900006DC209178193091791940917A19509107
:109DA0007B190D94849260E070E0CB0108954F928E
:109DB0005F926F927F928F929F92AF92BF92CF925B
:109DC000DF92EF92FF920F931F93CF93DF93CDB764
:109DD000DEB728970FB6F894DEBF0FBECDBF0F9445
:109DE0006D0980914702909148029093920B809365
:109DF000910BE0910C0BF0E0EE0FFF1FE955F54ED3
:109E000060817181882777FD8095982F0F941F932B
:109E100060937A0B70937B0B80937C0B90937D0BFC
:109E200080910A0B90910B0B9093790B8093780B98
:109E30000F94B0896093600B7093610B8093620BF9
:109E40009093630B8091200B9091210BA091220B9A
:109E5000B091230B89839A83AB83BC838093680B77
:109E60009093690BA0936A0BB0936B0B4090240BFB
:109E70005090250B6090260B7090270B40926C0B36
:109E800050926D0B60926E0B70926F0B8091280B4D
:109E90009091290BA0912A0BB0912B0B8D839E835F
:109EA000AF83B8878093700B9093710BA093720B64
:109EB000B093730B60912C0B70912D0B80912E0B36
:109EC00090912F0B6093740B7093750B8093760BAE
:109ED0009093770B20E030E040E85FE30F94A3918C
:109EE00060932C0B70932D0B80932E0B90932F0B64
:109EF0008CE09BE09F938F93812C912CB8ECAB2E40
:109F0000B3E4BB2E1CE2C12E1BE0D12EED80FE80FF
:109F10000F811885A301920169817A818B819C81CF
:109F20000E94DEEF20E030E040EA51E46091280B2F
:109F30007091290B80912A0B90912B0B0F94A49177
:109F40002B013C010F900F9020E030E042E553E4FC
:109F50000F94809418164CF04092280B5092290BC5
:109F600060922A0B70922B0B0CC080E090E0A2E56F
:109F7000B3E48093280B9093290BA0932A0BB09302
:109F80002B0BE090280BF090290B00912A0B1091DD
:109F90002B0B2091240B3091250B4091260B5091D7
:109FA000270B6091200B7091210B8091220B9091D7
:109FB000230BACE06A2EABE07A2E7F926F92812C5D
:109FC000912CB0E7AB2EB1E4BB2EECE2CE2EEBE051
:109FD000DE2E0E94DEEF1092A81A1092A71A10929D
:109FE000AA1A1092A91A1092AC1A1092AB1A80E019
:109FF00090E0A8E4B2E48093200B9093210BA0930F
:10A00000220BB093230B80E090E0AEE3B3E48093A7
:10A01000240B9093250BA093260BB093270BE09075
:10A02000280BF090290B00912A0B10912B0B7F929B
:10A030006F92812C912CF8E4AF2EF2E4BF2E9C019C
:10A04000AD01C501B4010E94DEEF10920B0B10921E
:10A050000A0B0F900F900F900F9028960FB6F89460
:10A06000DEBF0FBECDBFDF91CF911F910F91FF904B
:10A07000EF90DF90CF90BF90AF909F908F907F90A8
:10A080006F905F904F900D946D09E0910C0B84E000
:10A09000E89FF0011124E156F54E40815181628123
:10A0A0007381E8E6F9E08491882341F09091C00043
:10A0B00095FFFCCF8093C6003196F5CF22E030E0CB
:10A0C0008AED99E00E94A431E4E6F9E084918823C6
:10A0D00041F09091C00095FFFCCF8093C60031966F
:10A0E000F5CF60910C0B70E04AE050E08AED99E00A
:10A0F0000E94A630E0E6F9E08491882341F0909137
:10A10000C00095FFFCCF8093C6003196F5CF4091FB
:10A110008D1A50918E1A60918F1A7091901A21E0C9
:10A1200030E08AED99E00E94A4318091C00085FF63
:10A13000FCCF8AE08093C6000895CF93DF93CDB71C
:10A14000DEB72A970FB6F894DEBF0FBECDBF0F94CF
:10A15000B0896F83788789879A87179A1092110B35
:10A16000169A1092120BEBE5F9E08491882341F0E6
:10A170009091C00095FFFCCF8093C6003196F5CF3B
:10A180008091C00085FFFCCF8AE08093C60083E405
:10A190000F9406291C01409052105090531060906B
:10A1A0005410709055100E94B9FE481A590A61085F
:10A1B00071080E946EB4481A590A6108710877FE46
:10A1C00003C0412C512C3201909194138091931330
:10A1D000981799F0E091931327E5E29FF00111247D
:10A1E000EB56FC4E20E030E040E752E462A173A160
:10A1F00084A195A10F94529508C060910C027091B2
:10A200000D0280910E0290910F020F94EC927E83CA
:10A210006D830E9463EE0E941DAD10929D0B789499
:10A2200020E030E040E85FE360912C0B70912D0B53
:10A2300080912E0B90912F0B0F94A39169837A83B9
:10A240008B839C83E090280BF090290B00912A0BC4
:10A2500010912B0B2091240B3091250B4091260B54
:10A260005091270B6091200B7091210B8091220B54
:10A270009091230BACE0BBE0BF93AF93812C912C6A
:10A28000E8ECAE2EE3E4BE2EDE0111966D010E94D5
:10A29000DEEF20E030E040E85FE360912C0B70914E
:10A2A0002D0B80912E0B90912F0B0F94A39169830E
:10A2B0007A838B839C832FE832EC45EF5FE36091D8
:10A2C000280B7091290B80912A0B90912B0B0F94E6
:10A2D000A4916B017C0167E074E062197309F4E0FA
:10A2E00076956795FA95E1F780E090E00F941D93DD
:10A2F000209178193091791940917A1950917B19F0
:10A300000F9484929B01AC01C701B6010F94A491F4
:10A310007B018C012091240B3091250B4091260B61
:10A320005091270B6091200B7091210B8091220B93
:10A330009091230BACE0BBE0BF93AF93812C912CA9
:10A34000A0E2AA2EA2E4BA2EDE0111966D010E94AF
:10A35000DEEFB301A20181E99FE00F94149E0F90FC
:10A360000F900F900F9005E71FE0F12CB3E0EB2E5C
:10A370008091A712882341F18F2D6E2D0F94209785
:10A38000B5E18B02F001112423E09202E00DF11DF2
:10A390001124EE0FFF1FEE0FFF1FE955FD4E20E0C9
:10A3A00030E04AE754E461817281838194810F94A3
:10A3B000529520E030E040E05FE30F94A4910F94C9
:10A3C0005A930F94EC9202C060E070E0C8010F94C1
:10A3D0001C9EF3940E5F1F4F89E0F812C9CFB101A4
:10A3E00083E79FE00F941C9E4091200B5091210B1E
:10A3F0006091220B7091230B8DE99FE00F94149EC6
:10A400004091240B5091250B6091260B7091270BE6
:10A4100081EA9FE00F94149E4091280B5091290BE4
:10A4200060912A0B70912B0B8DE89FE00F94149E86
:10A43000BE016B5F7F4F89E89FE00F945239E09136
:10A440000C0BF0E0EE0FFF1FE955F54E60818CE834
:10A450009FE00F94029E6091A51A8BE89FE00F94F5
:10A46000029E60910A0B88E89FE00F94029E61E0D3
:10A4700085EA9FE00F94029E0F946D09E6E5F9E0EE
:10A480008491882341F09091C00095FFFCCF809388
:10A49000C6003196F5CF83E40F9406294AE050E0D8
:10A4A000BC018AED99E00E94033184E69FE00F949D
:10A4B000F09D61E0680F84E69FE00F94029EEBE45C
:10A4C000F9E08491882341F09091C00095FFFCCF82
:10A4D0008093C6003196F5CF8091C00085FFFCCFF8
:10A4E0008AE08093C6000F94B089AB01BC018F81D4
:10A4F0009885A985BA85481B590B6A0B7B0B2AE006
:10A5000030E08AED99E00E940F31F894FFCF6F9808
:10A510007798EAE6F0E080818F7B80838081806895
:10A520008083EF9A08951F920F920FB60F92112415
:10A530000BB60F920F931F932F933F934F935F93FD
:10A540006F937F938F939F93AF93BF93EF93FF93FB
:10A5500080910A0B90910B0B8B3491050CF441C048
:10A5600080916A0086FF0BC00F94B08960935C0BEA
:10A5700070935D0B80935E0B90935F0B2CC00F94D8
:10A58000B08900915C0B10915D0B20915E0B3091B6
:10A590005F0B601B710B820B930B20910A0B3091A8
:10A5A0000B0B253631052CF003E010E020E030E005
:10A5B00004C004E010E020E030E06017710782077B
:10A5C000930748F08091370B9091380B0296909347
:10A5D000380B8093370B80916A0090E48927809331
:10A5E0006A00FF91EF91BF91AF919F918F917F9101
:10A5F0006F915F914F913F912F911F910F910F900C
:10A600000BBE0F900FBE0F901F9018956C9874980A
:10A61000EAE6F0E080818160808380818D7F8083A5
:10A62000EC9A08951F920F920FB60F9211240BB659
:10A630000F922F933F934F935F936F937F938F93DB
:10A640009F93AF93BF93EF93FF93EC98E6E4F9E009
:10A650008491882341F09091C00095FFFCCF8093B6
:10A66000C6003196F5CF8091C00085FFFCCF8AE00F
:10A670008093C60080919D0B81115FDDFF91EF916A
:10A68000BF91AF919F918F917F916F915F914F910A
:10A690003F912F910F900BBE0F900FBE0F901F9008
:10A6A0001895BF92CF92DF92EF92FF920F931F9374
:10A6B000CF93DF93CDB7DEB7E1970FB6F894DEBF47
:10A6C0000FBECDBF88E89FE00F94F09DB82EBE016D
:10A6D000605D7F4F89E89FE00F946339EFEEF7E00C
:10A6E0008491882341F09091C00095FFFCCF809326
:10A6F000C6003196F5CF68A979A94AE050E08AED05
:10A7000099E00E94AD308E01015E1F4F85E9E82E71
:10A710008FE0F82ED02EC12EC7010F94F09DF801C6
:10A7200081938F01FFEFEF1AFF0A8DE9E8168FE0A2
:10A73000F80691F71FA2ED2DFC2D8191882339F0A9
:10A740009091C00095FFFCCF8093C600F6CF6AEED3
:10A7500077E08D2D9C2D0F949F9ACF92DF9283EE00
:10A7600097E09F938F938E010F5F1F4F1F930F935F
:10A770000F94C49B0F900F900F900F900F900F901D
:10A780007E0195E0E90EF11CF7018081882349F0F4
:10A79000992787FD90950F948E9AF70181937F01F9
:10A7A000F3CF60E0C8010E9493AD81E99FE00F9470
:10A7B000F89DF62EE72ED82EC92EE8ECF7E084910E
:10A7C000882341F09091C00095FFFCCF8093C60094
:10A7D0003196F5CF2AE030E04F2D5E2D6D2D7C2D8A
:10A7E0008AED99E00E940F3161E084EC97E00E94CD
:10A7F00093AD6FEB77E0C8010F94AA9A8DE99FE0C3
:10A800000F94F89D6CA77DA78EA79FA7CE018C966D
:10A810000F94BC41BC01C8010F94399B6CEB77E0ED
:10A82000C8010F949F9A81EA9FE00F94F89D6CA74E
:10A830007DA78EA79FA7CE018C960F94BC41BC012B
:10A84000C8010F94399B65EB77E0C8010F949F9A7C
:10A8500060E0C8010E9493AD60EB77E0C8010F94FF
:10A86000AA9A8DE89FE00F94F89D6CA77DA78EA70C
:10A870009FA7CE018C960F94BC41BC01C8010F94D8
:10A88000399B60E0C8010E9493AD61E085EA97E0E2
:10A890000E9493AD89A98F9388A98F938EE997E041
:10A8A0009F938F931F930F930F94C49B60E0C801F5
:10A8B0000E9493AD67E977E0C8010F94AA9A8B2DA7
:10A8C00090E09DA78CA7CE018C960F941E44BC01EE
:10A8D000C8010F94399B60E0C8010E9493ADCF92EC
:10A8E000DF92EF92FF928EE897E09F938F931F93F2
:10A8F0000F930F94C49B60E0C8010E9493AD61E088
:10A900008AE897E00E9493AD0FB6F894DEBF0FBEC1
:10A91000CDBFE1960FB6F894DEBF0FBECDBFDF917D
:10A92000CF911F910F91FF90EF90DF90CF90BF904C
:10A9300008954F925F926F927F92AF92BF92CF92A3
:10A94000DF92EF92FF920F931F93CF93DF93CDB7D8
:10A95000DEB7E0970FB6F894DEBF0FBECDBF2B0178
:10A960003C0169017A0180917B0A8111E5C0F8946C
:10A970000E9499FE8091521090915310A091541012
:10A98000B09155108093770A9093780AA093790A32
:10A99000B0937A0A0E94B9FE4091770A5091780AE2
:10A9A0006091790A70917A0A481B590B6109710903
:10A9B0004093770A5093780A6093790A70937A0AE1
:10A9C0000E946EB44091770A5091780A6091790A9A
:10A9D00070917A0A481B590B610971094093770AF3
:10A9E0005093780A6093790A70937A0A909194133D
:10A9F00080919313981799F0E091931387E5E89F5E
:10AA0000F0011124EB56FC4E20E030E040E752E428
:10AA100062A173A184A195A10F94529508C0609181
:10AA20000C0270910D0280910E0290910F026093C2
:10AA3000630A7093640A8093650A9093660A0E9481
:10AA400063EE80E1E0E2FBE0A7E6BAE001900D9260
:10AA50008A95E1F780910C0B8093620A809107023E
:10AA60008093610A0E941DAD10929D0B81E080933E
:10AA70007B0A789420E030E0A901C301B2010F9471
:10AA80007D9281110AC020E030E0A901C701B60122
:10AA90000F947D92882309F44FC065E877E0FE01AA
:10AAA00031965F01CF010F94AA9AF5010190002021
:10AAB000E9F78F010150110920916F0A3091700A56
:10AAC0004091710A5091720AC301B2010F94A4918E
:10AAD00023E048E00F94CD9762E877E0C5010F943A
:10AAE0009F9AF50101900020E9F78F0101501109AB
:10AAF00023E046E0C701B6010F94CD976FE777E0FA
:10AB0000C5010F949F9AF50101900020E9F78F018C
:10AB100001501109609151027091520280915302CB
:10AB20009091540223E048E00F94CD9760E0C50176
:10AB30000E9493AD0E9429AFE0960FB6F894DEBF55
:10AB40000FBECDBFDF91CF911F910F91FF90EF907E
:10AB5000DF90CF90BF90AF907F906F905F904F90BD
:10AB6000089520E030E0A90160E070E080E291E427
:10AB7000E0CE8F929F92AF92BF92CF92DF92EF92F0
:10AB8000FF920F931F93CF93DF9300D01F92CDB707
:10AB9000DEB79B01AC0180917B0A882309F497C042
:10ABA0008091620A80930C0B8091630A9091640AF1
:10ABB000A091650AB091660A80930C0290930D02F1
:10ABC000A0930E02B0930F026091730A7091740A01
:10ABD0008091750A9091760A0F94A39169837A8384
:10ABE0008B839C83CE0101960E942BFE20E030E0F7
:10ABF00040E551E4609151027091520280915302FC
:10AC0000909154020F9484924B015C01E0906F0A82
:10AC1000F090700A0091710A1091720A20916B0AEB
:10AC200030916C0A40916D0A50916E0A6091670AEA
:10AC30007091680A8091690A90916A0AECE0FBE0E1
:10AC4000FF93EF93E3E7CE2EEAE0DE2E0E94DEEFE5
:10AC50000F946D0980E1E7E6FAE0A0E2BBE0019025
:10AC60000D928A95E1F780E1E0E2FBE0ABEEBAE01D
:10AC700001900D928A95E1F74091770A5091780AF8
:10AC80006091790A70917A0A4093390E50933A0E86
:10AC900060933B0E70933C0E84E89DE00E94079504
:10ACA0008091770A9091780AA091790AB0917A0AF6
:10ACB0008093521090935310A0935410B09355105A
:10ACC00081E080939D0B10927B0A0F900F900F9064
:10ACD0000F900F900F90DF91CF911F910F91FF90E8
:10ACE000EF90DF90CF90BF90AF909F908F9008959E
:10ACF00060E070E0CB013DCFEAE6F7E08491882385
:10AD000041F09091C00095FFFCCF8093C600319632
:10AD1000F5CF4091200B5091210B6091220B709147
:10AD2000230B23E030E08AED99E00E94A431E7E6AE
:10AD3000F7E08491882341F09091C00095FFFCCF0B
:10AD40008093C6003196F5CF4091240B5091250B8E
:10AD50006091260B7091270B23E030E08AED99E09B
:10AD60000E94A431E4E6F7E08491882341F09091B9
:10AD7000C00095FFFCCF8093C6003196F5CF40917F
:10AD8000280B5091290B60912A0B70912B0B23E01B
:10AD900030E08AED99E00E94A431E2E6F7E0849188
:10ADA000882341F09091C00095FFFCCF8093C600AE
:10ADB0003196F5CF8091C00085FFFCCF8AE080936B
:10ADC000C6000895EAE4F7E08491882341F0909169
:10ADD000C00095FFFCCF8093C6003196F5CF0F944D
:10ADE000DC09AB01BC0123E030E08AED99E00E9470
:10ADF000A431E7E4F7E08491882341F09091C0000A
:10AE000095FFFCCF8093C6003196F5CF81E00F947B
:10AE1000DC09AB01BC0123E030E08AED99E00E943F
:10AE2000A431E4E4F7E08491882341F09091C000DC
:10AE300095FFFCCF8093C6003196F5CF82E00F944A
:10AE4000DC09AB01BC0123E030E08AED99E00E940F
:10AE5000A431E2E4F7E08491882341F09091C000AE
:10AE600095FFFCCF8093C6003196F5CF8091C0004E
:10AE700085FFFCCF8AE08093C6000895EF92FF9291
:10AE80000F931F93CF93DF93EEE2F7E08491882333
:10AE900041F09091C00095FFFCCF8093C6003196A1
:10AEA000F5CF07EA12E1FCE2EF2EF7E0FF2EC0E05B
:10AEB000D0E0F801EC0FFD1F418152816381748164
:10AEC00023E030E08AED99E00E94A431F7018491FB
:10AED000ECE2F7E0882349F09091C00095FFFCCFA9
:10AEE0008093C60031968491F5CF2496CC31D1055C
:10AEF00001F7045E1F4FF3E10B361F07C1F6EBE2CB
:10AF0000F7E08491882341F09091C00095FFFCCF39
:10AF10008093C6003196F5CF8091C00085FFFCCFAD
:10AF20008AE08093C600DF91CF911F910F91FF902F
:10AF3000EF9008952F923F924F925F926F927F927F
:10AF40008F929F92AF92BF92CF92DF92EF92FF9239
:10AF50000F931F93CF93DF93CDB7DEB7C555D109BC
:10AF60000FB6F894DEBF0FBECDBF8BE994E00E9410
:10AF70006B328823B1F080916A1090916B106AE275
:10AF800070E005960F94449B009711F0DC011C9231
:10AF900080916A1090916B1005960F94303A0C9442
:10AFA000528580EA94E00E946B32882309F4C4C180
:10AFB00086EA94E00E946B32882391F08091B21B64
:10AFC000882311F40C9452850F94B0896093970BE9
:10AFD0007093980B8093990B90939A0B0C945285D5
:10AFE0008BEA94E00E946B32882361F06091520BEF
:10AFF0007091530B4AE050E08AED99E00E940331D2
:10B000000C9452858FEA94E00E946B32882309F4F5
:10B0100046C0E3EBF4E08191882339F09091C000C1
:10B0200095FFFCCF8093C600F6CF8091310B9091B5
:10B03000320B2CE3289FB001299F700D11244AE0A8
:10B0400050E08AED99E00E94A63067EB74E08AED4B
:10B0500099E00E949930ECEBF4E08191882339F07B
:10B060009091C00095FFFCCF8093C600F6CF8091F1
:10B07000330B9091340B2CE3289FB001299F700D66
:10B0800011244AE050E08AED99E00E94A63067EB77
:10B0900074E08AED99E00E9499300C94528582EC1C
:10B0A00094E00E946B328823C1F08091B21B882308
:10B0B00061F06091B01B7091B11B4AE050E08AEDE5
:10B0C00099E00E94AD300C94528565EC74E08AEDF5
:10B0D00099E00E9499300C94528587ED94E00E948B
:10B0E0006B32882379F160916A1070916B106D5FFB
:10B0F0007F4F21E041E08BE99BE00E9455A78091C2
:10B100008C0D90918D0DA0918E0DB0918F0D80932F
:10B11000390E90933A0EA0933B0EB0933C0E84E808
:10B120009DE00E943E942091C00025FFFCCF8093BB
:10B13000C6000A9721F760E08BE99BE00E94E5A634
:10B140000C9452858AED94E00E946B32882399F02A
:10B150000E94FF3E81E08093540B60916A107091D1
:10B160006B106C5F7F4F21E040E08BE99BE00E9419
:10B1700055A70C9452858EED94E00E946B32882383
:10B1800009F445C08091B21B882309F49ECF109228
:10B190005F0AE1EEF4E08191882339F09091C000DC
:10B1A00095FFFCCF8093C600F6CF00E010E0FF24AF
:10B1B000F39480915B0A90915C0A20915D0A309132
:10B1C0005E0A821B930B8F779927892B89F08AED72
:10B1D00099E00E94B32FF0925F0A9091C00095FF12
:10B1E000FCCF8093C6000F5F1F4F10925F0AE1CF24
:10B1F00003311105F4F281E080935F0A8091C00071
:10B2000085FFFCCF8AE08093C6000C94528584EEC3
:10B2100094E00E946B328823A9F0E8EEF4E081917B
:10B22000882339F09091C00095FFFCCF8093C60031
:10B23000F6CF8091C00085FFFCCF8AE08093C600E6
:10B240000C94528583EF94E00E946B328823A9F01E
:10B25000E7EFF4E08191882339F09091C00095FFE9
:10B26000FCCF8093C600F6CF8091C00085FFFCCF55
:10B270008AE08093C6000C94528585E195E00E9497
:10B280006B32882321F00F94CE390C9452858AE1D9
:10B2900095E00E946B32882341F060E070E088EF17
:10B2A0009FE00F9452390C9452858DE195E00E94F5
:10B2B0006B32882359F06DE175E08AED99E00E94C8
:10B2C000993040E052EC61E070E010C088E295E017
:10B2D0000E946B32882381F068E275E08AED99E084
:10B2E0000E94993040E054E961E170E08AED99E014
:10B2F0000E94382F0C94CA8684E395E00E946B323A
:10B30000882361F00F94B0896093820B7093830B54
:10B310008093840B9093850B0C94528589E395E080
:10B320000E946B32882311F40C94528561E080E016
:10B330000E94E3360C9452858EE50E9455328111AD
:10B340000C94528587E40E945532882311F40C94A2
:10B3500005690E94C2320F94EC926C34710509F4B5
:10B3600030C47CF56430710509F409C154F46230CD
:10B37000710509F4ECC00CF0F6C077FF78C00C94AE
:10B3800052856C31710509F451C17CF46A30710544
:10B3900009F446C16B30710511F00C94528560E0E0
:10B3A00080E00E94E5430C9452856E31710509F4EA
:10B3B0004DC36B34710511F00C94528508E210E016
:10B3C000F6C36735710511F40C94856814F5603582
:10B3D000710511F40C94B9626CF46F34710511F0BD
:10B3E0000C9452850FEF10E0A2EDCA2EABE0DA2EDE
:10B3F0000C94A4626135710511F40C94CC67663528
:10B40000710511F00C94528586EE0E949A360C94C8
:10B4100052856C35710511F40C948E687CF46A3594
:10B42000710511F40C948A686B35710511F00C9458
:10B43000528581E08093D60A0C945285623671055C
:10B4400011F40C94F0686336710511F00C94528578
:10B450001092B21B0F94D3396091B21B84EC9FE021
:10B460000F94029E82E00F94BC3B0C945285809115
:10B47000C00A81110C9452850E941A4060914E0BB3
:10B4800070914F0B8091500B9091510B0F941D9325
:10B490004B015C01C0902C0BD0902D0BE0902E0B3B
:10B4A000F0902F0B4090F70A5090F80A6090F90A3C
:10B4B0007090FA0AA3019201C701B6010F94A391FB
:10B4C00020E030E048EC52E40F9452959B01AC012F
:10B4D000C501B4010F9480941816E4F4A7019601F5
:10B4E000C301B2010F94A39120E030E048EC52E494
:10B4F0000F9452959B01AC01C501B4010F94A49126
:10B500000F94F19260934E0B70934F0B8093500BFE
:10B510009093510B8091090B8823A9F088E50E9434
:10B520005532811110C089E50E94553281110BC03E
:10B530008AE50E945532811106C085E40E94553289
:10B5400081110C9455850E94E2420C9452858091A1
:10B55000C00A81110C9452850E949D4081E00E9496
:10B56000C0450C9452858091C00A81110C9452857B
:10B570000E949D4080E00E94C0450C94528580E569
:10B580000E945532882339F00E94C2320F94F19202
:10B590004B015C0103C0812C912C540183E50E9476
:10B5A0005532882361F00E94C23220E030E04AE741
:10B5B00054E40F9452950F94F1924B015C01811465
:10B5C0009104A104B10431F0E6E1F6E28591949191
:10B5D0000F943D3A0F946D090F94B0892B013C01F3
:10B5E000480C591C6A1C7B1C0F94B0896093D20ACA
:10B5F0007093D30A8093D40A9093D50A0F94B0899C
:10B60000641575058605970510F00C9452850F9406
:10B61000031B80E00E94F14680E00F94BC3BEECF1C
:10B6200060E081E00E94E5430C9452850F946D091F
:10B63000E0E0FDE08491882341F09091C00095FF07
:10B64000FCCF8093C6003196F5CF56DBE2EFFCE0ED
:10B650008491882341F09091C00095FFFCCF8093A6
:10B66000C6003196F5CFAEDB81E08093870B88E58D
:10B670000E945532182F89E50E945532082F8AE51D
:10B680000E945532782E101308C0181711F0012FA0
:10B6900004C07724739401E011E00E9435C66090E5
:10B6A000A7121092A71282E00F94DC096093280B76
:10B6B0007093290B80932A0B90932B0B71100E948F
:10B6C000AFE340910C0250910D0260910E02709117
:10B6D0000F024093D70A5093D80A6093D90A709307
:10B6E000DA0A80914702909148029093920B8093DE
:10B6F000910B84E690E090934802809347020F9468
:10B70000B0896093D20A7093D30A8093D40A90933D
:10B71000D50A81E00E94FAFF80E1E0E2FBE0ABEEB7
:10B72000BAE001900D928A95E1F710920C02109206
:10B730000D0210920E0210920F02112321F080E0F0
:10B7400090E00E949F3A002321F081E090E00E9467
:10B750009F3A88E50E945532882341F00E947F324B
:10B76000672B682B692B11F00C94848589E50E9466
:10B770005532882341F00E947F32672B682B692B5A
:10B7800011F00C949A85772009F4F1C08091110B87
:10B79000882321F08091120B811108C080E090E095
:10B7A0000E949F3A81E090E00E949F3A0E948AC6E0
:10B7B000EEEBF8E285919591A591B49189839A83F6
:10B7C000AB83BC83EAEBF8E285919591A591B491A6
:10B7D0008F8F98A3A9A3BAA32FEE3AE04BEE5AE0BD
:10B7E000BE016F5F7F4FCE014F960E94C9340E9409
:10B7F000FCC520E030E040E451EC6091EF0A70912C
:10B80000F00A8091F10A9091F20A0F947D9287FFDD
:10B810000CC080E090E0A0E4B1EC8093EF0A90933C
:10B82000F00AA093F10AB093F20A80E090E0A0EA57
:10B83000B0E48093F30A9093F40AA093F50AB093CE
:10B84000F60A20E030E040E251E46091510270914C
:10B85000520280915302909154020F94849260930B
:10B860000C0270930D0280930E0290930F021092BF
:10B87000280B1092290B10922A0B10922B0B80E0B0
:10B880000E94FAFFE090280BF090290B00912A0B00
:10B8900010912B0B2091240B3091250B4091260BFE
:10B8A0005091270B6091200B7091210B8091220BFE
:10B8B0009091230BFCE2CF2EFBE0DF2E0E948CFC4C
:10B8C00080900C0290900D02A0900E02B0900F029A
:10B8D000E090F30AF090F40A0091F50A1091F60A4C
:10B8E0002091EF0A3091F00A4091F10A5091F20A4A
:10B8F0006091EB0A7091EC0A8091ED0A9091EE0A4A
:10B90000ECE0FBE0FF93EF93A7EFCA2EAAE0DA2E5C
:10B910000E94DEEF0F946D098091EB0A9091EC0A82
:10B92000A091ED0AB091EE0A8093200B9093210B29
:10B93000A093220BB093230B8091EF0A9091F00A11
:10B94000A091F10AB091F20A8093240B9093250BF9
:10B95000A093260BB093270B81E00E94FAFF0E9470
:10B96000E2FF82E090E00E949F3A0F900F908AE5FC
:10B970000E945532882341F00E947F32672B682B4A
:10B98000692B11F00C94B085E090280BF090290BF6
:10B9900000912A0B10912B0B2091240B3091250B39
:10B9A0004091260B5091270B6091200B7091210B39
:10B9B0008091220B9091230BECE2CE2EEBE0DE2E59
:10B9C0000E948CFC80E00E94FAFF8091D70A90913F
:10B9D000D80AA091D90AB091DA0A80930C02909308
:10B9E0000D02A0930E02B0930F028091910B9091E3
:10B9F000920B90934802809347020F94B089609312
:10BA0000D20A7093D30A8093D40A9093D50A0E94E5
:10BA1000E2FF0E948AC60E94A6C888E50E945532AD
:10BA200081110C94C68589E50E94553281110C94D0
:10BA3000C68587E50E94553281110C94C6858AE53A
:10BA40000E94553281110C94C6858FC50F946D09E3
:10BA500081E00E9401328091510290915202A091A6
:10BA60005302B091540280930C0290930D02A09364
:10BA70000E02B0930F0220E030E043E060E070E09F
:10BA800080E291EC0E9435C9E2E6F6E2859194915C
:10BA9000FC012491222341F03091C00035FFFCCFFE
:10BAA0002093C6000196F4CFE9ECFCE08491882352
:10BAB00041F09091C00095FFFCCF8093C600319675
:10BAC000F5CF4091200B5091210B6091220B70918A
:10BAD000230B25E030E08AED99E00E94A431E4ECEC
:10BAE000FCE08491882341F09091C00095FFFCCF49
:10BAF0008093C6003196F5CF4091240B5091250BD1
:10BB00006091260B7091270B25E030E08AED99E0DB
:10BB10000E94A431EFEBFCE08491882341F09091E6
:10BB2000C00095FFFCCF8093C6003196F5CF4091C1
:10BB3000280B5091290B60912A0B70912B0B25E05B
:10BB400030E08AED99E00E94A431EDEBFCE08491B5
:10BB5000882341F09091C00095FFFCCF8093C600F0
:10BB60003196F5CF0E942F320C9452859091C000EF
:10BB700095FFFCCF8093C60081918111F7CFB8016A
:10BB8000882777FD8095982F0F941F930E94CF4AA6
:10BB9000AB01BC0122E030E08AED99E00E94A531C2
:10BBA0000F5F1F4F0F36110511F40C9452854AE0B8
:10BBB00050E0B8018AED99E00E94A630E4E5F9E092
:10BBC000DBCF8091110B882341F08091120B8823E9
:10BBD00021F08091130B811109C00E9429AF61E00F
:10BBE00086EB9CE00E9471AE0C945285E8E9FCE083
:10BBF0008491882341F09091C00095FFFCCF809301
:10BC0000C6003196F5CF8091C00085FFFCCF8AE059
:10BC10008093C6001A8219828090991A90909A1A7D
:10BC2000A0909B1AB0909C1A20E030E040EA50E4CB
:10BC3000C501B4010F9484920F94EC9245E0469FA5
:10BC40009001479F300D1124B901882777FD809519
:10BC5000982F0F941F932B013C0120E030E04CE023
:10BC600052E40F947D9287FF06C0412C512C9CE03A
:10BC7000692E92E4792EA5019401C301B2010F94BB
:10BC80007D9287FF0AC020E030E040EA50E4C30123
:10BC9000B2010F94A4912B013C01E4E8FCE08491F3
:10BCA000882341F09091C00095FFFCCF8093C6009F
:10BCB0003196F5CF22E030E0B301A2018AED99E0A0
:10BCC0000E94A53120E030E040EF51E4C301B20111
:10BCD0000F94A39120E030E040E251E40F9452959C
:10BCE00020E030E040EA50E40F94849220E030E01D
:10BCF00048E452E40F94A4910F94EC927093A61A26
:10BD00006093A51A84E090E09093470B8093460BD4
:10BD100081E090E09093450B8093440BEAEDF4E2D0
:10BD20008591949121E0892B09F420E02093490B1F
:10BD300080E090E0ACE8B2E48093200B9093210B7C
:10BD4000A093220BB093230B80E090E0A0E4B0EC32
:10BD50008093240B9093250BA093260BB093270B75
:10BD600080E090E0A0E8BFE38093280B9093290B3C
:10BD7000A0932A0BB0932B0B8CE09BE09F938F93A7
:10BD8000812C912C18E4A12E12E4B12E0CE2C02ECD
:10BD90000BE0D02EE12CF12C00E81FE320E030E096
:10BDA00040E450EC60E070E08CE892E40E94DEEF4A
:10BDB0000F946D090F900F90A30192016091991A51
:10BDC00070919A1A80919B1A90919C1A0F947D926F
:10BDD00087FF07C088EE93E00E9412490E944550F9
:10BDE000EBCF60E086EA9FE00F94029E80E090E057
:10BDF000A0EAB0E48093280B9093290BA0932A0B20
:10BE0000B0932B0B2091240B3091250B4091260BE6
:10BE10005091270B6091200B7091210B8091220B88
:10BE20009091230BECE0FBE0FF93EF93812C912C9E
:10BE3000E8E4AE2EE2E4BE2EFCE2CF2EFBE0DF2EE5
:10BE4000E12CF12C00EA10E40E94DEEFEAEBF8E2CC
:10BE500085919591A591B4918093200B9093210B9E
:10BE6000A093220BB093230BEEEBF8E225913591D2
:10BE7000459154912093240B3093250B4093260B2E
:10BE80005093270BE090280BF090290B00912A0B80
:10BE900010912B0B6091200B7091210B8091220B44
:10BEA0009091230BECE0FBE0FF93EF93812C912C1E
:10BEB000B8E4AB2EB2E4BB2E0E94DEEF0F946D0906
:10BEC00020E030E043E060E070E080E89FEB0E941B
:10BED00035C98091280B9091290BA0912A0BB09124
:10BEE0002B0B24968CAF9DAFAEAFBFAF2497E3E88A
:10BEF000FCE084910F900F900F900F904091280BD1
:10BF00005091290B60912A0B70912B0B882349F0DB
:10BF10009091C00095FFFCCF8093C600319684912C
:10BF2000F5CF8091C00085FFFCCF8AE08093C600EA
:10BF3000ECE7FCE08491882341F09091C00095FFEC
:10BF4000FCCF8093C6003196F5CF22E030E08AED39
:10BF500099E00E94A431EBE7FCE08491882341F052
:10BF60009091C00095FFFCCF8093C6003196F5CF2D
:10BF70008091C00085FFFCCF8AE08093C6002EEA46
:10BF8000A22E2FE0B22E33E2E32EF12C0FEF1FEFA3
:10BF90004AE0D42E54E4252E5CE0352E63E4862E50
:10BFA0006CE0962EB701882777FD8095982F0F9427
:10BFB0001F9368AF79AF8AAF9BAFE4E7FCE0849151
:10BFC000882341F09091C00095FFFCCF8093C6007C
:10BFD0003196F5CF4AE050E0B8016E5F7F4F8AEDB1
:10BFE00099E00E94A630E7E6FCE08491882341F0C6
:10BFF0009091C00095FFFCCF8093C6003196F5CF9D
:10C000008091C00085FFFCCFD092C600E3E5FCE044
:10C010008491882341F09091C00095FFFCCF8093DC
:10C02000C6003196F5CF4AE050E0B7018AED99E0BD
:10C030000E94A630F1018491E4E4FCE0882349F0F9
:10C040009091C00095FFFCCF8093C60031968491FB
:10C05000F5CF4AE050E060E070E08AED99E00E94A0
:10C06000A630F4018491E3E4FCE0882349F0909148
:10C07000C00095FFFCCF8093C60031968491F5CF28
:10C080008091C00085FFFCCFD092C6000F3FFFEF2C
:10C090001F0731F0BE016F5F7F4FC5010F9452390A
:10C0A00028AD39AD4AAD5BADC301B2010F947D92AD
:10C0B000181664F40F5F1F4F25E0E20EF11C32E00A
:10C0C000A30EB11C0530110509F06CCF280167E201
:10C0D000461A68EF560A440C551C380183E0680E76
:10C0E000711C85E0809F1001819F300C112419AED6
:10C0F00018AE9DE2290E311CC301029705970CF082
:10C10000C7C168AD79AD620D731D882777FD809535
:10C11000982F0F941F936CAF7DAF8EAF9FAFECE362
:10C12000FCE08491882341F09091C00095FFFCCF02
:10C130008093C6003196F5CF4AE050E0B3018AED16
:10C1400099E00E94A630E9E3FCE08491882341F065
:10C150009091C00095FFFCCF8093C6003196F5CF3B
:10C160008091C00085FFFCCFFAE0F093C60070928A
:10C17000450B6092440B20E030E040EF51E46CADA1
:10C180007DAD8EAD9FAD0F94A39120E030E040E2F5
:10C1900051E40F94529520E030E040EA50E40F94CF
:10C1A000849220E030E048E452E40F94A4910F948C
:10C1B000EC927093A61A6093A51A80E090E0ACE828
:10C1C000B2E48093200B9093210BA093220BB093A9
:10C1D000230B80E090E0A0E4B0EC8093240B9093DC
:10C1E000250BA093260BB093270B80E090E0A0E8EE
:10C1F000BFE38093280B9093290BA0932A0BB09355
:10C200002B0BACE0BBE0BF93AF93812C912CA8E447
:10C21000AA2EA2E4BA2EBCE2CB2EBBE0DB2EE12C90
:10C22000F12C00E81FE320E030E040E450EC60E057
:10C2300070E08CE892E40E94DEEF0F946D090F909D
:10C240000F902CAD3DAD4EAD5FAD6091991A7091E0
:10C250009A1A80919B1A90919C1A0F947D9287FF55
:10C2600007C088EE93E00E9412490E944550E9CF32
:10C2700080E090E0A0EAB0E48093280B9093290B33
:10C28000A0932A0BB0932B0B2091240B3091250BFC
:10C290004091260B5091270B6091200B7091210B40
:10C2A0008091220B9091230BACE0BBE0BF93AF9346
:10C2B000812C912CB8E4AB2EB2E4BB2E1CE2C12E33
:10C2C0001BE0D12EE12CF12C00EA10E40E94DEEFFD
:10C2D000EAEBF8E285919591A591B4918093200BBA
:10C2E0009093210BA093220BB093230BEEEBF8E27B
:10C2F00025913591459154912093240B3093250B32
:10C300004093260B5093270BE090280BF090290BBD
:10C3100000912A0B10912B0B6091200B7091210B37
:10C320008091220B9091230BACE0BBE0BF93AF93C5
:10C33000812C912CF8E4AF2EF2E4BF2E0E94DEEFA8
:10C340000F946D0920E030E043E060E070E080E8A9
:10C350009FEB0E9435C924962CAD3DAD4EAD5FAD2F
:10C3600024976091280B7091290B80912A0B909152
:10C370002B0B0F94A391209178193091791940914A
:10C380007A1950917B190F9452950F94EC927A83FD
:10C390006983E8E3FCE084910F900F900F900F9079
:10C3A000882349F09091C00095FFFCCF8093C60090
:10C3B00031968491F5CF8091C00085FFFCCFFAE0E3
:10C3C000F093C600E4E2FCE08491882341F0909170
:10C3D000C00095FFFCCF8093C6003196F5CF409109
:10C3E000991A50919A1A60919B1A70919C1A22E0A6
:10C3F00030E08AED99E00E94A431E5E1FCE084910F
:10C40000882341F09091C00095FFFCCF8093C60037
:10C410003196F5CF24962CAD3DAD4EAD5FAD249752
:10C420006091280B7091290B80912A0B90912B0B16
:10C430000F94A391AB01BC0122E030E08AED99E0BA
:10C440000E94A431E4E1FCE08491882341F09091C2
:10C45000C00095FFFCCF8093C6003196F5CF809148
:10C46000C00085FFFCCFFAE0F093C600BE016F5F0D
:10C470007F4FC2010F94523922E0420E511C3FEF10
:10C48000631A730A88AD99AD059699AF88AF34CE1B
:10C490001092470B1092460B1092490B61E086EA0E
:10C4A0009FE00F94029EE5EDFBE08491882341F02C
:10C4B0009091C00095FFFCCF8093C6003196F5CFD8
:10C4C0008091C00085FFFCCF8AE08093C600179A58
:10C4D0001092110B169A1092120B149AE8EDF4E2D6
:10C4E000859194910F943D3F81E00F94293D82E026
:10C4F0000F94BC3B1092A61A1092A51A0C94528568
:10C5000084E690E00E94124991E0E91AF108C1F72F
:10C510004AE050E0B8018AED99E00E94A630F601A9
:10C520002491E2EDFBE0211117C06091330B709173
:10C53000340B4AE050E08AED99E00E94AD3005509E
:10C54000110911F40C94528510930B0B00930A0BF4
:10C55000F4E6EF2EF12CD4CF3091C00035FFFCCFA4
:10C560002093C60031962491DECF0F946D0910926E
:10C57000870B81E08093570B86E50E945532882314
:10C5800059F0E0916A10F0916B108181893021F0AF
:10C590008F7D11F00E948A322091110B8091B61B81
:10C5A0009091B71B222341F02091120B222321F0FE
:10C5B0002091130B21110FC0029749F00E9429AF5F
:10C5C00061E08BEC9BE00E9471AE0C94528510925E
:10C5D000570B0C9452851092600A029721F4109226
:10C5E000570B0C945285F091490B2A96FFAF2A976E
:10C5F0002091460B3091470B2C963FAF2EAF2C97D6
:10C600008091440B9091450B2E969FAF8EAF2E9745
:10C6100081E08093490B81E090E09093470B8093F9
:10C62000460B83E190E09093450B8093440B81E0AF
:10C630000F94BC3B87EA92E10E9479E40E94AFE349
:10C6400080E090E0A0EAB0E48093280B9093290B5F
:10C65000A0932A0BB0932B0B20E030E040E752E48C
:10C660006091510270915202809153029091540254
:10C670000F9484924B015C012091240B3091250B87
:10C680004091260B5091270B6091200B7091210B4C
:10C690008091220B9091230BECE0FBE0FF93EF9352
:10C6A000BCE2CB2EBBE0DB2EE12CF12C00EA10E447
:10C6B0000E94DEEFEAEBF8E285919591A591B491A5
:10C6C0008093200B9093210BA093220BB093230B0C
:10C6D000EEEBF8E285919591A591B4918093240BAE
:10C6E0009093250BA093260BB093270B64E27BE07D
:10C6F00080E29BE00E94833520E030E040EF51E48F
:10C700006091490270914A0280914B0290914C02D3
:10C710000F9484924B015C01E090280BF090290B60
:10C7200000912A0B10912B0B2091240B3091250B9B
:10C730004091260B5091270B6091200B7091210B9B
:10C740008091220B9091230BECE0FBE0FF93EF93A1
:10C750000E94DEEF0F946D0920E030E040EA51E4E2
:10C760006091490270914A0280914B0290914C0273
:10C770000F9484920F94EC928B0120E030E040E221
:10C7800052E4609151027091520280915302909153
:10C7900054020F9484920F94EC927B010E94E8C59E
:10C7A00025968FAF259780E00E9401320F900F9061
:10C7B0000F900F90AAEBB8E22296BFAFAEAF2297D0
:10C7C000212C312CC701AA2797FDA095BA2F62967C
:10C7D0008CAF9DAFAEAFBFAF6297C801AA2797FDE0
:10C7E000A095BA2F66968CAF9DAFAEAFBFAF6697E0
:10C7F000C10163E070E00F9441977DAF6CAF99AFDA
:10C8000088AF60FF06C0A2E0B0E0A81BB90BB9AFCB
:10C81000A8AF2596BFAD2597BB2379F1211431042C
:10C8200061F18CAD9DAD880F991FECADFDAD8E0F04
:10C830009F1F28AD39AD820F931F880F991F8D530D
:10C84000904F0F94FD9DBC01882777FD8095982F10
:10C850000F941F932AE037ED43E25CE30F94529567
:10C860002091A8123091A9124091AA125091AB12B6
:10C870000F94A4912B013C0103C0412C512C320197
:10C8800080E090E0A0EAB0E48093280B9093290B1D
:10C89000A0932A0BB0932B0B62966CAD7DAD8EAD41
:10C8A0009FAD62970F941F9329966CAF7DAF8EAFAB
:10C8B0009FAF29972091240B3091250B4091260B97
:10C8C0005091270B6091200B7091210B8091220BCE
:10C8D0009091230BACE0BBE0BF93AF9329968CAC57
:10C8E0009DACAEACBFAC2997BCE2CB2EBBE0DB2E3F
:10C8F000E12CF12C00EA10E40E94DEEF0F946D09A8
:10C900002296EEADFFAD229785919591A591B491B8
:10C910008093200B9093210BA093220BB093230BB9
:10C920002296EEADFFAD2297349685919591A59113
:10C93000B4918093240B9093250BA093260BB09376
:10C94000270B64E27BE080E29BE00E9483356696E1
:10C950006CAD7DAD8EAD9FAD66970F941F934B016F
:10C960005C01E090280BF090290B00912A0B1091AC
:10C970002B0B2091240B3091250B4091260B5091CD
:10C98000270B6091200B7091210B8091220B9091CD
:10C99000230BACE0BBE0BF93AF930E94DEEF0F949C
:10C9A0006D090F900F900F900F902596FFAD259772
:10C9B000FF2361F02114310449F020E030E040E829
:10C9C0005FE3C301B2010F94A39104C060E070E083
:10C9D00080E291EC20E030E043E00E9435C9811113
:10C9E00003C0EEE4F6E21AC08090280B9090290B69
:10C9F000A0902A0BB0902B0BA501940160E070E091
:10CA000080EA90E40F94A3912DEC3CEC4CEC5DE3B8
:10CA10000F947D9287FF05C0ECE4F6E26590749078
:10CA20005DC025962FAD2597222391F0A501940195
:10CA3000C301B2010F94A3919F7720E030E040E85A
:10CA40005FE30F94809418161CF4E0E5F6E2E6CF5D
:10CA50000E94B64E9B01AC01A7E08CAD9DADA89F96
:10CA60008001A99F100D1124E8ADF9AD0E0F1F1F15
:10CA7000000F111F000F111F09551D4E6091280B4B
:10CA80007091290B80912A0B90912B0B0F94A391FD
:10CA9000D80111966D937D938D939C9314978091FB
:10CAA000440B9091450B01979093450B8093440B59
:10CAB000BFEF2B1A3B0A81E00F94BC3B2296EEADF0
:10CAC000FFAD229738962296FFAFEEAF2297F9E09E
:10CAD0002F16310409F08CCE612C712C80E090E08F
:10CAE000A0EAB0E48093280B9093290BA0932A0B23
:10CAF000B0932B0B2091240B3091250B4091260BEA
:10CB00005091270B6091200B7091210B8091220B8B
:10CB10009091230BECE0FBE0FF93EF9329968CAC14
:10CB20009DACAEACBFAC2997ECE2CE2EEBE0DE2E96
:10CB3000E12CF12C00EA10E40E94DEEF0F946D0965
:10CB40000F900F9029E02216310421F060E0C3011C
:10CB50000C9406700E942F32E8EBFBE0849188234E
:10CB600041F09091C00095FFFCCF8093C6003196B4
:10CB7000F5CF8091C00085FFFCCF8AE08093C6008E
:10CB80000E9497E3E7EAFBE08491882341F09091CB
:10CB9000C00095FFFCCF8093C6003196F5CF809101
:10CBA000C00085FFFCCF8AE08093C60080EC9FE048
:10CBB0000F94F09DE82ECE0101966C01F12C2CE42F
:10CBC000622E36E4732E698292E59A837B8282E438
:10CBD0008C83D6018D916D010E945532882319F006
:10CBE0000E947F321DC0B1E0EB1235C1BF1528F0A5
:10CBF000F11009C08FEB9FE00BC0E2E0FE1206C00F
:10CC00008DEB9FE005C08EEB9FE002C08CEB9FE0B8
:10CC10000F94F09D682F772767FD7095872F972FCA
:10CC2000611571058105910509F415C10F941F93D4
:10CC30002FE632E143E85AE30F9452954B015C0131
:10CC40009F7727E139ED4EEC5DE30F948094181641
:10CC50000CF037C0E4E8FEE08491882341F0909125
:10CC6000C00095FFFCCF8093C6003196F5CFE3E876
:10CC7000FBE08491882341F09091C00095FFFCCFA8
:10CC80008093C6003196F5CF22E030E0B501A401D3
:10CC90008AED99E00E94A431EAE7FBE084918823C1
:10CCA00041F09091C00095FFFCCF8093C600319673
:10CCB000F5CF8091C00085FFFCCF8AE08093C6004D
:10CCC000CAC0F2E0FF1609F469C023E0F21609F4C5
:10CCD00094C031E0F31689F120E030E040E05FE3FA
:10CCE000C501B4010F9452951B012C0108EA12E111
:10CCF000A2019101D80114966D917D918D919C9125
:10CD000017970F94A491F8016483758386839783A2
:10CD1000A501940160817181828193810F94A49116
:10CD2000D8016D937D938D939C931397045E1F4F51
:10CD3000B2E10C3F1B07E1F68EC020E030E040E09E
:10CD40005FE3C501B4010F9452951B012C010CEA5D
:10CD500012E1A2019101F8016081718182819381C8
:10CD60000F94A491D8016D937D938D939C93139709
:10CD7000A501940114966D917D918D919C911797C9
:10CD80000F94A491F8016483758386839783045E6E
:10CD90001F4FF3E100301F07E1F65DC020E030E0F7
:10CDA00040E05FE3C501B4010F9452951B012C01D3
:10CDB00008EA12E1A2019101D8015C966D917D9182
:10CDC0008D919C915F970F94A491F801648F758F5A
:10CDD000868F978FA50194016081718182819381F3
:10CDE0000F94A491D8016D937D938D939D938D01A4
:10CDF000B2E1043B1B07F1F62EC020E030E040E03A
:10CE00005FE3C501B4010F9452951B012C0104ECA2
:10CE100012E1A2019101F801608171818281938107
:10CE20000F94A491D8016D937D938D939D938D0163
:10CE3000A501940158966D917D918D919C915B9780
:10CE40000F94A491F801608F718F828F938FF2E11C
:10CE5000003D1F07F1F6F39424E0F212B4CEE9E5A9
:10CE6000FBE08491882341F09091C00095FFFCCFB6
:10CE70008093C6003196F5CF8091C00085FFFCCF2E
:10CE80008AE08093C60087EA92E10E9494E4E7E496
:10CE9000FBE08491882341F09091C00095FFFCCF86
:10CEA0008093C6003196F5CF8091C00085FFFCCFFE
:10CEB0008AE08093C60081E08093A712EBE2FBE05A
:10CEC0008491882341F09091C00095FFFCCF80931E
:10CED000C6003196F5CF8091C00085FFFCCF8AE077
:10CEE0008093C6000E9405DDEAE1FBE0849188237F
:10CEF00041F09091C00095FFFCCF8093C600319621
:10CF0000F5CF8091C00085FFFCCF8AE08093C600FA
:10CF1000E0910C0B34E0E39FF0011124E156F54E53
:10CF200020E030E042E053E46081718182819381AE
:10CF30000F948094181694F48091860B882371F0D6
:10CF400086EA9FE00F94F09D882341F08091A51A16
:10CF50009091A61AC29714F00C9428862A966FAD69
:10CF60002A976093490B2C968EAD9FAD2C9790938A
:10CF7000470B8093460B2E96AEADBFAD2E97B09368
:10CF8000450BA093440B1092570B1092560B82E066
:10CF90000F94BC3B0C9452858091A712882309F40E
:10CFA0009EC0E0E1FBE08491882341F09091C000B5
:10CFB00095FFFCCF8093C6003196F5CF4AE050E054
:10CFC00067E070E08AED99E00E94A630EEE0FBE0B9
:10CFD0008491882341F09091C00095FFFCCF80930D
:10CFE000C6003196F5CF4AE050E067E070E08AED88
:10CFF00099E00E94A630EBEFFAE08491882341F09B
:10D000009091C00095FFFCCF8093C6003196F5CF7C
:10D010004AE050E065E070E08AED99E00E94A630B9
:10D02000E9EEFAE08491882341F09091C00095FFE9
:10D03000FCCF8093C6003196F5CF8091C00085FF6C
:10D04000FCCF8AE08093C60000E010E086EEA82EB8
:10D050008AE0B82E94EE892E9AE0992EE12CF12CDC
:10D060009801215B3C4E6901F5018491E6EEFAE0FE
:10D07000882349F09091C00095FFFCCF8093C600B3
:10D0800031968491F5CFF601EE0DFF1D418152815D
:10D090006381748125E030E08AED99E00E94A4313B
:10D0A000F4E0EF0EF11C2CE1E216F104E9F6F401D4
:10D0B0008491E4EEFAE0882349F09091C00095FF56
:10D0C000FCCF8093C60031968491F5CF0C511109A5
:10D0D0000C33FFEF1F0709F0C1CF0C945285E6EC2B
:10D0E000FAE08491882341F09091C00095FFFCCF35
:10D0F0008093C6003196F5CF8091C00085FFFCCFAC
:10D100008AE08093C6000C94528581E00E949A3692
:10D110000C9452851092D60A0C94528585E40E9494
:10D120005532811102C00F946D09BCE76B2EB6E039
:10D130007B2E14E1812E1BE0912E00E2A02E0BE04D
:10D14000B02E512CD3018D913D010E945532882380
:10D15000D9F1B3E05B120CC00E94C232F5016083CA
:10D160007183828393838CE29BE00E942BFE2CC010
:10D170000E94C232D4012D913D914D915C910F944A
:10D18000A491F5016083718382839383E090280BDF
:10D19000F090290B00912A0B10912B0B2091240B5E
:10D1A0003091250B4091260B5091270B6091200B5D
:10D1B0007091210B8091220B9091230BACE2CA2E2F
:10D1C000ABE0DA2E0E948CFC5394F4E08F0E911C9D
:10D1D00024E0A20EB11C34E05312B4CF0C9452855B
:10D1E00081E08093B21B0F94B0896093970B70938A
:10D1F000980B8093990B90939A0B6091B21B84ECDF
:10D200009FE00F94029E0C9452858DE40E9455324B
:10D21000882311F40C945F83E0916A10F0916B10F5
:10D22000319681918032E9F38930D9F380538A3085
:10D23000B0F0E7EBFAE08491882341F09091C000D0
:10D2400095FFFCCF8093C6003196F5CF8091C0004A
:10D2500085FFFCCF8AE08093C6000C9452850E9423
:10D26000C2320F94EC926B3C710511F40C947C77F4
:10D270000CF021C16F32710509F4A6C60CF06AC02A
:10D280006931710509F451C3B4F56431710509F4CC
:10D29000F1C294F46131710509F4E0C234F46230F2
:10D2A000710508F434C20C944A836231710511F49B
:10D2B0000C9453730C944A836631710509F414C3BA
:10D2C0000CF40CC36731710509F414C3683171059E
:10D2D00011F00C944A838BE99BE00E94ADA20F945D
:10D2E000B0896093CA0A7093CB0A8093CC0A90935A
:10D2F000CD0A0C9452856E31710509F45FC38CF42C
:10D300006B31710509F425C30CF415C36C3171053B
:10D3100009F425C36D31710511F40C9452850C94F8
:10D320004A836A32710509F477C454F46F31710588
:10D3300009F412C46032710509F478C30C944A836D
:10D340006C32710509F4AFC46D32710509F4BAC4C9
:10D350000C944A836D36710509F4AEC70CF064C0B5
:10D360006535710511F40C948C730CF03DC0623579
:10D37000710511F40C944A735CF56135710511F077
:10D380000C944A830F949D130F946D09149A0F9473
:10D39000EF0910920B0B10920A0B68EE73E080E01D
:10D3A00090E00F94DF8910921002E2E8F5E24591D7
:10D3B000549122E73AE060E77AE08CE395E00E943E
:10D3C000CFB60F943D3A80E00F94BC3B0C9452854D
:10D3D0006335710511F40C944E736435710511F4C5
:10D3E0000C9453730C944A836936710509F421C671
:10D3F0005CF46C35710511F40C94A77368367105F3
:10D4000009F4E6C50C944A836A36710511F40C944C
:10D410001A736B36710511F00C944A8310920B0B42
:10D4200010920A0B0C9452856837710511F40C9414
:10D430007275FCF46237710511F40C946A744CF443
:10D440006037710511F00C944A8363E084E998E039
:10D45000DDC56337710511F40C942A7467377105C3
:10D4600011F00C944A83EEEAF5E2859194910C94C4
:10D4700083756E3B710509F4B5C75CF469377105B6
:10D4800011F40C9477756C38710509F4C1C50C94CE
:10D490004A83683C710511F40C94EA76693C710585
:10D4A00011F00C944A830CE716E060E6E62E69E181
:10D4B000F62E0C946177673F81E0780711F40C94A5
:10D4C000A77B0CF07EC06C32A1E07A0711F40C94BB
:10D4D000AC79C4F5603D710511F40C948678A4F420
:10D4E0006D3C710511F40C94BB7714F40C9499778E
:10D4F0006E3C710511F40C9432786F3C710511F497
:10D500000C944F780C944A836D3D710511F40C9482
:10D51000207964F4613D710511F40C94AE786C3D92
:10D52000710511F40C940F790C944A83623E7105D5
:10D5300011F40C944A79603F710511F40C945285F2
:10D540000C944A836036E1E07E07E4F46E35F1E046
:10D550007F0714F00C9452856E3221E0720711F4AB
:10D560000C94517B14F40C94E4796F3281E07807C9
:10D5700011F40C94607B6033714011F40C94AF7A19
:10D580000C944A83643FA1E07A0711F40C94997BD0
:10D590004CF46039714011F00C944A830F946D097A
:10D5A0000C945285653FF1E07F0711F40C94A07B49
:10D5B000663F714011F00C944A830E945B250C94E5
:10D5C00052856E3833E0730711F40C948B800CF0A5
:10D5D00047C06D3B92E0790711F40C94DC81FCF4B8
:10D5E0006835B2E07B0711F40C94BB7C5CF46D3FB2
:10D5F000714011F00C944A830F94CE39EEE7FEE0AF
:10D600000C94B37B693522E0720711F40C944680C8
:10D610006A35724011F40C9454800C944A83643837
:10D6200083E0780711F40C9462806CF46E3BA2E006
:10D630007A0711F40C94EC826335734011F40C9466
:10D64000C57B0C944A836B38E3E07E0711F40C949D
:10D6500065806C38734011F40C9452850C944A83A5
:10D66000633923E0720711F40C94F580D4F4603927
:10D6700083E0780711F40C94C08014F40C948E802D
:10D680006139A3E07A0711F40C94F2806239734097
:10D6900011F00C944A831092121B0F946B260C9479
:10D6A00052856639E3E07E0711F40C94AA816CF48C
:10D6B000643923E0720711F40C94FB8065397340E0
:10D6C00011F40C9478810C944A83603A83E07807D3
:10D6D00009F415C2673E734011F00C944A8310920E
:10D6E000C00A0F94693A8091561090915710A091FA
:10D6F0005810B091591080935A1090935B10A093DA
:10D700005C10B0935D100E94EC3F0C945285009128
:10D710006A1010916B100E5F1F4F80E50E9455320A
:10D72000882379F00E94C2320F94F1924B015C0180
:10D73000FF24F394611571058105910531F4F12CF5
:10D7400004C0F12C812C912C540183E50E945532A8
:10D75000882399F00E94C23220E030E04AE754E486
:10D760000F9452950F94F1924B015C01EE24E394D7
:10D77000611571058105910509F4E12C6AE270E0FB
:10D78000C8010F94449B009711F0DC011C92F80132
:10D79000CF0121912032E1F3F11007C0E11005C063
:10D7A000222319F00F94303A06C0E4ECF4E285919C
:10D7B00094910F943D3A81E00F94103A0F946D09C3
:10D7C0000F94B0896093D20A7093D30A8093D40ADD
:10D7D0009093D50A81149104A104B104A9F00F9487
:10D7E000B0892B013C01480C591C6A1C7B1C0F940E
:10D7F000B0896415750586059705C8F40F94503EE9
:10D80000811115C00C946A860F944E3E882311F442
:10D810000C9452850F94503E81110CC00F94031B41
:10D8200081E00E94F14680E00F94BC3BF3CF80E0A2
:10D830000F94103A80919D0B882341F0E2E5F5E2C8
:10D84000859194910F943D3A0C945285ECEAF4E260
:10D85000859194910F943D3A0C945285E4E8F5E259
:10D86000859194910F943D3A1798169815981498AD
:10D870000C945285E8E3F6E285919491FC012491A1
:10D88000222341F03091C00035FFFCCF2093C60029
:10D890000196F4CF8091C00085FFFCCF8AE0809391
:10D8A000C6008BE99BE00E947EA1EEE0F6E2859146
:10D8B0009491FC012491222341F03091C00035FF66
:10D8C000FCCF2093C6000196F4CF8091C00085FF65
:10D8D000FCCF8AE08093C6000C9452858BE99BE0D4
:10D8E0000E94D4A10C9452858BE99BE00E94A9A2CE
:10D8F0000C94528580916A1090916B106AE270E0EE
:10D9000004960F94449B009711F0DC011C926091E7
:10D910006A1070916B106C5F7F4F21E041E08BE9E2
:10D920009BE00E9455A70C9452858BE99BE00E94D6
:10D93000B4A20C94528580919E0B882311F40C9410
:10D94000528583E50E94553281110C9474860C94A3
:10D9500052858BE99BE00E9459A40C9452858091DA
:10D960006A1090916B106AE270E004960F94449BE9
:10D970008C010097A9F080917410909175106EE45D
:10D9800070E087589F4E0F94449B60E270E00F94C4
:10D99000449B019690936B1080936A10F80110825B
:10D9A00060916A1070916B106C5F7F4F21E040E0D6
:10D9B0008BE99BE00E9455A70C94528580919E0BA9
:10D9C000882311F40C94528560E08BE99BE00E945F
:10D9D000E5A680916A1090916B106AE270E004965F
:10D9E0000F94449B8C010097A9F080917410909142
:10D9F00075106EE470E087589F4E0F94449B60E270
:10DA000070E00F94449B019690936B1080936A1082
:10DA1000D8011C9260916A1070916B106C5F7F4FFF
:10DA20008BE99BE00E9418A30C94528580919D0B7A
:10DA300081110F946D0900916A1010916B100C5FA9
:10DA40001F4F6AE270E0C8010F94449B7C0161E2C1
:10DA500070E0C8010F94449B009719F08C010F5F90
:10DA60001F4FE114F10411F0F701108280E50E94CC
:10DA70005532F82E20916A1030916B10021713075F
:10DA800008F4F12C80919E0B882311F40C9452859C
:10DA900021E02F2541E0B8018BE99BE00E9455A7CA
:10DAA00083E50E9455328823B9F020916A103091A5
:10DAB0006B102017310780F40E947F32AB01BC014C
:10DAC0004093390E50933A0E60933B0E70933C0E88
:10DAD00084E89DE00E9407958BE99BE00E94ADA23F
:10DAE000F1100C9452850F94B0896093CA0A709318
:10DAF000CB0A8093CC0A9093CD0A0C9452858091E6
:10DB00006A1090916B106AE270E005960F94449B46
:10DB10008C010097A9F080917410909175106EE4BB
:10DB200070E087589F4E0F94449B60E270E00F9422
:10DB3000449B019690936B1080936A10D8011C92BD
:10DB400060916A1070916B106B5F7F4F8BE99BE067
:10DB50000E9493AA0C9452850F94B0896093C60AD0
:10DB60007093C70A8093C80A9093C90A0091CA0AA1
:10DB70001091CB0A2091CC0A3091CD0A601B710B19
:10DB8000820B930B28EE33E040E050E00F94549763
:10DB9000CA01B9012CE330E040E050E00F94549703
:10DBA0007F936F933F932F9388EA9AE09F938F938D
:10DBB000CE0101969F938F930F94C49BEEE7FEE0F6
:10DBC00084910FB6F894DEBF0FBECDBFEEE7FEE046
:10DBD000882349F09091C00095FFFCCF8093C60048
:10DBE00031968491F5CFFE0131968191882339F0E9
:10DBF0009091C00095FFFCCF8093C600F6CF809136
:10DC0000C00085FFFCCF8AE08093C600CE0101965C
:10DC10000F94303A0C94528583E50E945532882344
:10DC200011F40C9452850E94C2320F94EC92F62E9D
:10DC3000E72E862F9E2D8C0180E50E945532882389
:10DC400031F00F3F110509F010F40C9485860DE0BA
:10DC500010E0E4E4F6E0819191918017910711F4CE
:10DC60000C94528526E0EC37F207A9F7063011052F
:10DC700039F48F2D9E2D90930B0B80930A0B04C0CB
:10DC800017FF02C00C94528561E0802F0F949B8B8C
:10DC90006F2D802F0F94D48B6F2D7E2D802F0F949E
:10DCA000838A0C9452858FEF0E949A3660E070E070
:10DCB00088EF9FE00F941C9E0E94A2C50E9435C66B
:10DCC0000C9452858AE50E945532382E811112C07B
:10DCD0001092A61A1092A51A1092A81A1092A71ABA
:10DCE0001092AA1A1092A91A1092AC1A1092AB1A9A
:10DCF0000F94793980E00F94293D87EA92E10E94E0
:10DD000079E40E9435C60E94CAE31092110B10926A
:10DD1000120B1092130B81E00E940132EAE6F6E248
:10DD200085919491BE016F5F7F4F0F94653D0E9476
:10DD3000C13E0E944F39882309F441C10E94F43E3C
:10DD400020E030E048E452E460919F1A7091A01AFC
:10DD50008091A11A9091A21A0F948094181684F0C1
:10DD600020E030E048E452E460918D1A70918E1A00
:10DD700080918F1A9091901A0F948094181624F421
:10DD8000332011F40C948C8680E090E0A0EAB0E49B
:10DD90008093280B9093290BA0932A0BB0932B0B05
:10DDA00020E030E040E252E4609151027091520272
:10DDB00080915302909154020F9484924B015C0124
:10DDC0002091240B3091250B4091260B5091270B6D
:10DDD0006091200B7091210B8091220B9091230B6D
:10DDE000ECE0FBE0FF93EF93ECE2CE2EEBE0DE2ED7
:10DDF000E12CF12C00EA10E40E94DEEF0F946D0993
:10DE000086E50E9455320F900F90882369F0E091CB
:10DE10006A10F0916B108181893041F08F7D49F05B
:10DE20000E948A3288AF07C018AE05C031E038AF13
:10DE300002C061E068AF3320B1F00E942F320E942F
:10DE40008AC60E94A6C80E946BDD882309F4B5C06B
:10DE500087EF9FE00F94F09D803F09F0AEC081E016
:10DE60000E949A36AAC08FEF0E949A3660E070E056
:10DE700088EF9FE00F941C9E1982BE016F5F7F4F59
:10DE800088AD0E944BDA3C010E942F32212C312CAC
:10DE900010EA412E10E4512E2092280B3092290BCB
:10DEA00040922A0B50922B0B20E030E040E252E4EB
:10DEB00060915102709152028091530290915402EC
:10DEC0000F9484924B015C012091240B3091250B1F
:10DED0004091260B5091270B6091200B7091210BE4
:10DEE0008091220B9091230BACE0BBE0BF93AF93EA
:10DEF0000CE2C02E0BE0D02E820171010E94DEEFF9
:10DF00000F946D090F900F9077FC48C0198287EA33
:10DF100092E10E9479E40E94FCC581E00E940132F6
:10DF20000E94C13EAE014F5F5F4F68AD81E00E942D
:10DF300082DF3C010E942F322092280B3092290B65
:10DF400040922A0B50922B0B20E030E040E252E44A
:10DF5000609151027091520280915302909154024B
:10DF60000F9484924B015C012091240B3091250B7E
:10DF70004091260B5091270B6091200B7091210B43
:10DF80008091220B9091230BACE0BBE0BF93AF9349
:10DF90000E94DEEF0F946D090F900F906981C3010D
:10DFA0000F94743F77FC09C086EE0E949A36E4E62F
:10DFB000F6E2859194910F943D3F0F946A2581E09C
:10DFC0000F94293D0C9452850F94FC520C94528569
:10DFD00088E690E00E94AB4781110C94528583E55E
:10DFE0000E945532882371F00091C10A0E94C2320A
:10DFF00010E0000F111F0955154E0F94EC92D80137
:10E000006D937C930F949C130C9452850E947246DE
:10E0100083E50E945532882311F40C9452850E94A6
:10E02000C2320F94EC927093A61A6093A51A0C94C6
:10E03000528589E690E00E94AB4781110C9452858D
:10E04000E2EAFAE08491882341F09091C00095FFC4
:10E05000FCCF8093C6003196F5CFE091C10AB4E0C1
:10E06000EB9FF0011124E156F54E40815181628110
:10E07000738121E030E08AED99E00E94A431EFE95C
:10E08000FAE08491882341F09091C00095FFFCCF85
:10E090008093C6003196F5CFE091C10AF0E0EE0F13
:10E0A000FF1FE955F54E60817181882777FD8095C6
:10E0B000982F0F941F93AB01BC0121E030E08AED53
:10E0C00099E00E94A431EBE9FAE08491882341F0C1
:10E0D0009091C00095FFFCCF8093C6003196F5CF9C
:10E0E00040918D1A50918E1A60918F1A7091901AEA
:10E0F00021E030E08AED99E00E94A431E8E9FAE0FD
:10E100008491882341F09091C00095FFFCCF8093CB
:10E11000C6003196F5CF6091A51A7091A61A88278E
:10E1200077FD8095982F0F941F93AB01BC0121E0E0
:10E1300030E08AED99E00E94A431E5E9FAE08491AB
:10E14000882341F09091C00095FFFCCF8093C600DA
:10E150003196F5CF4AE050E060E070E08AED99E05A
:10E160000E94A630E3E9FAE08491882341F090917F
:10E17000C00095FFFCCF8093C6003196F5CF40914B
:10E180009F1A5091A01A6091A11A7091A21A21E0D1
:10E1900030E08AED99E00E94A431E0E9FAE0849150
:10E1A000882341F09091C00095FFFCCF8093C6007A
:10E1B0003196F5CF6091A71A7091A81A882777FD3C
:10E1C0008095982F0F941F93AB01BC0121E030E0A4
:10E1D0008AED99E00E94A431ECE8FAE0849188236A
:10E1E00041F09091C00095FFFCCF8093C60031961E
:10E1F000F5CF8091C10A90E00F941D114AE050E0E4
:10E20000BC018AED99E00E94A630E7E8FAE084912B
:10E21000882341F09091C00095FFFCCF8093C60009
:10E220003196F5CF8FEF9FEF0F941D114AE050E02C
:10E23000BC018AED99E00E94A630E3E8FAE08491FF
:10E24000882341F09091C00095FFFCCF8093C600D9
:10E250003196F5CF4091991A50919A1A60919B1A74
:10E2600070919C1A21E030E08AED99E00E94A4317F
:10E27000EFE7FAE08491882341F09091C00095FF88
:10E28000FCCF8093C6003196F5CF4091931A509100
:10E29000941A6091951A7091961A21E030E08AEDF7
:10E2A00099E00E94A4318091C00085FFFCCF8AE0F4
:10E2B0008093C6000C94CA868DE690E00E94AB471E
:10E2C00081110C945285EAEDF5E2859194910F94B9
:10E2D0003D3A81E090E090934D0B80934C0B809100
:10E2E000B21B882321F081E090E00F94AB3983E5E5
:10E2F0000E945532882391F00091C10A0E94C232D7
:10E3000010E0000F111F0955154E0F94EC92F80103
:10E310007183608381E08093060215C082E50E94CC
:10E320005532882381F00091C10A0E94C23210E068
:10E33000000F111F0955154E0F94EC92D8016D93E3
:10E340007C93109206020F949C130F94B0896B017A
:10E350007C010091C10A10E0F801EE0FFF1FE955A2
:10E36000F54E60817181882777FD8095982F0F94F5
:10E370001F93F801EE0FFF1FEE0FFF1FE156F54E42
:10E3800011E020813181428153810F9480941816CD
:10E390000CF010E01093BF0A1092FB0AC701B601FF
:10E3A0000E943449E8EDF5E2859194910F943D3A4D
:10E3B00082E090E090934D0B80934C0B8091B21BC8
:10E3C000882321F082E090E00F94AB390F94B0895C
:10E3D0006093D20A7093D30A8093D40A9093D50A9B
:10E3E0000C945285E2E5F6E2859194910F943D3AC2
:10E3F00083E090E090934D0B80934C0B8091B21B87
:10E40000882321F081E090E00F94AB3983E50E94EE
:10E410005532882361F00E94C2320F94EC927093BF
:10E42000A61A6093A51A81E0809306020FC082E5C8
:10E430000E945532882351F00E94C2320F94EC9210
:10E440007093A61A6093A51A109206020F94B089D1
:10E450002B013C011092FB0A6091A51A7091A61A3B
:10E46000882777FD8095982F0F941F9311E02091B6
:10E470008D1A30918E1A40918F1A5091901A0F94E4
:10E48000809418160CF010E01093BF0A0CE71AE005
:10E4900098E7E92E9AE0F92E24E7A22E2AE0B22E80
:10E4A0003AE0D32E8091BF0A6091A51A7091A61A06
:10E4B000882309F490C08091FB0A81118CC08827C1
:10E4C00077FD8095982F0F941F9320918D1A30918E
:10E4D0008E1A40918F1A5091901A0F9480941816AA
:10E4E0000CF090C00F94B0896419750986099709DA
:10E4F000693E73408105910508F464C08091B21BA8
:10E5000081115CC0E0910C0B24E0E29FF00111242A
:10E51000E156F54E4081518162817381F801849109
:10E52000ECE7FAE0882349F09091C00095FFFCCF1A
:10E530008093C60031968491F5CF22E030E08AEDD9
:10E5400099E00E94A431F7018491E8E7FAE088237A
:10E5500049F09091C00095FFFCCF8093C6003196A2
:10E560008491F5CF60910C0B70E04AE050E08AEDA9
:10E5700099E00E94A630F5018491E4E7FAE088234F
:10E5800049F09091C00095FFFCCF8093C600319672
:10E590008491F5CF40918D1A50918E1A60918F1A07
:10E5A0007091901A21E030E08AED99E00E94A43148
:10E5B0008091C00085FFFCCFD092C6000F94B08937
:10E5C0002B013C010F94031B80E00E94F14680E088
:10E5D0000F94BC3B67CF882777FD8095982F0F94C9
:10E5E0001F9320918D1A30918E1A40918F1A50915D
:10E5F000901A0F947D9287FF05C0809106028823B0
:10E6000009F470CFE4E5F6E2859194910F943D3AD8
:10E6100084E090E090934D0B80934C0B0F94B08965
:10E620006093D20A7093D30A8093D40A9093D50A48
:10E630000C94528583E50E945532882319F10E947B
:10E64000C23220E030E0A9010F947D9287FD0FC017
:10E650000E94C23220E030E04FE753E40F948094F0
:10E66000181644F00E94C2320F94EC9205C060E08C
:10E6700070E002C06FEF70E070930B0B60930A0BB9
:10E680000C9452858FEF90E090930B0B80930A0BC4
:10E690000C9452851092960B0C94528581E08093D5
:10E6A000960B0C94528583E50E945532882399F08D
:10E6B0000E94C23220E030E04AE754E40F945295C1
:10E6C0000F94F192609308027093090280930A02FA
:10E6D00090930B021DC088E50E94553281110C9465
:10E6E000AB8689E50E94553281110C94AB868AE590
:10E6F0000E94553281110C94AB8685E40E945532FC
:10E7000081110C94AB860F946D09149A0F94EF0944
:10E710001092430B0C94528583E50E945532882356
:10E7200011F40C9452850E94C23220E030E04AE796
:10E7300054E40F9452950F94F1926093CE0A709323
:10E74000CF0A8093D00A9093D10A0C9452852CE77B
:10E7500036E039AF28AF00E719E1B0E8EB2EB9E1B8
:10E76000FB2E80E3282E89E1382ED12CA8ADB9AD3F
:10E770008D91B9AFA8AF0E945532882309F45CC0CF
:10E78000B3E0DB1252C00E94C2322B013C0120E0F8
:10E7900030E040EA51E40F947D9287FF3FC0A3012F
:10E7A0009201F80160817181828193810F9484923A
:10E7B0004B015C019B01AC016091501970915119A2
:10E7C00080915219909153190F945295609350195A
:10E7D000709351198093521990935319A501940184
:10E7E000D7016D917D918D919C910F945295F70178
:10E7F0006083718382839383D1016D917D918D912B
:10E800009C910F941D93A50194010F9452950F9420
:10E81000F192F1016083718382839383D8014D92D9
:10E820005D926D927C92139707C00E94C232F801EC
:10E830006083718382839383D3940C5F1F4FF4E0D2
:10E84000EF0EF11C24E0220E311C34E0D3128ECFE7
:10E850000C94528586E50E9455328823B9F00F94B6
:10E86000FD85FC012491222341F03091C00035FF49
:10E87000FCCF2093C6000196F4CF8091C00085FFA5
:10E88000FCCF8AE08093C6000C94528585E50E94F7
:10E890005532882369F080916A1090916B1001962F
:10E8A00090936B1080936A100F946E880C9452852D
:10E8B000E0EBF5E285919491FC012491222311F47F
:10E8C0000C9452853091C00035FFFCCF2093C600D8
:10E8D0000196F2CFEDE6FAE08491882341F0909121
:10E8E000C00095FFFCCF8093C6003196F5CF4091D4
:10E8F000200B5091210B6091220B7091230B22E091
:10E9000030E08AED99E00E94A431E9E6FAE08491D2
:10E91000882341F09091C00095FFFCCF8093C60002
:10E920003196F5CF4091240B5091250B6091260B29
:10E930007091270B22E030E08AED99E00E94A4312B
:10E94000E5E6FAE08491882341F09091C00095FFBC
:10E95000FCCF8093C6003196F5CF4091280B5091A3
:10E96000290B60912A0B70912B0B22E030E08AED8D
:10E9700099E00E94A431E1E6FAE08491882341F015
:10E980009091C00095FFFCCF8093C6003196F5CFE3
:10E9900040912C0B50912D0B60912E0B70912F0BF1
:10E9A00022E030E08AED99E00E94A431E0E2F6E254
:10E9B00085919491FC012491222341F03091C00073
:10E9C00035FFFCCF2093C6000196F4CF80E00F9472
:10E9D000CE090F941F9320917019309171194091B5
:10E9E0007219509173190F948492AB01BC0122E00B
:10E9F00030E08AED99E00E94A431EDE5FAE08491DF
:10EA0000882341F09091C00095FFFCCF8093C60011
:10EA10003196F5CF81E00F94CE090F941F9320918A
:10EA200074193091751940917619509177190F9496
:10EA30008492AB01BC0122E030E08AED99E00E94B3
:10EA4000A431E9E5FAE08491882341F09091C00077
:10EA500095FFFCCF8093C6003196F5CF82E00F94EE
:10EA6000CE090F941F932091781930917919409114
:10EA70007A1950917B190F948492AB01BC0122E06A
:10EA800030E08AED99E00E94A431E5E5FAE0849156
:10EA9000882341F09091C00095FFFCCF8093C60081
:10EAA0003196F5CF83E00F94CE090F941F932091F8
:10EAB0007C1930917D1940917E1950917F190F94E6
:10EAC0008492AB01BC0122E030E08AED99E00E9423
:10EAD000A4318091C00085FFFCCF8AE08093C600FE
:10EAE0000C94528580E00E94FAFF0C94528581E0DC
:10EAF0000E94FAFF0C9452853091C00035FFFCCF84
:10EB00002093C6000196FC0124912111F5CF80913C
:10EB1000C00085FFFCCF8AE08093C600EAEBF4E2F8
:10EB200085919491FC012491222341F03091C00001
:10EB300035FFFCCF2093C6000196F4CF1E9B10C07A
:10EB4000E2E1F6E285919491FC0124912223C1F047
:10EB50003091C00035FFFCCF2093C6000196F4CF62
:10EB6000E0E1F6E285919491FC012491222341F0A9
:10EB70003091C00035FFFCCF2093C6000196F4CF42
:10EB80008091C00085FFFCCF8AE08093C600ECEB4B
:10EB9000F4E285919491FC012491222341F030917B
:10EBA000C00035FFFCCF2093C6000196F4CF8091C2
:10EBB000060182FF10C0E2E1F6E285919491FC012A
:10EBC00024912223C1F03091C00035FFFCCF209367
:10EBD000C6000196F4CFE0E1F6E285919491FC0144
:10EBE0002491222341F03091C00035FFFCCF2093C7
:10EBF000C6000196F4CF8091C00085FFFCCF8AE06B
:10EC00008093C600E4EBF4E285919491FC01249199
:10EC1000222341F03091C00035FFFCCF2093C60085
:10EC20000196F4CF1D9B10C0E2E1F6E2859194912C
:10EC3000FC0124912223C1F03091C00035FFFCCFAC
:10EC40002093C6000196F4CFE0E1F6E2859194911D
:10EC5000FC012491222341F03091C00035FFFCCF0C
:10EC60002093C6000196F4CF8091C00085FFFCCFB1
:10EC70008AE08093C600E6EBF4E285919491FC0172
:10EC80002491222341F03091C00035FFFCCF209326
:10EC9000C6000196F4CF8091060187FF10C0E2E123
:10ECA000F6E285919491FC0124912223C1F03091E8
:10ECB000C00035FFFCCF2093C6000196F4CFE0E101
:10ECC000F6E285919491FC012491222341F0309148
:10ECD000C00035FFFCCF2093C6000196F4CF809191
:10ECE000C00085FFFCCF8AE08093C600EEEAF4E224
:10ECF00085919491FC012491222341F03091C00030
:10ED000035FFFCCF2093C6000196F4CF1C9B10C0AA
:10ED1000E2E1F6E285919491FC0124912223C1F075
:10ED20003091C00035FFFCCF2093C6000196F4CF90
:10ED3000E0E1F6E285919491FC012491222341F0D7
:10ED40003091C00035FFFCCF2093C6000196F4CF70
:10ED50008091C00085FFFCCF8AE08093C600E0EB85
:10ED6000F4E285919491FC012491222341F03091A9
:10ED7000C00035FFFCCF2093C6000196F4CF019967
:10ED800010C0E2E1F6E285919491FC0124912223E6
:10ED9000C1F03091C00035FFFCCF2093C600019632
:10EDA000F4CFE0E1F6E285919491FC0124912223D5
:10EDB00041F03091C00035FFFCCF2093C600019692
:10EDC000F4CF8091C00085FFFCCF8AE08093C6001D
:10EDD0000C94528580910C0B8093C10A84E50E94AB
:10EDE0005532882329F10E94C2320F94F192609328
:10EDF000C10A6623E9F0EEE7FEE08491882341F042
:10EE00009091C00095FFFCCF8093C6003196F5CF5E
:10EE1000ECEAF5E2A591B4918D91882311F40C945C
:10EE200052859091C00095FFFCCF8093C600F4CF2F
:10EE300084E40E945532882311F40C9452850E9478
:10EE4000C23220E030E0A9010F947D92811103C00D
:10EE50001092300B32C00091C10A10E00E94C23201
:10EE6000F801EE0FFF1FEE0FFF1FE35CFD4F608305
:10EE7000718382839383E0903D02F0903E02009183
:10EE80003F021091400220E030E0A901B701C80123
:10EE90000F947D92811104C0E12CF12C00E410E468
:10EEA000C701D80180933D0290933E02A0933F0298
:10EEB000B093400281E08093300B0E9400490C9493
:10EEC0005285D8018D918D010E945532882349F0D9
:10EED0000E94C2320F94F192F701608371838283A2
:10EEE0009383F4E0EF0EF11C26E00038120749F797
:10EEF0000E9451FE0C9452850CE716E050E8E52E76
:10EF000059E1F52ED8018D918D010E94553288234B
:10EF100039F00E94C232F701608371838283938348
:10EF2000F4E0EF0EF11C26E00038120759F70C94BC
:10EF3000528583E50E945532882351F00E94C232E7
:10EF4000609358197093591980935A1990935B19CB
:10EF500084E50E945532882311F40C9452850E9456
:10EF6000C232609354197093551980935619909337
:10EF700057190C94528583E50E945532882351F02D
:10EF80000E94C23260935C1970935D1980935E1980
:10EF900090935F1984E50E945532882351F00E94B6
:10EFA000C232609340197093411980934219909333
:10EFB000431982E40E945532882361F00E94C232D4
:10EFC0000F94F19260939019709391198093921914
:10EFD0009093931988E50E945532882391F00E94FE
:10EFE000C232609348197093491980934A199093DB
:10EFF0004B19609344197093451980934619909367
:10F00000471989E50E945532882351F00E94C23287
:10F01000609348197093491980934A1990934B193A
:10F020008AE50E945532882351F00E94C2326093D3
:10F030004C1970934D1980934E1990934F1985E494
:10F040000E945532882311F40C9452850E94C232DA
:10F0500060935019709351198093521990935319DA
:10F060000C9452850CE716E044E1E42E4BE0F42EBC
:10F07000D8018D918D010E945532882339F00E946C
:10F08000C232F7016083718382839383F4E0EF0ED1
:10F09000F11C26E00F37120759F70C94528583E5CF
:10F0A0000E945532882351F00E94C23260931D02A3
:10F0B00070931E0280931F029093200286E40E94A8
:10F0C0005532882381F00E94C23220E030E040E7D0
:10F0D00052E40F9484926093150270931602809309
:10F0E0001702909318028AE50E945532882311F482
:10F0F0000C9452850E94C2326093040B7093050BEE
:10F100008093060B9093070B0C94528583E50E9425
:10F110005532882351F00E94C2326093000B7093E5
:10F12000010B8093020B9093030B86E40E945532EF
:10F13000882311F40C9452850E94C23220E030E002
:10F1400040E752E40F94849260931102709312028C
:10F1500080931302909314020C94528583E50E94CD
:10F160005532882311F40C9452850E94C2320F94B8
:10F17000EC926115710551F06130710569F481E01F
:10F180008093090B1092080B0C9452851092090B76
:10F190001092080B0C945285EEE7FEE084918823D0
:10F1A00041F09091C00095FFFCCF8093C60031964E
:10F1B000F5CFECECF4E285919491FC0124912223AB
:10F1C00041F03091C00035FFFCCF2093C60001967E
:10F1D000F4CFE0917410F0917510E758FF4E8191D3
:10F1E000882339F09091C00095FFFCCF8093C60032
:10F1F000F6CFE0E5FAE08491882341F09091C000D9
:10F2000095FFFCCF8093C6003196F5CF8091C0006A
:10F2100085FFFCCF8AE08093C6000C94528583E57D
:10F220000E945532882311F40C9452850E94C232F8
:10F230000F94EC9270934802609347020C945285AD
:10F2400083E50E945532882311F40C9452850E9464
:10F25000C2320F94EC926B017C0184E50E9455321E
:10F26000882391F08DED90E00E94AB4781110C94C2
:10F270005285E091C10AF0E0EE0FFF1FED5BFD4FFC
:10F28000D182C0820C945285D0924602C09245022F
:10F290000C94528580E50E945532882311F40C9419
:10F2A00052850E94C2320F94EC92D62E062F172F51
:10F2B00083E50E945532882331F00E94C2320F94B8
:10F2C000EC927B0103C0EE24EA94FE2CC701019668
:10F2D000039710F00C945285E4E4F6E0819191914B
:10F2E0008017910711F40C94528526E0EC37F20751
:10F2F000A9F717FF02C00C9452850F946D09CD2C0D
:10F3000060E08D2D0F949B8B3FEFE316F30631F0F9
:10F31000EA94EF2871F000E010E00DC08D2D0F94FD
:10F32000098C31E020E0892B09F030E0032F122F07
:10F3300002C001E010E08C2D0F94098C801791071A
:10F3400011F40C9452850F94031B80E00E94F14647
:10F3500080E00F94BC3BEFCF83E50E9455328823B9
:10F3600031F00E94C2320F94EC928B0102C00EE683
:10F3700010E080E50E945532882331F00E94C232AD
:10F380000F94EC92CB0102C088EE93E06C01EE2466
:10F39000D7FCE094FE2C1016110684F420E030E037
:10F3A000A901B80184E50F94FE8DC701B6010F9441
:10F3B000DF8984E50F9422910C945285C701B60130
:10F3C0000F94DF890C94528580E50E945532882382
:10F3D00051F00E94C23260939E0270939F0280930C
:10F3E000A0029093A10289E40E945532882361F023
:10F3F0000E94C2320F94AA2160939A0270939B02DA
:10F4000080939C0290939D0284E40E94553288234D
:10F4100061F00E94C2320F94B621609396027093FD
:10F420009702809398029093990283E40E94553248
:10F43000882351F00E94C23260939202709393022B
:10F4400080939402909395020F94F010E0E8F5E217
:10F4500085919491FC012491222341F03091C000C8
:10F4600035FFFCCF2093C6000196F4CFE9E4F5E028
:10F470008191882339F09091C00095FFFCCF809353
:10F48000C600F6CF40919E0250919F026091A0026B
:10F490007091A10222E030E08AED99E00E94A4314F
:10F4A000EDE4F5E08191882339F09091C00095FF5B
:10F4B000FCCF8093C600F6CF60919A0270919B02B8
:10F4C00080919C0290919D020F94B021AB01BC01F0
:10F4D00022E030E08AED99E00E94A431E1E5F5E018
:10F4E0008191882339F09091C00095FFFCCF8093E3
:10F4F000C600F6CF609196027091970280919802B3
:10F50000909199020F94BC21AB01BC0122E030E044
:10F510008AED99E00E94A431E5E5F5E08191882328
:10F5200039F09091C00095FFFCCF8093C600F6CFD4
:10F5300040919202509193026091940270919502D1
:10F5400022E030E08AED99E00E94A4318091C00071
:10F5500085FFFCCF8AE08093C6000C94528580E53D
:10F560000E945532882351F00E94C23260938E026D
:10F5700070938F02809390029093910289E40E948D
:10F580005532882361F00E94C2320F94AA21609301
:10F590008A0270938B0280938C0290938D0284E494
:10F5A0000E945532882361F00E94C2320F94B62126
:10F5B00060938602709387028093880290938902F9
:10F5C0000F94F010E0E8F5E285919491FC0124910C
:10F5D000222341F03091C00035FFFCCF2093C600BC
:10F5E0000196F4CFE9E4F5E08191882339F0909118
:10F5F000C00095FFFCCF8093C600F6CF40918E02ED
:10F6000050918F02609190027091910222E030E05F
:10F610008AED99E00E94A431EDE4F5E08191882320
:10F6200039F09091C00095FFFCCF8093C600F6CFD3
:10F6300060918A0270918B0280918C0290918D0270
:10F640000F94B021AB01BC0122E030E08AED99E0DB
:10F650000E94A431E1E5F5E08191882339F0909191
:10F66000C00095FFFCCF8093C600F6CF6091860264
:10F670007091870280918802909189020F94BC2139
:10F68000AB01BC0122E030E08AED99E00E94A43198
:10F690008091C00085FFFCCF8AE08093C6000C9467
:10F6A000528583E50E945532882319F00E94C232A8
:10F6B00003C060E070E0CB010E9448FE0C945285CC
:10F6C00085E40E945532882341F00E94C2320F9493
:10F6D000EC928B0177FF03C009C000E010E0812CA1
:10F6E000912C96E1A92E93E4B92E06C0812C912C81
:10F6F0008CE8A82E82E4B82E83E50E945532882338
:10F7000021F00E94C2324B015C0183E40E94553219
:10F71000882331F00E94C2320F94EC929B0102C008
:10F7200025E030E0A801C501B4010F94B0130C949A
:10F73000528560E084E190E00E94581F0C9452854D
:10F7400060E084E190E00E94E7260C94528580E01E
:10F750000E9478200C9452859091C00095FFFCCFB8
:10F760008093C600319684918111F6CFE0E4FAE0EF
:10F770008491882311F40C9452859091C00095FFD8
:10F78000FCCF8093C6003196F3CF8AE50E945532B4
:10F79000882309F4B0C00E94C2324B015C0120E012
:10F7A00030E040E751EC0F94809487FD4EC020E09C
:10F7B00030E040EA50ECC501B4010F947D92181678
:10F7C0000CF443C0B7FAB094B7F8B09480920D0B24
:10F7D00090920E0BA0920F0BB092100BEEE7FEE092
:10F7E0008491882341F09091C00095FFFCCF8093D5
:10F7F000C6003196F5CFE0E8F5E245915491E2EB91
:10F80000F4E2859194912FE33AE065E579E00E9476
:10F81000CFB6FC012491222341F03091C00035FF86
:10F82000FCCF2093C6000196F4CF8091C00085FFE5
:10F83000FCCF8AE08093C6008091C00085FFFCCF9A
:10F840008AE08093C6000C945285EEE7FEE0849136
:10F85000882341F09091C00095FFFCCF8093C600B3
:10F860003196F5CFE2EBF4E285919491FC0124917D
:10F87000222341F03091C00035FFFCCF2093C60019
:10F880000196F4CFEEEAF4E285919491FC01249183
:10F89000222341F03091C00035FFFCCF2093C600F9
:10F8A0000196F4CF4AE050E061EF7FEF8AED99E0F6
:10F8B0000E94A630E0EBF4E285919491FC01249142
:10F8C000222341F03091C00035FFFCCF2093C600C9
:10F8D0000196F4CF4AE050E06BEF7FEF8AED99E0BC
:10F8E0000E94A6308091C00085FFFCCF8AE0809303
:10F8F000C6000C945285EEE7FEE08491882341F027
:10F900009091C00095FFFCCF8093C6003196F5CF53
:10F91000E2EBF4E2859194916BE37AE00E94AEB65B
:10F92000FC012491222341F03091C00035FFFCCF2F
:10F930002093C6000196F4CF8091C00085FFFCCFD4
:10F940008AE08093C60040910D0B50910E0B6091A0
:10F950000F0B7091100B705822E030E08AED99E0A7
:10F960000E94A4318091C00085FFFCCF8AE0809383
:10F97000C6000C94528569E575E08AED99E00E9415
:10F9800099300F946D098091B21B882321F086E194
:10F9900090E00F94AB398091470290914802909388
:10F9A000420280934102C090200BD090210BE09046
:10F9B000220BF090230BCF8ED8A2E9A2FAA20091DD
:10F9C000240B1091250B2091260B3091270B0BA3B4
:10F9D0001CA32DA33EA34091280B5091290B6091AD
:10F9E0002A0B70912B0B4FA358A769A77AA7809178
:10F9F0002C0B90912D0BA0912E0BB0912F0B8BA760
:10FA00009CA7ADA7BEA7C982DA82EB82FC820D83D8
:10FA10001E832F83388749875A876B877C878D871A
:10FA20009E87AF87B88B85E40E945532882359F0B2
:10FA30000E94C2329B01AC016BA57CA58DA59EA541
:10FA40000F94A4910AC020E030E040E050E46BA5A0
:10FA50007CA58DA59EA50F94A3916BA77CA78DA7D0
:10FA60009EA7EFA0F8A409A51AA52BA13CA14DA122
:10FA70005EA16F8D78A189A19AA1ECE0FBE0FF93D4
:10FA8000EF93812C912CB8EEAB2EB2E4BB2EDE01AD
:10FA90009B966D010E94DEEF8AE50E9455320F9021
:10FAA0000F90882349F00E94C2329B01AC016FA1E4
:10FAB00078A589A59AA51EC020E030E040E050E47A
:10FAC0006FA178A589A59AA50F94A4914B015C011B
:10FAD0006FA378A789A79AA720E030E040E251E41D
:10FAE0000F947D9287FF0CC020E030E040E251E4AB
:10FAF000C501B4010F94A4916FA378A789A79AA711
:10FB0000EFA0F8A409A51AA52BA13CA14DA15EA1C7
:10FB10006F8D78A189A19AA1ECE0FBE0FF93EF93B0
:10FB2000812C912CA0E7AA2EA1E4BA2EFE01BB964F
:10FB30006F010E94DEEF88E50E9455320F900F9012
:10FB4000882379F00E94C2329B01AC016F8D78A1AD
:10FB500089A19AA10F94A4916F8F78A389A39AA3E6
:10FB600008C080E090E0A3E5B3E48F8F98A3A9A339
:10FB7000BAA389E50E945532882339F00E94C23227
:10FB80006BA37CA38DA39EA304C01BA21CA21DA2D9
:10FB90001EA2EFA0F8A409A51AA52BA13CA14DA176
:10FBA0005EA16F8D78A189A19AA1ECE0FBE0FF93A3
:10FBB000EF93812C912CF8E4AF2EF2E4BF2EDE01FE
:10FBC0009B966D010E94DEEF0F946D0981E080939A
:10FBD000490BEAECF4E2859194910F943D3A8CE460
:10FBE0000E9455320F900F90882359F00E94C23224
:10FBF0009B01AC016BA57CA58DA59EA50F94A4913E
:10FC00000AC020E030E040EA52E46BA57CA58DA557
:10FC10009EA50F94A3916BA77CA78DA79EA7EFA08D
:10FC2000F8A409A51AA52BA13CA14DA15EA16F8D39
:10FC300078A189A19AA1ECE0FBE0FF93EF93812CDE
:10FC4000912CE8E6AE2EE2E4BE2EFE01BB966F01DB
:10FC50000E94DEEF0F946D09149A64E670E080E074
:10FC600090E00F94DF890F9460570F94B0896093F0
:10FC7000580B7093590B80935A0B90935B0B0F901A
:10FC80000F9000E010E0F12C0F94503E81112AC03B
:10FC9000F3940F94031B81E00E94F146F110F4CF1E
:10FCA000043FF1E01F0711F400E010E08091010132
:10FCB0008460809301010115110531F49FB7F89418
:10FCC00080910201846008C00431110541F49FB79E
:10FCD000F894809102018B7F809302019FBF0F5F98
:10FCE0001F4FD2CF9FB7F894809102018B7F8093F2
:10FCF00002019FBF20E030E04CE852E46BA57CA5F8
:10FD00008DA59EA50F94A4916BA77CA78DA79EA7F8
:10FD1000EFA0F8A409A51AA52BA13CA14DA15EA1B5
:10FD20006F8D78A189A19AA1FCE06F2EFBE07F2E58
:10FD30007F926F92812C912CA0EAAA2EA1E4BA2E78
:10FD4000DE019B966D010E94DEEF20E030E048E48A
:10FD500052E46BA57CA58DA59EA50F94A4916BA7DD
:10FD60007CA78DA79EA7EFA0F8A409A51AA52BA193
:10FD70003CA14DA15EA16F8D78A189A19AA17F922E
:10FD80006F92812C912CA12CB0E4BB2E0E94DEEF4F
:10FD900010927F0B10927E0B0F94C8570F900F900C
:10FDA0000F900F9080917E0B90917F0B019709F43B
:10FDB0008CC010927F0B10927E0B0F94085880918C
:10FDC0007E0B90917F0B8230910571F1039709F0C2
:10FDD00076C020E030E048E452E46BA57CA58DA518
:10FDE0009EA50F94A4916BA77CA78DA79EA7EFA0BB
:10FDF000F8A409A51AA52BA13CA14DA15EA16F8D68
:10FE000078A189A19AA17F926F92812C912CA12C2B
:10FE1000A0E4BA2EDE019B966D010E94DEEF0F94E6
:10FE200088570F900F90BECF20E030E04CE852E4AE
:10FE30006BA57CA58DA59EA50F94A4916BA77CA70F
:10FE40008DA79EA7EFA0F8A409A51AA52BA13CA1F8
:10FE50004DA15EA16F8D78A189A19AA17F926F9229
:10FE6000812C912CB0EAAB2EB1E4BB2EDE019B9627
:10FE70006D010E94DEEF20E030E048E452E46BA523
:10FE80007CA58DA59EA50F94A4916BA77CA78DA79B
:10FE90009EA7EFA0F8A409A51AA52BA13CA14DA1EE
:10FEA0005EA16F8D78A189A19AA17F926F92812C1A
:10FEB000912CA12CE0E4BE2E0E94DEEF6DCF0F94BA
:10FEC0007A5781E00F94293D6DCF20E030E040EA81
:10FED00050E46BA57CA58DA59EA50F94A4916BA75E
:10FEE0007CA78DA79EA7EFA0F8A409A51AA52BA112
:10FEF0003CA14DA15EA16F8D78A189A19AA1ECE0F2
:10FF00006E2EEBE07E2E7F926F92812C912CA12C95
:10FF1000F0E4BF2EFE01BB966F010E94DEEFA5014B
:10FF200094016BA57CA58DA59EA50F94A3916BA7AD
:10FF30007CA78DA79EA7EFA0F8A409A51AA52BA1C1
:10FF40003CA14DA15EA16F8D78A189A19AA17F925C
:10FF50006F92812C912CA8EEAA2EA2E4BA2E0E94B8
:10FF6000DEEFEFA0F8A409A51AA52D813E814F81EF
:10FF7000588569817A818B819C817F926F92812CD7
:10FF8000912CB8E4AB2EB2E4BB2E0E94DEEFE984E4
:10FF9000FA840B851C852D813E814F8158856981AE
:10FFA0007A818B819C817F926F92812C912CE0E7EA
:10FFB000AE2EE1E4BE2E0E94DEEF20E030E040E015
:10FFC00050E46BA57CA58DA59EA50F94A4916BA76D
:10FFD0007CA78DA79EA7E984FA840B851C852D81BB
:10FFE0003E814F81588569817A818B819C817F9286
:10FFF0006F92812C912CF8EEAF2EF2E4BF2E0E946E
:020000021000EC
:10000000DEEFCE010D960E942BFE80914102909171
:10001000420280934702909348029F938F9382E31A
:100020009AE09F938F938E01015D1F4F1F930F9353
:100030000F94C49B60E0C8010E9493ADECEAF4E227
:10004000859194910F943D3A1092490B1092470B71
:100050001092460B0FB6F894DEBF0FBECDBF809155
:100060006612882309F41EC50E94BDAC0F946D0969
:100070000E942DAF811105C00E949A570E94BDAC0D
:10008000F7CF0E94D0B40E94CBB40CC58091B61BB0
:100090009091B71B892B09F005C585E090E09093FE
:1000A000B71B8093B61BFEC48091B61B9091B71B03
:1000B000892B09F0F7C486E090E09093B71B8093FA
:1000C000B61BF0C40E940038EDC488E50E9455328A
:1000D000882339F00E94C2320F94EC9280E00F9492
:1000E000E50A8AE50E945532882339F00E94C2321F
:1000F0000F94EC9281E00F94E50A85E40E9455325A
:10010000882309F4CFC40E94C2320F94EC9282E09B
:100110000F94E50AC7C40F946B26C4C488E50E94F7
:100120005532882339F00E94C2320F94F19280E058
:100130000F94E92589E50E945532882339F00E9401
:10014000C2320F94F19281E00F94E9258AE50E9472
:100150005532882339F00E94C2320F94F19282E026
:100160000F94E92585E40E945532882309F49AC446
:100170000E94C2320F94F19283E00F94E92592C459
:1001800088E50E945532882339F00E94C2320F94CC
:10019000F19280E00F942A2689E50E945532882347
:1001A00039F00E94C2320F94F19281E00F942A2616
:1001B0008AE50E945532882339F00E94C2320F949A
:1001C000F19282E00F942A2685E40E94553288231A
:1001D00009F468C40E94C2320F94F19283E00F9434
:1001E0002A2660C40F9476225DC481E08093121B9E
:1001F0000F946B2657C488E50E945532882331F04E
:100200000E94C2320F94F1926093A70289E50E9486
:100210005532882331F00E94C2320F94F1926093DC
:10022000A8028AE50E945532882331F00E94C2322A
:100230000F94F1926093A90285E40E9455328823BD
:1002400031F00E94C2320F94F1926093AA02E6E666
:10025000F5E08191882339F09091C00095FFFCCFA3
:100260008093C600F6CF4AE050E06091A7028AED85
:1002700099E00E94F130E9E7F5E08191882339F0B7
:100280009091C00095FFFCCF8093C600F6CF4AE066
:1002900050E06091A8028AED99E00E94F130ECE80C
:1002A000F5E08191882339F09091C00095FFFCCF53
:1002B0008093C600F6CF4AE050E06091A9028AED33
:1002C00099E00E94F130EFE9F5E08191882339F05F
:1002D0009091C00095FFFCCF8093C600F6CF4AE016
:1002E00050E06091AA028AED99E00E94F130DAC3F1
:1002F00088E50E945532882339F00E94C2320F945B
:10030000F19280E00F94EA2389E50E945532882318
:1003100039F00E94C2320F94F19281E00F94EA23E7
:100320008AE50E945532882339F00E94C2320F9428
:10033000F19282E00F94EA2385E40E9455328823EB
:1003400009F4B0C30E94C2320F94F19283E00F947B
:10035000EA23A8C388E50E945532882339F00E9419
:10036000C2320F94F19280E00F94412489E50E94FB
:100370005532882339F00E94C2320F94F19281E005
:100380000F9441248AE50E945532882339F00E9457
:10039000C2320F94F19282E00F94412485E40E94CE
:1003A0005532882309F47EC30E94C2320F94F19221
:1003B00083E00F94412476C3159881E08093490B24
:1003C00082E090E09093470B8093460BECEBF5E2D4
:1003D000859194910F943D3A20E030E04CE852E44E
:1003E00060912C0B70912D0B80912E0B90912F0B07
:1003F0000F94A49160932C0B70932D0B80932E0B74
:1004000090932F0BE090280BF090290B00912A0B72
:1004100010912B0B2091240B3091250B4091260B32
:100420005091270B6091200B7091210B8091220B32
:100430009091230BECE06E2EEBE07E2E7F926F927C
:10044000812C912CF0ECAF2EF0E4BF2EACE2CA2E42
:10045000ABE0DA2E0E94DEEF20E030E048EC51E421
:1004600060912C0B70912D0B80912E0B90912F0B86
:100470000F94A49160932C0B70932D0B80932E0BF3
:1004800090932F0BE090280BF090290B00912A0BF2
:1004900010912B0B2091240B3091250B4091260BB2
:1004A0005091270B6091200B7091210B8091220BB2
:1004B0009091230B7F926F92812C912CB0E8AB2E00
:1004C000BFE3BB2E0E94DEEF0F946D090F900F90DB
:1004D0000F900F908091B21B8823A9F081E00F94B8
:1004E000293D82E00F94BC3BECEAF4E285919491C3
:1004F0000F943D3A1092480B1092490B1092470B03
:100500001092460BCFC28091480B882339F300EF3D
:10051000602E05E2702EF3018591949141E060E038
:100520000F94B36191E0811101C090E01CE0412E75
:100530001BE0512E9111D2CF81E00F94293D82E032
:100540000F94BC3B20E030E048EC51E460912C0B70
:1005500070912D0B80912E0B90912F0B0F94A491E5
:1005600060932C0B70932D0B80932E0B90932F0B7D
:10057000E090280BF090290B00912A0B10912B0B87
:100580002091240B3091250B4091260B5091270B85
:100590006091200B7091210B8091220B9091230B85
:1005A0005F924F92812C912CA0E8AA2EAFE3BA2E35
:1005B000BCE2CB2EBBE0DB2E0E94DEEF0F946D0978
:1005C000F3018591949141E060E00F94B3610F9045
:1005D0000F90811183CFB0CF81E08093490B82E0EF
:1005E00090E09093470B8093460BEAECF4E2859100
:1005F00094910F943D3A20E030E040EA52E460915B
:100600002C0B70912D0B80912E0B90912F0B0F9432
:10061000A39160932C0B70932D0B80932E0B9093D2
:100620002F0BE090280BF090290B00912A0B1091D2
:100630002B0B2091240B3091250B4091260B5091D0
:10064000270B6091200B7091210B8091220B9091D0
:10065000230BECE0FBE0FF93EF93812C912CE8EE71
:10066000AE2EE2E4BE2EFCE2CF2EFBE0DF2E0E9497
:10067000DEEF0F946D09ECEAF4E2859194910F940A
:100680003D3A1092490B1092470B1092460B0F9077
:100690000F9008C2E2E2FAE08491882341F0909141
:1006A000C00095FFFCCF8093C6003196F5CF8091B6
:1006B000C00085FFFCCF8AE08093C600F3C184E5CB
:1006C0000E945532882309F4D1C0E0916A10F0915C
:1006D0006B10319681918032E9F38930D9F390ED36
:1006E000980F9A30E0F08F33A9F0E2E1FAE08491BC
:1006F000882341F09091C00095FFFCCF8093C60005
:100700003196F5CF8091C00085FFFCCF8AE08093C1
:10071000C600C8C10F94F3848093C10A06C00E942A
:10072000C2320F94F1926093C10A2091C10A81E014
:1007300090E0022E01C0880F0A94EAF79091430BD3
:10074000982B9093430B222309F442C0EEE7FEE07E
:100750008491882341F09091C00095FFFCCF809355
:10076000C6003196F5CFE0E1FAE08491882341F0AC
:100770009091C00095FFFCCF8093C6003196F5CFD5
:100780006091C10A70E04AE050E08AED99E00E9471
:10079000A6308091C00085FFFCCF8AE08093C60020
:1007A000E4ECF5E285919491FC012491222341F03F
:1007B0003091C00035FFFCCF2093C6000196F4CFE6
:1007C0008091C00085FFFCCF8AE08093C6006AC19B
:1007D00086E40E9455328823D9F00E94C2324B0130
:1007E0005C016093DB0A7093DC0A8093DD0A9093CE
:1007F000DE0A20E030E0A9010F948094181644F43A
:1008000080920C0290920D02A0920E02B0920F0202
:10081000EEE7FEE08491882341F09091C00095FFBF
:10082000FCCF8093C6003196F5CFE0E7F6E28591E4
:100830009491FC012491222341F03091C00035FFB6
:10084000FCCF2093C6000196F4CF60910C0B70E0B2
:100850004AE050E08AED99E00E94A6308091C00005
:1008600085FFFCCF8AE08093C6001CC184E40E940F
:100870005532882309F4D5C00E94C2320F94EC92FD
:1008800067307105B9F1B4F463307105E1F154F4E6
:100890006130710591F1A4F5672B09F003C10E9445
:1008A000972800C16530710589F10CF08CC00E9459
:1008B000592AF8C0673EF3E07F07F1F16CF46A3023
:1008C000710539F16C30710541F16830710509F03D
:1008D000E9C0E2EBF5E097C0693E33E0730709F445
:1008E00067C00CF45FC0653A734209F0DBC00E9438
:1008F000E02AD8C0EFEBF5E071C00E94B728D2C063
:100900000E94CE28CFC00E948F29CCC00E94DB2A33
:10091000C9C086EE0E949A36C5C060E086E69FE0B8
:100920000F94029E60E085E69FE00F94029E60E0D7
:1009300084E69FE00F94029E6DEC75E08AED99E0ED
:100940000E9499300F946D0981E00F94293D0F9416
:10095000263982E00F94BC3B86E69FE00F94F09D21
:1009600061E0680F86E69FE00F94029E81E00F949D
:10097000293D82E00F94BC3BECEAF4E2859194912E
:100980000F943D3A61E08AE09AE00E9493AD61E005
:1009900084E09AE00E9493AD61E08EEF99E00E94BE
:1009A00093AD80C00E94785681E08093A2027AC005
:1009B00010929D0B60E08BE99BE00E94E5A681E030
:1009C0008093A2026FC081E090E00E949F3A6AC0CB
:1009D0009091C00095FFFCCF8093C600819181115A
:1009E000F7CF68EC88EC0E947DEA4AE050E0BC0159
:1009F0008AED99E00E94AD3055C09091C00095FFFE
:100A0000FCCF8093C60081918111F7CF85E70F94C9
:100A1000450D4AE050E0BC018AED99E00E94AD30FE
:100A200041C0EEE7FEE08491882341F09091C00040
:100A300095FFFCCF8093C6003196F5CFECECF4E245
:100A400085919491FC012491222341F03091C000C2
:100A500035FFFCCF2093C6000196F4CFE0917410CF
:100A6000F0917510E758FF4E8191882339F09091ED
:100A7000C00095FFFCCF8093C600F6CFE9EFF9E008
:100A80008491882341F09091C00095FFFCCF809322
:100A9000C6003196F5CF8091C00085FFFCCF8AE07B
:100AA0008093C6000E94C13F75C18090F70A909064
:100AB000F80AA090F90AB090FA0A20912C0B309114
:100AC0002D0B40912E0B50912F0BC501B4010F94AB
:100AD000A3912DEC3CEC4CEC5DE30F948094181644
:100AE00014F00C94A35A80922C0B90922D0BA09290
:100AF0002E0BB0922F0B8CE29BE00E942BFE60E04D
:100B000080E00E94E54346C10E94C2322091140B4E
:100B10003091150B4091160B5091170B0F94A49127
:100B20006093200B7093210B8093220B9093230BE7
:100B30000C94B65B0E94C2322091180B3091190BB5
:100B400040911A0B50911B0B0F94A4916093240BAE
:100B50007093250B8093260B9093270B0C94C35B0B
:100B60000E94C23220911C0B30911D0B40911E0B34
:100B700050911F0B0F94A4916093280B7093290B35
:100B800080932A0B90932B0B0C94C45C711028C09B
:100B9000662031F181E08093A7120F94DC096B018C
:100BA0007C0180E00F94DC09AB01BC019701860158
:100BB00087EA92E10E94CB329B01AC016091280B45
:100BC0007091290B80912A0B90912B0B0F94A3917C
:100BD0006093280B7093290B80932A0B90932B0B17
:100BE0008091B21B882321F084E190E00F94AB390F
:100BF0001092870BE6EEFCE08491882341F09091FF
:100C0000C00095FFFCCF8093C6003196F5CF0E94BF
:100C10007C56EAEDFCE08491882341F09091C0007D
:100C200095FFFCCF8093C6003196F5CF0E94E25627
:100C3000EEECFCE08491882341F09091C00095FF98
:100C4000FCCF8093C6003196F5CF0E943E572ACF45
:100C500020E030E040E85FE360912C0B70912D0BB9
:100C600080912E0B90912F0B0F94A49160932C0BDD
:100C700070932D0B80932E0B90932F0BE090280BED
:100C8000F090290B00912A0B10912B0B2091240B33
:100C90003091250B4091260B5091270B6091200B32
:100CA0007091210B8091220B9091230BECE0FBE0E3
:100CB000FF93EF93812C912CA8ECAA2EA3E4BA2EDB
:100CC000BCE2CB2EBBE0DB2E0E94DEEF0F900F903C
:100CD0000C94AE670F94031B81E00E94F14680E004
:100CE0000F94BC3B0C94F76B0E947F32AB01BC01AC
:100CF0004093390E50933A0E60933B0E70933C0E26
:100D000084E89DE00E940795CDCE0E94C2320F94E8
:100D1000EC928B010C94296E0F94554DEEE7F5E2A1
:100D2000859194910F943D3FE8EEF5E28591949181
:100D3000BE016F5F7F4F0F94653D41E050E062E080
:100D400080E00F943139E6EEF5E2859194910F94AD
:100D5000B84E0C94C46E0F946D0988E50E9455320C
:100D6000882319F0179A1092110B89E50E945532C9
:100D7000882319F0169A1092120B8AE50E945532B8
:100D800085E40E945532882311F40C948873149AD8
:100D90000C948873CB5ADF4F0FB6F894DEBF0FBEAA
:100DA000CDBFDF91CF911F910F91FF90EF90DF901A
:100DB000CF90BF90AF909F908F907F906F905F90FB
:100DC0004F903F902F9008950F931F93CF93DF93F1
:100DD0001F92CDB7DEB78091800B9091810B892B4C
:100DE000A1F00F94B0890091C20A1091C30A20911A
:100DF000C40A3091C50A601B710B820B930B693ECC
:100E000073408105910508F0B1C08091800B9091ED
:100E1000810B892B11F41092880B8091540B88233D
:100E200019F00E94163F7EC00E9436AF60E08BE949
:100E30009BE00E94EFA58091701090917110892B1A
:100E400009F470C010926F1080919B0B8823B1F051
:100E5000009174101091751007581F4E63E17DE0EA
:100E6000C8010F94EF9A892B09F5B8018BE99BE033
:100E70000E943EA580919C0B882319F00E949A57EE
:100E800031C0E0E8F5E285919491FC0124912223A0
:100E900041F03091C00035FFFCCF2093C600019691
:100EA000F4CF8091C00085FFFCCF19C060E08BE9D2
:100EB0009BE00E94E5A6ECEEF5E285919491FC01A1
:100EC0002491222341F03091C00035FFFCCF2093C4
:100ED000C6000196F4CF8091C00085FFFCCF8AE068
:100EE0008093C60080916F1081111CC0809170109A
:100EF00090917110892BB1F0F89410E090E0E0919E
:100F00007410F0917510EA58FF4E8081823011F410
:100F10001181928199830E94BDAC812F99810E9499
:100F2000A0FE78940F94031B8091B31B882311F0CB
:100F300081E001C080E00E94F1460E9430FF80E025
:100F40000F94BC3B0E948EB60F94F6278091F81A3E
:100F5000882319F11092F81A61E08EE09DE00F905D
:100F6000DF91CF911F910F910C9493AD81E080930D
:100F7000880B8091800B9091810B01979093810B4E
:100F80008093800B0F94B0896093C20A7093C30A58
:100F90008093C40A9093C50A38CF0F90DF91CF9108
:100FA0001F910F9108959F92AF92BF92CF92DF92BF
:100FB000EF92FF920F931F93CF93DF931F921F9295
:100FC000CDB7DEB78DE99FE00F94F89D6093200BBD
:100FD0007093210B8093220B9093230B81EA9FE067
:100FE0000F94F89D6093240B7093250B8093260B30
:100FF0009093270B8DE89FE00F94F89D6B017C0187
:1010000083E79FE00F94FD9D8C012FE832EC45EFC4
:101010005FE3C701B6010F94A4916B017C0167E007
:1010200074E0601B710B04E0769567950A95E1F713
:1010300080E090E00F941D932091781930917919F8
:1010400040917A1950917B190F9484929B01AC01C5
:10105000C701B6010F94A4916093280B7093290BDC
:1010600080932A0B90932B0B80E1E0E2FBE0ABEE48
:10107000BAE001900D928A95E1F7EDE5F8E08491F0
:10108000882341F09091C00095FFFCCF8093C6006B
:101090003196F5CF0E947C560E948AC61092A71204
:1010A000A5E7EA2EAFE0FA2ED12CB3E0BB2EAA249E
:1010B000A39417E0C12E8D2D6B2D0F942097082F30
:1010C000992E42E050E0B701CE0101960F94E09DC9
:1010D00069817A816115710511F0A092A7122C2DFA
:1010E000020380011124090D111D97FC1A95000FB0
:1010F000111F000F111F09551D4E882777FD809580
:10110000982F0F941F932FE632E143E85AE30F9490
:101110005295F8016183728383839483D394F2E0C0
:10112000EF0EF11C29E0D212C6CF8091A7128823BE
:1011300021F087EA92E10E9494E4EBE2F8E08491E6
:10114000882341F09091C00095FFFCCF8093C600AA
:101150003196F5CF0E943E570E9488E3E090280B1D
:10116000F090290B00912A0B10912B0B2091240B4E
:101170003091250B4091260B5091270B6091200B4D
:101180007091210B8091220B9091230BECE2CE2EDB
:10119000EBE0DE2E0E948CFC81E08093110B17980F
:1011A0008093120B16988093130B1598E9EFF7E0D4
:1011B0008491882341F09091C00095FFFCCF8093EB
:1011C000C6003196F5CF0E94E2568CE89FE00F945E
:1011D000F09DE0910C0BF0E0EE0FFF1FE955F54E8E
:1011E00090E0918380838BE89FE00F94F09D90E0E6
:1011F0009093A61A8093A51A0F900F90DF91CF912C
:101200001F910F91FF90EF90DF90CF90BF90AF9024
:101210009F900895FF920F931F93CF93DF93CDB7C5
:10122000DEB76E970FB6F894DEBF0FBECDBFF82EB7
:1012300081E00F94293D82E00F94BC3BEAE5F5E2A2
:10124000859194910F943D3AAEDEE0910C0BF0E065
:10125000EE0FFF1FE955F54E81818F9380818F93AB
:101260008DE399E09F938F938E010F5F1F4F1F9324
:101270000F930F94C49B60E0C8010E9493AD8091CE
:10128000A61A8F938091A51A8F9324E339E03F9398
:101290002F931F930F930F94C49B60E0C8010E948B
:1012A00093AD0FB6F894DEBF0FBECDBF20E030E0A7
:1012B00048EC51E46091280B7091290B80912A0B26
:1012C00090912B0B0F947D9287FF05C061E088E21F
:1012D00099E00E9493AD61E080E299E00E9493ADB5
:1012E000E0910C0BF0E0EE0FFF1FE955F54E818108
:1012F0008F9380818F9327E139E03F932F931F9342
:101300000F930F94C49B60E0C8010E9493AD80913D
:10131000A61A8F938091A51A8F932EE039E03F9300
:101320002F931F930F930F94C49B60E0C8010E94FA
:1013300093AD61E08AE099E00E9493AD0FB6F89416
:10134000DEBF0FBECDBFF11005C061E08FEF98E0AA
:101350000E9493AD61E083EF98E00E9493AD60E05E
:1013600085EA9FE00F94029EEBEDF8E084918823DC
:1013700041F09091C00095FFFCCF8093C60031965C
:10138000F5CFE2ECF8E08491882341F09091C00021
:1013900095FFFCCF8093C6003196F5CF4091200B8E
:1013A0005091210B6091220B7091230B22E030E0D1
:1013B0008AED99E00E94A531E9EAF8E0849188235A
:1013C00041F09091C00095FFFCCF8093C60031960C
:1013D000F5CF4091240B5091250B6091260B709115
:1013E000270B22E030E08AED99E00E94A5310E94AF
:1013F0005153EFE8F8E08491882341F09091C000C8
:1014000095FFFCCF8093C6003196F5CF4091280B15
:101410005091290B60912A0B70912B0B22E030E048
:101420008AED99E00E94A4316E960FB6F894DEBF63
:101430000FBECDBFDF91CF911F910F91FF90089507
:10144000CF92DF92EF92FF920F94813B4BEF5DE0E2
:1014500061E080E00F94B46A46EE5DE062E080E017
:101460000F94B46A84EC9FE00F94F09D8093B21BBC
:1014700060EB7BE181EC9FE00F9463392091B21B1C
:101480008091B01B9091B11B2F3F11F4009721F078
:101490008F3F2FEF920711F41092B21B019621F4A7
:1014A0001092B11B1092B01B8091B21B882341F0A7
:1014B00088E090E00F94AB3981E080935F0A02C02E
:1014C00010925F0A40E052EC61E070E08AED99E032
:1014D0000E94382FE0EEFDE08491882341F0909146
:1014E000C00095FFFCCF8093C6003196F5CF809168
:1014F000C00085FFFCCF8AE08093C6002EE73EE067
:10150000F9018491882341F09091C00095FFFCCFB0
:101510008093C6003196F5CF44B740FF17C0EEE682
:10152000F5E285919491FC015491552341F060912D
:10153000C00065FFFCCF5093C6000196F4CF8091A8
:10154000C00085FFFCCF8AE08093C60041FF17C032
:10155000EAEFF5E285919491FC015491552341F015
:101560006091C00065FFFCCF5093C6000196F4CF98
:101570008091C00085FFFCCF8AE08093C60042FFC7
:1015800017C0E6E3F6E285919491FC01549155234E
:1015900041F06091C00065FFFCCF5093C6000196FA
:1015A000F4CF8091C00085FFFCCF8AE08093C60015
:1015B00043FF17C0EEEBF4E285919491FC01549146
:1015C000552341F06091C00065FFFCCF5093C600E9
:1015D0000196F4CF8091C00085FFFCCF8AE0809314
:1015E000C60045FF17C0E4EFF4E285919491FC0139
:1015F0004491442341F05091C00055FFFCCF4093EB
:10160000C6000196F4CF8091C00085FFFCCF8AE030
:101610008093C60014BEF9018491EEE7FEE08823B2
:1016200049F09091C00095FFFCCF8093C6003196A1
:101630008491F5CFE6E2F6E285919491FC01449124
:10164000442341F05091C00055FFFCCF4093C600A9
:101650000196F4CFEBECFDE08491882341F090916A
:10166000C00095FFFCCF8093C6003196F5CFECE625
:10167000F6E285919491FC014491442341F050910C
:10168000C00055FFFCCF4093C6000196F4CFE4EBB9
:10169000FDE08491882341F09091C00095FFFCCF3C
:1016A0008093C6003196F5CF8091C00085FFFCCFB6
:1016B0008AE08093C600E9EAFDE08491882341F046
:1016C0009091C00095FFFCCF8093C6003196F5CF76
:1016D000EDE9FDE08491882341F09091C00095FFF1
:1016E000FCCF8093C6003196F5CF8091C00085FF76
:1016F000FCCF8AE08093C600F9012491EEE7FEE07A
:10170000222349F08091C00085FFFCCF2093C600C2
:1017100031962491F5CFE0EEF5E285919491FC01AC
:101720002491222341F03091C00035FFFCCF20935B
:10173000C6000196F4CF0E946C9A4AE050E0BC01CA
:101740008AED99E00E94A630E2E7F5E28591949156
:10175000FC012491222341F03091C00035FFFCCFE1
:101760002093C6000196F4CF4AE050E060E775E0B0
:101770008AED99E00E94A6308091C00085FFFCCFE1
:101780008AE08093C60060E084E190E00E94E72652
:101790000E94839A0F94BE120E94D1ED8FEF9FE0BA
:1017A0000F94F09D91E0811101C090E09093121B85
:1017B00089E69FE00F94F09D882329F00E94C236AD
:1017C0006AED75E004C00E94D4366FEE75E08AEDD4
:1017D00099E00E949930E4E0F6E08191882339F0A5
:1017E0009091C00095FFFCCF8093C600F6CF68ECC7
:1017F00088EC0E947DEA7C014AE050E0BC018AED61
:1018000099E00E94AD3087E69FE00F94F09DEF28AD
:1018100039F0882329F00E94D0B462E176E004C058
:101820000E94E7B46BE276E08AED99E00E9499307D
:101830000F94810B48E85DE061E080E00F94B46AAA
:1018400043E75DE062E080E00F94B46A0E94FCC56B
:101850008091000186FD3AC0FFEF23ED80E3F15057
:1018600020408040E1F700C000008091000186FD2B
:101870002DC00F94263985E69DE00F94B84E8091D7
:1018800001018460809301019FB7F8948091020167
:101890008460809302019FBF8091000186FFFCCF8E
:1018A0009FB7F894809102018B7F809302019FBFC4
:1018B0009FEFE7EAF1E69150E040F040E1F700C029
:1018C00000000F94D03F60E00E94E3363D9AE8E4C8
:1018D000FDE08491882341F09091C00095FFFCCFFA
:1018E0008093C6003196F5CF83E40F9406294AE031
:1018F00050E0BC018AED99E00E9403319FB7F89453
:1019000080910B01846080930B019FBF83E40F944F
:10191000062908967C0124E0F694E7942A95E1F7DD
:10192000E114F10491F0429A62E070E080E090E00E
:101930000F94DF89429862E070E080E090E00F94BD
:10194000DF8921E0E21AF108EBCFEBE2FDE08491C0
:10195000882341F09091C00095FFFCCF8093C60092
:101960003196F5CF83E40F9406294AE050E0BC019C
:101970008AED99E00E940331159884EC9FE00F9462
:10198000F09D8093B21B60EB7BE181EC9FE00F94B4
:1019900063392091B21B8091B01B9091B11B2F3FF6
:1019A00011F4009721F08F3FEFEF9E0711F4109292
:1019B000B21B019621F41092B11B1092B01B8091C2
:1019C000B21B882321F088E090E00F94AB398BEBB9
:1019D0009FE00F94F09D91E0813009F090E09093AA
:1019E000610D8BE99BE00E94D4A18CEF9FE00F94E6
:1019F000F89D6F3F7F4F8F4F9F4FB9F488EF9FE067
:101A00000F94F89D6F3F7F4F8F4F9F4F71F484EF7E
:101A10009FE00F94F89D6F3F7F4F8F4F9F4F29F4AA
:101A200060E08FEF9FE00F94209E8EEF9FE00F9479
:101A3000F09D8093550B81110F9414698FEA9FE0FC
:101A40000F94F09D8F3F41F460E08FEA9FE00F9488
:101A5000209E1092860B06C091E0811101C090E09B
:101A60009093860B86EA9FE00F94F09D8F3F29F4B8
:101A700060E086EA9FE00F94209E85EA9FE00F9445
:101A8000F09D8F3F29F460E085EA9FE00F94209E4F
:101A90000E94924A0E9406530E9487520E944FB5AC
:101AA00069E87BE087EA9FE00F9463396BE87BE0AD
:101AB00089EA9FE00F9463396DE87BE08BEA9FE051
:101AC0000F9463396FE87BE08DEA9FE00F946339F0
:101AD00081E00F94293D0F94263982E00F94BC3B9E
:101AE0000F94008985EA9FE00F94F09D813009F002
:101AF00049C00F94031BC0908D1AD0908E1AE090AD
:101B00008F1AF090901A8BE89FE00F94F09D682F49
:101B100070E080E090E00F941D9320E030E040EA18
:101B200050E40F94A3919B01AC01C701B6010F943F
:101B30008094181614F481E00BC0E8E5F5E2859175
:101B4000949140E060E00F94B361882331F080E02D
:101B5000FF90EF90DF90CF905DCB60E085EA9FE053
:101B60000F94029E81E00F94293D82E00F94BC3BCC
:101B7000ECEAF4E285919491FF90EF90DF90CF90A2
:101B80000D943D3AFF90EF90DF90CF90089524E8B8
:101B900036E0FC01318320832781222319F004964B
:101BA0000C94EA9508958F929F92AF92BF92CF9234
:101BB000DF92EF92FF920F931F93CF93DF938C01ED
:101BC0008B519E4FE4DF680189E8C80ED11CC11417
:101BD000D10419F1780181E4E81A8EEFF80AE701DF
:101BE00057018FE1A81AB10834E8832E36E0932E0E
:101BF000CC15DD0591F0FE01EE19FF09EA0DFB1D84
:101C000091828082FE0178978081811102C06F9756
